:020000040800F2
:10000000000001109537040859FF02083DC200089E
:100010009938040899380408993804080000000049
:10002000000000000000000000000000A50503081B
:10003000A1050308000000009D05030899D80008E9
:10004000993804089938040899380408993804083C
:100050009938040899380408F16501081D670108FA
:10006000E1660108A56601086966010821A2000889
:1000700011A2000801A20008F1A10008E1A10008F6
:10008000CDA10008B9A100089938040899380408DE
:100090009938040899380408993804082D6601082D
:1000A0009938040875CF00089938040885CF0008EE
:1000B00065CF000855CF000899380408F9BA000840
:1000C000FFBA0008EDBA0008F3BA0008993804082E
:1000D0009938040805DB00089938040865DA000837
:1000E000B5650108993804080D0E030815CF0008FE
:1000F00025CF00089938040835CF0008A5A10008CD
:10010000993804089938040845CF0008993804083C
:10011000C5D9000899380408E1590208C5590208F0
:1001200091A100087DA1000869A1000855A100085F
:1001300041A100089938040899380408993804083E
:100140009938040899380408993804085DFF0208B2
:100150002DA1000819A1000805A1000825D9000853
:10016000E1BA0008E7BA0008993804089938040889
:10017000993804089938040899380408993804080B
:080180009938040899380408BD
:080188002C330400010000000B
:1001900002020300741F0020701F002000000000F6
:1001A0000000000016000800C4240020DC24002009
:1001B00000000000400600080E020200E8240020B3
:1001C000EC24002000000000480600081D0001008B
:1001D000A826002030270020000000004A06000862
:1001E00027000400C826002034270020000000005B
:1001F0004C0600080101040080270020203B00205D
:10020000000000000000000008020900443A00203D
:10021000243B0020000000003357010806020C00B8
:10022000BC3A0020303B002000000000575B010872
:1002300007020200F03A00203C3B002000000000D2
:1002400050060008FF010100183B0020403B002041
:10025000000000005206000802000C00C83A00200E
:10026000443B00200000000000000000F7010600F1
:10027000383A0020503B00200000000054060008DF
:1002800003123300173E0020E43D00200000000070
:100290005C06000825005A00303D00208A3D002001
:1002A0000000000000000000F6110C00243D0020BA
:1002B000183D0020000000009006000815007000A6
:1002C000383C0020A83C0020000000000000000096
:1002D0002A006000783B0020D83B0020000000008E
:1002E000C95903080A020A00F03F0020004000201C
:1002F000000000009C0600081E000400484000208A
:100300008043002000000000A606000822000C0028
:10031000E84200208443002000000000AA060008F4
:100320001B00F4009C440020185500200000000031
:100330007162020826000E001C5600200C56002098
:1003400000000000999302080B2010004C4600208A
:100350002C56002000000000B60600081000030024
:100360004C5800205858002000000000C606000825
:10037000280010003C5800205C58002000000000BD
:10038000BDC40208230010002C5800206C58002027
:1003900000000000C9BF0308190005002458002010
:1003A0007C58002000000000CA060008F811010077
:1003B000205800208458002000000000D0060008CB
:1003C000000104001C580020885800200000000094
:1003D000D20600082F001100085800208C58002079
:1003E00000000000D606000814000200405C002057
:1003F000885D002000000000E8060008040080007E
:10040000CC7E0020607F0020000000000000000083
:10041000F90104003C610020E07F002000000000A2
:1004200025570108FD01240014610020E47F00200D
:10043000000000006DBF0008060016008C5D002063
:100440000880002000000000555A030803010A003C
:10045000149100202091002000000000EA0600080E
:10046000FB010100F0AD0020B4AE00200000000050
:10047000F5BB0008FC010900BCAC0020B8AE0020B0
:1004800000000000C1BB00080A10120090AC002060
:10049000C4AE002000000000F40600083400100084
:1004A000E0A30020D8AE002000000000F1590308AE
:1004B00011000C0078980020E8AE00200000000039
:1004C0006DE9010818102C0010980020F4AE0020EF
:1004D00000000000F10004080D003C003C980020E2
:1004E00020AF00200000000049DF030805100600CF
:1004F00094B0002074B1002000000000080700083C
:100500000E20EA0074AF00207CB100200000000043
:10051000355A03081300040018B1002068B2002007
:100520000000000010070008020103005FAF002078
:100530006CB20020000000002DE901080120080035
:1005400070B8002090B800200000000014070008D8
:100550001A00080054B8002098B8002000000000DD
:100560001C070008FE010900C4BA0020D8BA002008
:1005700000000000FDBB00081F000E0044BC00206E
:1005800018BE00200000000024070008050201003A
:100590002CBC002028BE002000000000320700080C
:1005A0000902010089BE0020B8BE00200000000042
:1005B0003407000812200C00D0C6002088C7002095
:1005C00000000000360700080C002400DCC60020F4
:1005D00094C700200000000005E9010800020500A2
:1005E000B0C60020B8C700200000000000000000D6
:1005F0002C00100010CA002000CA002000000000DB
:100600006DFE03082B00240044CA002020CA0020ED
:10061000000000003DFE03082900500034C90020FE
:1006200068CA002000000000000000000300010074
:100630006CCC002074CC0020000000000000000002
:10064000C409000019012828000000002003000050
:10065000013C000024010000000000000000000038
:10066000000000000000000000000000000000008A
:10067000000000000000000000000000000000007A
:100680000000000000000000000000000000010069
:1006900000000000000000000000000000004A010F
:1006A000B400D601000000000100C800141E0100C3
:1006B00064002C0128002B21231E6400020000008E
:1006C00001000A01290000010500000028010000C6
:1006D0000400900100000000000000000000000085
:1006E00000000000000000000300040101006C167F
:1006F0000000000000300100005A000000009001DE
:100700002C01C8006400000020000201000000006D
:1007100008000000E8036400040A00017E05EA0501
:10072000B4053200000000000000010000000005D8
:10073000000000002E000000000100054134534479
:020740000000B7
:10074200500100000700000002000000000000004D
:10075200000000000102030406070809685E0C009D
:10076200FF0000000101000028800408C0AA04085C
:1007720000000000000000003880040840800408E7
:100782000000000001200000448004084C8004089E
:100792000000000001400000508004086494040836
:1007A20000000000012000005C800408688004084A
:1007B20000000000040000006C8004087880040837
:1007C20000000000040000007C80040878A40408F3
:1007D2000000000001000000020100000000803F54
:1007E2000000803F00000000000000000000000048
:1007F2000000803FFC4F04080508040000000000D0
:10080200607A04080C7704084C7A0408000000009F
:100812002850040805080A0000000000607A040855
:100822000C770408F073040800000000FFFFFFFFCC
:10083200000001FFFF00000009024300020100C0A6
:100842003209040000010202010005240010010522
:100852002401000104240202052406000107058286
:10086200030800FF09040100020A00000007050155
:10087200024000000705810240000000FF00000066
:10088200010000005C9B0408000000000000000062
:1008920041E90108A08601000400000000000000F8
:1008A2000000000000000000000000000000000046
:1008B2000000000000000000DCAC0408B09A04084C
:1008C20000000000397D01087D00000006000000E4
:1008D2000000000000000000000000000000000016
:1008E200000000000000000000000000C4AA04088C
:1008F200000000000000000059E80008E8030000C2
:1009020003000000000000000000000000000000E2
:1009120000000000000000000000000000000000D5
:10092200CCAA04080000000000000000915B03084C
:10093200102700000300000000000000000000007B
:1009420000000000000000000000000000000000A5
:1009520000000000D8AA040800000000F1C9030842
:1009620049EC0008204E00000500000000000000D5
:100972000000000000000000000000000000000075
:100982000000000000000000E89C040800000000D5
:10099200000000001DDC000810270000010000001C
:1009A2000000000000000000000000000000000045
:1009B200000000000000000000000000DCAA0408A3
:1009C20000000000000000008DBB0008E8030000EA
:1009D2000500000000000000000000000000000010
:1009E2000000000000000000000000000000000005
:1009F200E8AA04080000000000000000A1EB0108C2
:100A0200204E000003000000000000000000000073
:100A120000000000000000000000000000000000D4
:100A220000000000F8AA0408000000000000000016
:100A3200A9E90108204E00000300000000000000A8
:100A420000000000000000000000000000000000A4
:100A5200000000000000000008AB040800000000D5
:100A620000000000690C0108400D030003000000B3
:100A72000000000000000000000000000000000074
:100A8200000000000000000000000000209C04089C
:100A920000000000000000005DEA030810270000CB
:100AA2000100000000000000000000000000000043
:100AB2000000000000000000000000000000000034
:100AC200CC9A04080000000000000000BD74020877
:100AD20010270000030000000000000000000000DA
:100AE2000000000000000000000000000000000004
:100AF2000000000018AB0408000000000000000025
:100B0200E5E60008A08601000100000000000000E8
:100B120000000000000000000000000000000000D3
:100B22000000000000000000BC9A04080000000061
:100B32000000000005E6000850C3000001000000AC
:100B420000000000000000000000000000000000A3
:100B520000000000000000000000000020AB0408BC
:100B620000000000000000006DE10008A861000024
:100B72000100000000000000000000000000000072
:100B82000000000000000000000000000000000063
:100B92002CAB0408000000000000000039FB030831
:100BA200A08601000100000000000000000000001B
:100BB2000000000000000000000000000000000033
:100BC20000000000F09C040800000000000000008B
:100BD200D90E0108A00F0000010000000000000073
:100BE2000000000000000000000000000000000003
:100BF200000000000000000038AB04080000000004
:100C020000000000219602081027000001000000E9
:100C120000000000000000000000000000000000D2
:100C2200000000000000000000000000489C0408D2
:100C32000000000000000000A9ED0108A00F000064
:100C420001000000000000000000000000000000A1
:100C52000000000000000000000000000000000092
:100C6200549D040800000000000000006D99030874
:100C7200102700000100000000000000000000003A
:100C82000000000000000000000000000000000062
:100C920000000000989A0408000000000000000014
:100CA200354D03081A410000010000000000000059
:100CB2000000000000000000000000000000000032
:100CC200000000000000000044AB04080000000027
:100CD2000000000089D20108400D0300000000005E
:100CE2000000000000000000000000000000000002
:100CF2000000000000000000000000004CAB0408EF
:100D0200000000000000000025D20108400D030091
:100D120000000000000000000000000000000000D1
:100D220000000000000000000000000000000000C1
:100D320054AB0408000000000000000069F803083A
:100D4200A086010003000000000000000000000077
:100D52000000000000000000000000000000000091
:100D620000000000000101010100000000600240DB
:100D72001060024000000000000B00000000200094
:100D820000000000000000000060024028600240F5
:100D920000000000060C000000002000000000001F
:100DA20000000000006002404060024000000000BD
:100DB200100D0000000020000000000000000000F4
:100DC200006002405860024000000000160E000061
:100DD200000020000000000000000000006002404F
:100DE2007060024000000000200F000000002000A0
:100DF2000000000000000000006002408860024025
:100E0200000000002610000000002000000000008A
:100E12000000000000600240A060024000000000EC
:100E2200301100000000200000000000000000005F
:100E320000600240B860024000000000362F00004F
:100E420000002000000000000000000000640240DA
:100E52001064024000000000003800000000400062
:100E6200000000000000000000640240286402400C
:100E720000000000063900000000400000000000F1
:100E820000000000006402404064024000000000D4
:100E9200103A0000000040000000000000000000C6
:100EA200006402405864024000000000163B00004B
:100EB200000040000000000000000000006402404A
:100EC2007064024000000000203C0000000040006E
:100ED200000000000000000000640240886402403C
:100EE2000000000026440000000040000000000056
:100EF2000000000000640240A06402400000000004
:100F0200304500000000400000000000000000002A
:100F120000640240B864024000000000364600004F
:100F22000000400000000000000000000000803FC0
:100F32000403090412010002020200408304405724
:100F4200000201020301000031160308591B0308C5
:100F5200AD1603089D0F03081D120308AD0F030809
:100F6200C90F0308750F0308650F0308000000008E
:100F7200000000000000000001020304010203045B
:100F8200060708090D150308F57E0208457E0208CA
:100F920000000000997A0208997D0208197E020871
:100FA200017D020800000000000000008D7A0208A6
:100FB20025FA020821FA02081DFA020811FA0208AB
:100FC2000DFA020819FA020815FA020899FA02083B
:100FD2008DFA020865FA020879FA020851FA020843
:100FE2003DFA020829FA02080100000020700020E0
:100FF200702D720000000000000000004416002066
:10100200FFFFFFFFFA0000000100000001000000E6
:1010120000B0040800000000000000000000000012
:1010220000000000EBAF040804000000B7B303089F
:10103200000000000000000008B0040801000000E9
:10104200000000000000000000000000000000009E
:101052000D00000000000000000000000000000081
:10106200929000200100C40900000000909000202E
:101072000100C409000000008E9000200100C40994
:10108200000000008C9000200100C4090000000054
:10109200889000200100C409000000008A9000200E
:1010A2000100C40900000000869000200100C4096C
:1010B20000000000849000200100C409000000002C
:1010C2000000000000000000D0080020E8BB002063
:1010D2009CFF2C0100000000901700200A00000075
:1010E200F07304082CBE0020E0150C17000000006D
:1010F20092170020080000000C77040891170020C6
:1011020005000000607A04082EBE002002000000E4
:10111200087404089AB000200100FF7F010000005B
:1011220093B00020020000001474040868AF00208D
:10113200030000002474040867AF002003000000CD
:101142002474040866B000200000F40101000000CD
:1011520064B000200000F4010100000062B0002031
:101162000000F4010100000060B000200000F40162
:10117200010000005EB0002000FF01007EB00020F0
:10118200E803D0070A0000007CB0002000640100E0
:101192000A00000078B000200064010077B000204F
:1011A200006401007DB00020006401000A0000001C
:1011B20076B00020006401000A0000007BB000202D
:1011C200006401000A0000007AB0002000640100FF
:1011D2000A00000079B00020006401000A0000004B
:1011E20075B0002000FF01000A00000074B000206A
:1011F20000FF01000A00000070AF00200000F401AF
:10120200010000006EAF00200000F40101000000A8
:101212006CAF00200000F401010000006AAF002062
:101222000000F4010100000070B000201400E80387
:10123200010000006EB00020E803307501000000DC
:101242006DB0002000C801006CB0002000C8010091
:101252006BB0002000C801006AB0002000640100E9
:101262000A00000069B0002000FF01000A0000002F
:1012720089B0002000C8010088B0002000C8010029
:1012820087B0002000C8010086B0002000C801001D
:1012920085B0002000C8010084B0002000C8010011
:1012A20083B0002000C8010082B0002000C8010005
:1012B20081B0002000C801003CB00408000000001A
:1012C2000000000000000000000000004CB0040814
:1012D2000900000000000000740900200400000062
:1012E20054B0040809000000000000006809002052
:1012F2000400000024B404080900000000000000FB
:101302005C090020040000005CB004080900000031
:1013120000000000500900200400000060B0040832
:101322000900000000000000440900200400000041
:1013320068B004080900000000000000380900201D
:101342000400000070B00408090000000000000062
:101352002C0900200400000078B0040809000000F5
:1013620000000000200900200400000008B004086A
:10137200010000000000000000000000000000006A
:10138200000000000D00000000000000000000004E
:101392000000000080B1040800000000000000000E
:1013A200000000000000000090B1040805000000E9
:1013B2000000000066AF00200000000008B0040832
:1013C200010000000000000000000000000000001A
:1013D200000000000D0000000000000000000000FE
:1013E2000000000098B104080000000000000000A6
:1013F2000000000000000000C0AA04080000000075
:10140200000000004F17002004000000A4B10408EF
:101412000C00000019B40308C809002000000000F5
:101422008CB604080C00000021AE0308BC090020A1
:1014320000000000A8B104080C00000005AE03087B
:10144200B009002000000000B0B10408080000004C
:1014520000000000A409002004000000B8B1040844
:101462000C00000051AD03089809002000000000A4
:10147200C0B1040809000000000000008C0900202F
:1014820004000000C8B10408030000004D4703082F
:10149200800900200000000008B0040801000000DC
:1014A200000000000000000000000000000000003A
:1014B2000D0000000000000000000000000000001D
:1014C200CCB1040800000000000000000000000091
:1014D20000000000DCB104080C0000000000000065
:1014E200E009002000000000E4B104080A00000046
:1014F200000000001CB1002000000000F0B1040850
:101502000A0000000000000024B1002000000000DA
:10151200F8B104080A000000000000002CB100200D
:101522000000000000B204080800000000000000F3
:10153200D40900200000000008B0040801000000E7
:101542000000000000000000000000000000000099
:101552000D0000000000000000000000000000007C
:1015620008B20408000000000000000000000000B3
:10157200000000001CB204080C0000000000000083
:10158200F8090020000000002CB20408040000004A
:1015920041490308000000000000000034B20408C2
:1015A2000C00000000000000EC0900200000000018
:1015B20048B20408040000002149030800000000AA
:1015C2000000000008B00408010000000000000054
:1015D2000000000000000000000000000D000000FC
:1015E20000000000000000000000000050B20408EB
:1015F20000000000000000000000000000000000E9
:1016020064B204080700000000000000340A002051
:101612000000000070B20408080000000000000092
:10162200280A0020000000007CB204080800000024
:10163200000000001C0A00200000000088B204081C
:101642000800000000000000100A00200000000056
:1016520094B204080800000000000000040A002000
:101662000000000008B004080100000000000000B3
:101672000000000000000000000000000D0000005B
:10168200000000000000000000000000A0B20408FA
:101692000000000000000000AF0800200000000071
:1016A200ACB204080B00000000000000AC0A0020ED
:1016B20000000000B4B204080B00000000000000AB
:1016C200A00A002000000000C0B204080B000000C5
:1016D20000000000940A002000000000CCB20408C0
:1016E2000B00000000000000880A0020000000003B
:1016F200D8B204080B000000000000007C0A0020A1
:1017020000000000E4B204080B000000000000002A
:10171200700A002000000000ECB204080B00000078
:1017220000000000640A002000000000F8B2040873
:1017320007000000000000005C0A0020000000001A
:1017420000B304080700000000000000540A002053
:10175200000000000CB304080B00000000000000B1
:10176200480A00200000000018B304080800000026
:10177200000000003C0A00200000000008B004083D
:101782000100000000000000000000000000000056
:10179200000000000D00000000000000000000003A
:1017A2000000000024B30408000000000000000054
:1017B200000000000000000038B304080800000028
:1017C20000000000DC0A00200000000044B304080E
:1017D2000800000000000000D00A00200000000005
:1017E20050B304080800000000000000C40A0020F2
:1017F200000000005CB304080800000000000000C4
:10180200B80A00200000000008B00408010000002F
:1018120000000000000000000000000000000000C6
:101822000D000000000000000000000000000000A9
:1018320064B304080000000000000000AC080020AF
:101842000000000074B304080B0000000000000058
:10185200240B00200000000080B304080B000000ED
:1018620000000000180B0020000000008CB30408E8
:101872000700000000000000100B00200000000024
:1018820098B304080700000000000000080B0020C5
:1018920000000000A4B304080700000000000000DC
:1018A200000B002000000000B0B304080800000094
:1018B20000000000F40A002000000000B8B3040891
:1018C2000800000000000000E80A002000000000FC
:1018D20008B0040801000000000000000000000041
:1018E20000000000000000000D00000000000000E9
:1018F2000000000000000000C0B304080000000067
:1019020000000000AC08002000000000CCB3040876
:101912000700000000000000700B00200000000023
:10192200D4B304080700000000000000680B002088
:1019320000000000DCB30408070000000000000003
:10194200600B002000000000E4B304080700000060
:1019520000000000580B002000000000ECB3040857
:101962000700000000000000500B002000000000F3
:10197200F4B304080700000000000000480B002038
:1019820000000000FCB30408070000000000000093
:10199200400B00200000000004B40408070000000F
:1019A20000000000380B0020000000000CB4040806
:1019B2000700000000000000300B002000000000C3
:1019C20008B0040801000000000000000000000050
:1019D20000000000000000000D00000000000000F8
:1019E200000000000000000000000000A9430308FE
:1019F200780B002064AF00201B0000003474040840
:101A020063AF00200A32010062AF002001FA010038
:101A12005EAF002000C801005CAF0020E803D007E1
:101A220001000000414952424F54463453440000E1
:101A3200BF430308F5480308540C00208DAD03088A
:101A420000000000A40C00203D4A030805460308DC
:101A5200800D0020E143030800000000200E00205A
:101A62006944030839440308AC0E0020F14403081A
:101A7200354503084C0F002072B00020010301001D
:101A820015440308F1430308641000209944030835
:101A920061490308F010002065450308B9490308AD
:101AA200B811002068B000200103010014B404083A
:101AB2000000000000000000000000000000000024
:101AC20020B404080800000000000000D812002022
:101AD2000000000028B40408070000000000000015
:101AE200D01200200000000038B4040807000000F3
:101AF20000000000C81200200000000044B40408E6
:101B02000700000000000000C012002000000000DA
:101B120050B404080C00000000000000B4120020C1
:101B2200000000005CB40408030000004D470308F5
:101B3200A81200200000000008B004080100000004
:101B42000000000000000000000000000000000093
:101B52000D00000000000000000000000000000076
:101B620064B404080000000000000000000000004F
:101B72000000000074B404080A0000000000000025
:101B820088800408000000007CB404080A000000F9
:101B920000000000088004080000000084B404086B
:101BA2000A000000000000008AB0002000000000CF
:101BB2008CB404080A00000000000000E4120020B7
:101BC2000000000008B0040801000000000000004E
:101BD2000000000000000000000000000D000000F6
:101BE20000000000000000000000000094B404089F
:101BF20000000000000000000000000000000000E3
:101C0200A8B40408030000004D470308081300208D
:101C120000000000B4B40408030000004D470308AC
:101C22009417002000000000BCB404080300000068
:101C32004D470308FC12002000000000C4B4040851
:101C4200030000004D470308F012002000000000CE
:101C520008B00408010000000000000000000000BD
:101C620000000000000000000D0000000000000065
:101C72000000000000000000D0B4040800000000D2
:101C8200000000000000000000000000DCB40408B6
:101C920007000000054A030864130020000000004A
:101CA200DCAC0408030000004D4703085813002071
:101CB20000000000E8B40408030000004D470308D8
:101CC2004C13002000000000F0B4040803000000E0
:101CD2004D4703084013002000000000F8B4040838
:101CE20007000000E9490308381300200000000043
:101CF200A8B60408030000004D4703082C13002077
:101D02000000000004B50408030000004D4703086A
:101D1200201300200000000010B50408030000009A
:101D22004D470308141300200000000008B0040807
:101D320001000000000000000000000000000000A0
:101D4200000000000D000000000000000000000084
:101D52000000000071430308394303086C1300209C
:101D6200D1450308000000002014002000000000FC
:101D720000000000AC140020A9450308214A030812
:101D8200381500201CB50408000000000000000007
:101D9200000000000000000028B504080300000055
:101DA2004D470308381600200000000030B5040833
:101DB200030000004D4703082C160020000000001D
:101DC2003CB50408030000004D470308201600201C
:101DD2000000000048B50408030000004D47030856
:101DE200141600200000000050B504080200000094
:101DF200954B0308000000000000000058B50408DD
:101E020002000000954B03080100000000000000E2
:101E120064B5040802000000954B030802000000AC
:101E220000000000000000000D00000000000000A3
:101E320000000000000000000000803F00000000E1
:101E420000000000000000000000803F00000000D1
:101E52000000000000000000000000000000000080
:101E62000000000000000000000000000000000070
:101E72000000803F000000000000000000000000A1
:101E820000FFFF0000000000AA5505010000012D1F
:101E9200202D2D202D2D2D2D202D2D2D2D0000001E
:101EA2000000000000000000000000000000AA5531
:101EB2000B010000AA5507010000AA550902000003
:101EC2000000000001000000C012AA5503009F009C
:101ED200010101003DAE03080000000008190020C6
:101EE200E0B604080000000000000000000000004E
:101EF20000000000C0AA040800000000000000006A
:101F0200481D0020040000008CB604080C000000EC
:101F1200CD480308301D002000000000A8B10408CD
:101F22000C000000A5480308241D0020000000004A
:101F3200B0B104080800000000000000181D0020D5
:101F420004000000B8B104080C00000015430308A7
:101F52000C1D002000000000C8B1040803000000AE
:101F62004D470308001D002000000000F0B60408E1
:101F7200030000004D470308F41C0020000000008D
:101F820008B004080100000000000000000000008A
:101F920000000000000000000D0000000000000032
:101FA2000000000000000000E0B60408000000008D
:101FB200000000000000000000000000C0AA0408A9
:101FC2000000000000000000481D00200400000086
:101FD20034B60408030000003DB40308E81C0020E6
:101FE20008000000B8B104080C0000001543030803
:101FF2000C1D002000000000C8B10408030000000E
:102002004D470308001D002000000000F0B6040840
:10201200030000004D470308F41C002000000000EC
:1020220008B00408010000000000000000000000E9
:1020320000000000000000000D0000000000000091
:102042000000000000000000F8B6040800000000D4
:10205200000000000000000000000000C0AA040808
:102062000000000000000000481D002004000000E5
:102072003CB60408030000004D4703083C1D002045
:102082000000000008B00408010000000000000089
:102092000000000000000000000000000D00000031
:1020A20000000000000000000000000032BE00201E
:1020B20088136F170100000034BE002088136F17C9
:1020C2000000000090B504080000000000000000BD
:1020D2000000000000000000A0B504080800000095
:1020E200000000007819002004000000ACB50408CC
:1020F20008000000000000006C1900200000000031
:10210200C8B10408040000007DB403080000000008
:102112000000000008B004080100000000000000F8
:102122000000000000000000000000000D000000A0
:1021320000000000000000000000000030BE00208F
:1021420088136F170100000024BC002088136F174A
:10215200000000009DAE030800000000841900206A
:1021620088BE002001000000207A040826BC00205E
:10217200010000002C7A04081CBC002002000000B0
:10218200347A0408DA900020000000000000000009
:10219200D89000200000000000000000D69000202F
:1021A2000000000000000000D490002000000000A9
:1021B20000000000D290002000000000000000009B
:1021C200D0900020000000000000000088170020CE
:1021D20000000000000000002FBE002002000000EE
:1021E200407A0408ECB5040800000000000000007A
:1021F2000000000000000000A0B504080800000074
:1022020000000000081A002004000000ACB5040819
:102212000800000000000000FC190020000000007F
:10222200C8B104080400000071AE030800000000F9
:102232000000000008B004080100000000000000D7
:102242000000000000000000000000000D0000007F
:10225200000000000000000000000000FCB50408BF
:10226200000000000000000000000000000000006C
:102272000CB604080C0000004D480308381A002070
:102282000400000018B604080C000000F54703081B
:102292002C1A00200400000024B604080C000000E0
:1022A20019480308201A00200000000030B6040874
:1022B200030000005DB40308141A002008000000A7
:1022C2003CB60408030000004D4703083C1D0020F3
:1022D2000000000008B00408010000000000000037
:1022E2000000000000000000000000000D000000DF
:1022F20000000000000000000000000000B0040820
:1023020000000000000000000000000000000000CB
:1023120044B604080400000099B403080000000059
:102322000000000008B004080100000000000000E6
:102332000000000000000000000000000D0000008E
:1023420000000000000000000000000094B6040835
:10235200000000000000000000000000000000007B
:10236200E89D04080C00000000000000981A0020FC
:1023720004000000A4B604080800000000000000E9
:102382008C1A002004000000B0B604080800000007
:1023920000000000801A002004000000B8B6040803
:1023A2000800000000000000741A00200400000071
:1023B200C0B604080800000000000000681A0020EF
:1023C20004000000C8B60408080000000000000075
:1023D2005C1A002004000000D0B6040808000000C7
:1023E20000000000501A002004000000D8B60408C3
:1023F2000800000000000000441A00200400000051
:1024020008B0040801000000000000000000000005
:1024120000000000000000000D00000000000000AD
:10242200000000000000000089AE03080000000068
:10243200A41A002000000000000000001C1B002065
:102442000000000000000000BC1B002022BC002095
:10245200040000004C7A040820BC0020E0150C1790
:10246200000000001FBC0020080000000C770408D8
:102472001EBC002005000000607A04080000000075
:10248200000000000C1C00202D202D2D202D2D2DB4
:102492002D202D2D2D000000000000000000000066
:1024A20000000000000000000101D60141C5030840
:1024B200000000000000000001000000801D00205C
:1024C200000000000000000000000000000000000A
:1024D20000000000000000000000000000000000FA
:1024E20000000000000000000000000000000000EA
:1024F20000000000000000000000000000000000DA
:1025020000000000000000000000000000000000C9
:1025120000000000000000000000000000000000B9
:102522004300000000000000000000000000000066
:102532000000000000000000000000000000000099
:102542004300000000000000000000000000000046
:102552000000000000000000000000000000000079
:102562004300000000000000000000000000000026
:102572000000000000000000000000000000000059
:102582004300000000000000000000000000000006
:102592000000000000000000000000000000000039
:1025A20043000000000000000000000000000000E6
:1025B2000000000000000000000000000000000019
:1025C20043000000000000000000000000000000C6
:1025D20000000000000000000000000000000000F9
:1025E20043000000000000000000000000000000A6
:1025F20000000000000000000000000000000000D9
:10260200373B0408133B040800000000D2BA040858
:10261200E7AF04087AA604087AA604087AA6040892
:102622007AA604087AA604087AA604087AA60408F8
:102632007AA604087AA60408FFFFFFFFFFFFFFFF48
:10264200FFFFFFFFFFFF0000010041534349490024
:102652000000000000000000000000000000000078
:1026620000000000000000000000415343494900FF
:102672000000000000000000000000000000000058
:102682000000000000000000000000000100000047
:108000000378407840EA032010FB01F04FF48071C0
:1080100090FBF1F000F30F0000B270472DE9F74F2D
:108020006A4CDFF8ACE123880091DEF80010B4F967
:108030000480C3EB21125B00C3EBE103B4F902102F
:1080400052435943131308FB03F84FEAA83808EBCF
:10805000E12101EB8102B1F5FA3802F180024FEA29
:10806000E1794FEA222349F1FF39B4F9082001935D
:10807000A8FB08AB08FB09F30BEB430BA161D3177B
:1080800002FB09F108FB0311A2FB08230B441F03A9
:10809000160347EA1257B4F90A2002FB0BF1D31773
:1080A0000AFB03130546A2FB0A011944020A42EA2D
:1080B000016292194FEA2123E6887B41003243F5A1
:1080C0000043A2FB060106FB03114A10CB1752EA3C
:1080D00003016FD0B4F91060B4F90E00F71706FB76
:1080E0000BF10AFB0711A6FB0AAB8B4400FB09F658
:1080F000C11708FB0161A0FB08898944DEF8041060
:108100004FEA4846C1F5801E4FEA494747EAD8374B
:108110001AEB060AB4F90C8076464BEB070BF717FF
:1081200000264FEACE70F90716EB0A064FEAC80799
:1081300041EA5E0147EB0B0740F6354E861B61EBCB
:108140000707A6FB0E010EFB07113BF04FF9B4F930
:1081500016204E13470B47EAC14702FB06FED31712
:1081600007FB03EEA2FB07237344564307FB03669A
:10817000A2FB07233344560E46EAC3163218B4F95D
:1081800014604FEA636747EB01037143F71700FB85
:108190000717A6FB00013944C60C46EA413692197E
:1081A0004FEAE147B4F912607B41100A40EA0360EC
:1081B000320112180DB1120A2A60009B13B11A463F
:1081C000019B136003B0BDE8F08F00BFD85C0020B6
:1081D000501F0020704770472DE9F041324E334F59
:1081E00074893B89B6F91420B6F902E0B6F90E801D
:1081F000B6F920C01B1B34895C43E313B6F9124067
:108200001A44E4020A2594FBF2F41C44B6F9043043
:10821000F4616543A4F57A6404FB04F204FB0EFEEA
:108220005C43B6F90C30121302FB08F85A431214DF
:108230004FEAEE2E02EB64340EEBE828B6F900E0CC
:10824000F388FE680234A41008EB8E0804F500449D
:1082500008FA0CF863434CF2503208F10208DC0BC8
:10826000A6EBA80642FA0CF3734353BF5B00B3FBC3
:10827000F4F35B00B3FBF4F31A1202FB02F440F6D2
:10828000DE3262430A4C12145C4302EB244208358E
:1082900002F6CF622D1103EB221300B1036001B18E
:1082A0000D60BDE8F08100BFA05C0020501F0020E1
:1082B00043E3FFFF2DE9F04F654B664EB3F80AC06C
:1082C0003469B3F8048087B04FEA0C2A0590188906
:1082D000B4EB0A0A4FF000024FF0000565EB020B09
:1082E000A0FB0A4500FB0B55E00940EA45604FEA58
:1082F000084407198E46D8884FEAE51141EB020879
:10830000A0FB0A45CDE90278B3F8028000FB0B55CB
:10831000200A40EA05604FEAC83410EB04084FEA2F
:10832000252141EB02099A89A2FB0A0102FB0B11EC
:10833000C20D42EA412212F5FA604FEAE15343F1DD
:108340000001B0F5FA6FCDE9000171F10001B4460A
:108350005EDA0524A2FB040104FB031100FB03F415
:1083600002FB0144DDE90267A0FB020121444D103C
:108370004FEA3004361B4FEA900444EA817467EBFD
:1083800005078D10B8EB040869EB0509DDE9004528
:1083900031484FF0FF31844275EB0101CDE90267AE
:1083A00023DA40F6AC5012184FF000014B4102FBAB
:1083B00003F1A2FB022303EB4103D900D000101A02
:1083C00041EA527163EB0101341847EB0105CDE935
:1083D00002450B24A2FB040104FB031149104FEAE0
:1083E0003000B8EB000869EB01090AFB0BF3DDE98B
:1083F0000001AAFB0AAB0BEB430B4FEADA7242EA2D
:108400004B02801A4FEAEB7361EB0301CDE90001E7
:10841000DCF81410A1FB082301FB0933540D5D1592
:1084200044EAC324DDE90223A21A65EB03031D46D7
:10843000D30B059A43EA454302B11360BEF1000F26
:1084400002D0009BCEF8003007B0BDE8F08F00BF2F
:10845000C45C0020501F002024FAFFFF4FF400638B
:10846000838270474FF40063838270473122F42186
:108470000EF09EBA044B93F820209201343202F0A1
:10848000FC02F4210EF094BAA05C00202E22F4210C
:108490000EF08EBA012248210EF08ABA012258212C
:1084A0000EF086BA012380F8453070474FF48053B0
:1084B00083827047BFF34F8F0549064BCA6802F4A9
:1084C000E0621343CB60BFF34F8F00BFFDE700BFF7
:1084D00000ED00E00400FA0570B4037B04681F2B74
:1084E00008D9203B2021626801FA03F31A421CD10B
:1084F00070BC70472021226801FA03F31A42F7D0BA
:10850000426914495C2000FB021251685689CD680B
:108510000868296821F001012960828992B222EA63
:1085200006028281A36070BC7047426909495C20E1
:1085300000FB021251685689CD680868296821F04D
:1085400001012960828992B222EA06028281E360F7
:1085500070BC7047B45D00202B4B1978002951D0B6
:108560002A4B30B41C68988800226262A5899A80E0
:10857000284380B20129A08143D09C689889626217
:10858000A589284380B20229A0819A8139D01C692B
:10859000988A6262A589284380B20329A0819A82C1
:1085A0002FD09C69988B6262A589284380B20429E8
:1085B000A0819A8325D01C6A988C6262A589284381
:1085C00080B20529A0819A841BD09C6A988D626232
:1085D000A589284380B20629A0819A8511D01C6BF9
:1085E000988E6262A589284380B20729A0819A8665
:1085F00007D0986B998F42628489214389B2818127
:108600009A8730BC704700BF9460002098600020BB
:1086100010B4037B01681F2B09D9203B20224C6832
:1086200002FA03F31C4214D15DF8044B7047202278
:108630000C6802FA03F31C42F6D00C4A406800248E
:10864000147002685DF8044B22F0010202608B6036
:108650007047064A40680024147002685DF8044BB5
:1086600022F001020260CB60704700BF99440020F5
:10867000F0B5C40022189200AE498B585B689D8A01
:10868000ADB2EEB2F7070A445CD4B70732D5BFF3F8
:108690005F8F167EF6B2012E00F0C780A64D1A8BB2
:1086A000BFF35F8F221801EB8202167E022E00F0CC
:1086B000D580221801EB8202167E032E00F08880FE
:1086C0009A8895F9186092B242F480629A802218D2
:1086D00001EB8202127E013296425BD1AA7E002615
:1086E0006E76002A40F09580204401EB8000002344
:1086F0004375F0BD77074ED416F0400600F0C980F0
:108700008D4D1E8A95F918E0176AF6B207F80E60CB
:108710005FFA8EFE0EF1010C4FFA8CFC177E85F885
:1087200018C00CF103029742664600F01C81221823
:1087300001EB8202127E9445C9D10EF1020676B297
:108740002E76C4E71E887C4D26F400663604360C6F
:108750001E801E88B6B246F480661E80967E002774
:108760002F76002E48D06E7E002E42D0221801EBCC
:1087700082020126127E6E76022A00F0B98022184B
:1087800001EB8202927D42F001021A82204401EB49
:108790008000037EF0BD684D967E0127AF76002EE7
:1087A00073D06E7E002E7BD1221801EB8202527EA6
:1087B000002A00F0A3801A882E7E92B2013642F47D
:1087C000007276B21A802E761A88D205FCD47EE723
:1087D000927E002A3FF474AF6A7E002A3FF470AFA5
:1087E0009A8895F9186022F480621204120C9A801B
:1087F0006DE7D27DFF2AB9D0221801EB8202967D67
:1088000006F0FE061E82D37DFF2BBFD0FF232B7602
:10881000BCE79A8822F4407212042044120C01EB47
:1088200080009A8000234375F0BD927E424D002A5D
:108830003FF435AF6A7E002A3FF431AF1A8822F444
:1088400080621204120C1A80BFF35F8F1A8B1A8891
:10885000AE7692B242F400721A8031E7927E002A1C
:108860003FF427AF6A7E002A3FF423AF1A8895F9B8
:10887000186022F480621204120C1A809A8822F482
:1088800080621204120C9A8021E76A7E002A8BD043
:1088900091E715F0800F284D3AD195F9186016E749
:1088A000167ED2F820E01F88022E95F9186045D96F
:1088B00027F480673F043F0C1F801F8AFFB20EF829
:1088C00006701F88D2F820E0BFB247F400771F80FF
:1088D000F2B21F8A561C76B2FFB20EF806709F885D
:1088E000961CBAB276B242F480622E769A806BE71A
:1088F0001A8892B242F400621A8040E71A8895F909
:10890000186092B242F4807201271A806F765BE79A
:1089100095F91870B7F1FF3F2CD0D669F65D1E822D
:1089200092F818E001377AB2964516462A767FF417
:10893000CEAEA3E7503A0020501F0020BFB247F44C
:1089400000771F801F8AFFB20EF80670F6B21F8AEA
:10895000D2F820E0721C52B20336FFB276B20EF8A3
:1089600002702E7630E79A8822F480621204120C8C
:108970009A80DCE6D77D1F822E76957E1DB9127E09
:10898000002A7FF403AF9A8822F480621204120C4A
:108990009A80FBE637B506236A4604460D460C303E
:1089A00003210DF03DFF024690B1B4F91A1068465C
:1089B000FFF726FB2880B4F91E100DF10200FFF727
:1089C0001FFBA880B4F91C1001A8FFF719FB6880F1
:1089D000104603B030BD2DE9F04F4FF4807385B0E1
:1089E00043838383C38300F10C050446322004F0E3
:1089F000B5FE1122002128460DF0DAFF6022012188
:108A000028460DF0D5FF642004F0A8FE02A92046F8
:108A10000027FFF7BFFF0123B946B8463E46019342
:108A2000012E14BF11221222002128460DF0C0FF92
:108A3000002E0CBF4FF0010B4FF0FF3B4FF00A0A26
:108A40000122022128460DF0B3FF142004F086FE17
:108A500002A92046FFF79EFFBDF90A20BDF90C00D0
:108A6000BDF90810224B82420BFB0299A8BF0246B7
:108A70008A42A8BF0A469A4201FB0B880BFB00778B
:108A800033DB01200DF082F9BAF1010AD8D10136A9
:108A9000022EC5D1174B93FBF8F893FBF9F970221E
:108AA000A3F58423002193FBF7F7A4F81A80A4F818
:108AB0001C90E78328460DF07BFF202201212846E9
:108AC0000DF076FF0022314628460DF071FF64203C
:108AD00004F044FE019B23B94FF480736383A383A6
:108AE000E383012005B0BDE8F08F00230193CEE7BA
:108AF00001F0FFFF00D03B0007B506236A46F721CF
:108B00000DF08EFE9DF801309DF800100B4A1B0100
:108B100043EA01339DF8021043EA111353609DF8B4
:108B200004309DF803101B0143EA01339DF8051042
:108B300043EA1113136003B05DF804FB501F0020DB
:108B400007B5032301AAF6210DF06AFE9DF8053052
:108B50009DF804201B0243EA02439DF806201343BC
:108B6000054AB2F92020C2F10802D340034AD3607B
:108B700003B05DF804FB00BFA05C0020501F002084
:108B800007B5022301AAF6210DF04AFE9DF8042044
:108B90009DF8053043EA0223024A138103B05DF8D1
:108BA00004FB00BF501F002007B5032301AA0021CA
:108BB0000DF036FE9DF805309DF804001B0243EAD7
:108BC00000439DF80600184303B05DF804FB08B5A8
:108BD000FFF7EAFF014B586108BD00BF501F00209E
:108BE00008B5FFF7E1FF014B186108BD501F0020D9
:108BF00070B582B00446062310306A4643210DF05A
:108C00000FFEA8B19DF804009DF800609DF80110CA
:108C10009DF802509DF803209DF8053041EA062199
:108C200043EA002342EA052221876287A3870120C5
:108C300002B070BD70B582B00446062308306A46A3
:108C40003B210DF0EDFDA8B19DF804009DF80060FA
:108C50009DF801109DF802509DF803209DF8053005
:108C600041EA062143EA002342EA0522E182228307
:108C70006383012002B070BDF0B5876983B00646FA
:108C800017B13B68BA885A837069DFF8A4E083891A
:108C9000C3244FF47A734FF0060C6D464FF6FF7104
:108CA0000EF1010E03E0013B9BB28B4220D0028902
:108CB0009207F8D5A3B283814FF47A7302E0A3B28E
:108CC0008B4215D00289D20703F1FF34F7D5828990
:108CD00092B20DB12A700135BCF1000F0BD00CF12E
:108CE000FF3CFF24BEF1000FE1D09EF80040D7E723
:108CF0000DF07AFDB76917B13B68BA881A839DF801
:108D000005009DF801509DF802109DF803409DF864
:108D100004209DF8063041EA052143EA002342EA97
:108D20000422012031877287B38703B0F0BD00BFF2
:108D3000484C0408F8B5057B466903681F2D29D9FE
:108D4000A5F120045F682021A1400F422A4613D0DC
:108D50001022A240D960DA605A68E240D10703D5F8
:108D6000012202FA04F4DC600446304604F01AFFE3
:108D7000227B23681F2A20D9A2F1200008215A68EB
:108D80008140114200D0D9600422596882400A42D1
:108D900021D1F8BD20211C68A9400C422A460CD0E4
:108DA0001022AA4099609A601A68EA40D207DBD57F
:108DB000012202FA05F59D60D6E708211868914066
:108DC000014200D099600421186801FA02F20242BF
:108DD00003D09A60F8BDDA60F8BDF8BD144B984234
:108DE00024D003F58063984220D0028822F040020C
:108DF0001204120C0280028822F038031B041B0CA0
:108E000059B141F48071002991FAA1F2B2FA82F1CC
:108E100008BF4FF0FF310139C9000B439BB20380FB
:108E200003889BB243F04003038070474908DCE7A6
:108E30000038004008B540F2E93300E0A3B10289F0
:108E4000013B12F0020F9BB2F8D089B2818140F24F
:108E5000E93300E043B10289013B12F0010F9BB2FC
:108E6000F8D08089C0B208BD0DF0BEFCC0B208BD0C
:108E70000C4B984213D0A3F5806398420FD003F5B2
:108E8000804398420BD003F58063984207D003F5E6
:108E90008063984203D0044B186840087047024B27
:108EA0001868704700040140B0A40020F0B5774B6B
:108EB000774A87B01968914200AF00F0DB80002349
:108EC000744A3B607B60136843F48033136003E0B3
:108ED0003B68B3F5A04F09D0136803F400337B60FF
:108EE0003B6801333B607B68002BF1D0694B1B680A
:108EF00013F4003318BF01237B607B68012B7BD008
:108F0000654D644B654AEA606549586F654A08607B
:108F1000AA605E6B644C654A654826F080065E6315
:108F20005E6F46F080765E67196B0C431C63596B6D
:108F30005963996B9963196C41F05B5141F47B1152
:108F400041F41F6141F00F011964596C07F11804D5
:108F50000A4348F2FF715A6444F8101D0026214666
:108F60000123FB733E737E73BE7329F011F9214612
:108F70004FF6FF734F48BB6029F00AF94FF6FF73B5
:108F800021464D48BB6029F003F921464B4829F0A2
:108F9000FFF821464A4829F0FBF82146494829F0C4
:108FA000F7F82146484829F0F3F82146474829F0C8
:108FB000EFF82146464829F0EBF8204628F0A6FEB7
:108FC000444B454C1B68BA6844484549A4FB0343DD
:108FD0009B09A0FB0202013B920CB3F1807F0A6067
:108FE00007D2404AF0200721536085F8230096609D
:108FF00011601C37BD46F0BD264B3B4D1A6C3B48FB
:1090000042F080521A642C684268816844F44044FB
:109010002C609C689C609C6844F400449C609C6844
:1090200044F4A0549C600068120642EA801242F4A4
:109030008002490842F00802013942EA01425A60BE
:109040001A6842F080721A601A689201FCD52849A9
:10905000104A40F205700860996821F00301996098
:10906000996841F002019960936803F00C03082BA2
:10907000FAD145E700221A6062B61E4B1B6883F3E3
:1090800008881D4B1B689847FEE700BFFCFF0120C6
:10909000EFBEADDE0038024000ED00E00005FA054D
:1090A0003861002000000008FF916700335F07006F
:1090B000000002400004024000080240000C024090
:1090C000001002400014024000180240001C024040
:1090D00000200240B0A40020D34D621083DE1B4369
:1090E00064BA002010E000E00070004000000020A2
:1090F000003C02400000FF1F0400FF1F08B5054BA5
:109100001B6803B19847044B044A1A6072B6FFF714
:10911000D1F900BFA4580020FCFF0120EFBEADDE56
:109120002DE9F04F90F8553085B00646002B40F001
:10913000A58002AB0093A34BDB7E002B00F0F980EF
:109140007069A14B984200F06684A04A90420CBF1F
:1091500030223822038823F040031B041B0C0380B9
:1091600003889BB223F038031A43028003889BB222
:1091700043F040030380B36996F84E4013B11A6878
:109180009B88538340F2E93304E0013B9BB2002B00
:1091900000F0EC8402899707F7D51A23838140F207
:1091A000E93304E0013B9BB2002B00F0DF8402892D
:1091B000D507F7D5838940F2E93304E0013B9BB240
:1091C000002B00F0CF8402899107F7D5A4B28481E7
:1091D00040F2E93304E0013B9BB2002B00F0C28473
:1091E0000289D207F7D58389B36913B11A689B88BE
:1091F0001383012004F058FA7369734A934200F014
:10920000C68472498B4214BF082100211A8822F0BB
:1092100040021204120C1A801A8892B222F038020C
:10922000114319801988009A89B241F040011980D0
:1092300006F11000062343210DF0F2FA002800F099
:1092400017849DF80A509DF80B309DF808409DF852
:1092500009109DF80C009DF80D2043EA05231BB270
:1092600041EA042142EA002273873187B2875BB268
:10927000013300F0D38305B0BDE8F08F1D09013D37
:10928000032D03F00F0300F27984514A32F81500E0
:1092900040FA03F2D70740F17184012404FA03F382
:1092A000013B18403AF0F2F84A4B4B4A5B5D1844D8
:1092B00012EBC00500F0628400232021EB71A9713C
:1092C00052F83000454A00F13F4303F57E039B0A04
:1092D000D25C02F01F035209032A04FA03F300F0E0
:1092E000A984042A00F0A084022A00F09784AB88A5
:1092F000029302A900230091039328F049FF31460D
:10930000374B41F80C3F28462FF0C4FCAB88B3FA2A
:1093100083F3C3F11F03012212FA03F33FF40BAFEF
:1093200030490A6813430B60264BDB7E002B7FF429
:1093300007AF7069244B984200F08484234A90421E
:109340000CBF30223822038823F040031B041B0C7F
:10935000038003889BB223F038031A4302800388FA
:109360009BB243F040030380B36913B11A689B8832
:10937000538340F2E93304E0013B9BB2002B00F041
:10938000108402899407F7D56B23838140F2E93377
:1093900004E0013B9BB2002B00F003840289D1075B
:1093A000F7D5838940F2E93304E0013B9BB2002BFF
:1093B00000F0E18302899207F7D58023838140F290
:1093C000E93316E0501F002000380040003C004008
:1093D0008C76040888760408A0B80020007504087C
:1093E000A5840008003C0140013B9BB2002B00F02B
:1093F000C2830289D707F7D58389B36913B11A6885
:109400009B8813839623A24CA24DDFF890A2A2481A
:10941000DFF88CC201964FF010084FF47A77994626
:10942000DAF80430C3F30803002B40F07E83EFF337
:109430001183002B40F079832368816800BF226884
:109440009342F9D12A6807FB02FEAEEB010EBEFB88
:10945000F2FE07FB03EE0126DAF80430C3F308033B
:10946000002B40F00983EFF31183002B40F00483BD
:109470002368816800BF22689342F9D1D5F800B013
:1094800007FB0BF2521AB2FBFBF207FB0323A3EB21
:109490000E03B3F57A7FDFD3B9F10109C0D1019E84
:1094A000B36913B11A689B885383706940F2E9333A
:1094B00004E0013B9BB2002B00F09E8302899707DA
:1094C000F7D56823838140F2E93304E0013B9BB286
:1094D000002B00F091830289D107F7D5838940F2F0
:1094E000E93304E0013B9BB2002B00F07F8302894B
:1094F0009207F7D50323838140F2E93304E0013B6F
:109500009BB2002B00F072830289D707F7D58389BD
:10951000B36913B11A689B8813839623DFF87CA183
:109520005D48DFF87CC101964FF010084FF47A7760
:109530009946DAF80430C3F30803002B40F0D882D0
:10954000EFF31183002B40F0D3822368816800BFC2
:1095500022689342F9D12A6807FB02FEAEEB010EA6
:10956000BEFBF2FE07FB03EE0126DAF80430C3F37C
:109570000803002B40F09E82EFF31183002B40F094
:1095800099822368816800BF22689342F9D1D5F897
:1095900000B007FB0BF2521AB2FBFBF207FB0323EE
:1095A000A3EB0E03B3F57A7FDFD3B9F10109C0D184
:1095B000019EB36913B11A689B885383706940F2A6
:1095C000E93304E0013B9BB2002B00F00B830289DE
:1095D0009407F7D56B23838140F2E93304E0013B24
:1095E0009BB2002B00F0FE820289D107F7D5838958
:1095F00040F2E93304E0013B9BB2002B00F0CA8249
:1096000002899207F7D50323838140F2E93304E00E
:10961000013B9BB2002B00F0BD820289D707F7D532
:109620008389B36913B11A689B8813830F2004F0F0
:109630003BF8B36913B11A689B885383706940F291
:10964000E93304E0013B9BB2002B00F0A6820289C3
:109650009507F7D56A23838140F2E93304E0013BA3
:109660009BB2002B00F099820289D407F7D5838939
:1096700040F2E93304E0013B9BB2002B00F09682FC
:1096800002899107F7D51023838140F2E9330EE078
:1096900060BA002064BA002010E000E000ED00E0B5
:1096A0005CBA0020013B9BB2002B00F07F82028954
:1096B000D207F7D58389B36913B11A689B881383DE
:1096C0000F2003F0F1FFB36913B11A689B8853832D
:1096D000706940F2E93304E0013B9BB2002B00F0DB
:1096E000688202899707F7D56C23838140F2E933BA
:1096F00004E0013B9BB2002B00F05B820289D5079E
:10970000F7D5838940F2E93304E0013B9BB2002B9B
:1097100000F0538202899407F7D50023838140F239
:10972000E93304E0013B9BB2002B00F04682028942
:10973000D107F7D58389B36913B11A689B8813835E
:109740000F2003F0B1FFB36996F8504013B11A68C7
:109750009B885383706940F2E93304E0013B9BB27C
:10976000002B00F02D8202899207F7D519238381FF
:1097700040F2E93304E0013B9BB2002B00F0208271
:109780000289D707F7D5838940F2E93304E0013B2A
:109790009BB2002B00F0188202899507F7D5A4B27E
:1097A000848140F2E93304E0013B9BB2002B00F0DE
:1097B0000B820289D107F7D58389B36913B11A687F
:1097C0009B8813830F2003F06FFFB36913B11A68EE
:1097D0009B885383706940F2E93304E0013B9BB2FC
:1097E000002B00F0F48102899207F7D51B238381B7
:1097F00040F2E93304E0013B9BB2002B00F0E7812B
:109800000289D707F7D5838940F2E93304E0013BA9
:109810009BB2002B00F0DF8102899507F7D5182352
:10982000838140F2E93304E0013B9BB2002B00F05E
:10983000D2810289D407F7D58389B36913B11A6835
:109840009B8813830F2003F02FFFB36913B11A68AD
:109850009B885383706940F2E93304E0013B9BB27B
:10986000002B00F0BB8102899107F7D51C2383816F
:1098700040F2E93304E0013B9BB2002B00F0AE81E3
:109880000289D207F7D5838940F2E93304E0013B2E
:109890009BB2002B00F0B48102899707F7D5102303
:1098A000838140F2E93304E0013B9BB2002B00F0DE
:1098B000A7810289D507F7D58389B36913B11A68DF
:1098C0009B8813830F2003F0EFFEB36913B11A686E
:1098D0009B885383706940F2E93304E0013B9BB2FB
:1098E000002B00F0908102899407F7D537238381FC
:1098F00040F2E93304E0013B9BB2002B00F083818E
:109900000289D107F7D5838940F2E93304E0013BAE
:109910009BB2002B00F07B8102899207F7D51023C0
:10992000838140F2E93304E0013B9BB2002B00F05D
:109930006E810289D707F7D58389B36913B11A6895
:109940009B8813830F2003F0AFFEB36913B11A682D
:109950009B885383706940F2E93304E0013B9BB27A
:10996000002B00F0578102899507F7D538238381B2
:1099700040F2E93304E0013B9BB2002B00F04A8146
:109980000289D407F7D5838940F2E93304E0013B2B
:109990009BB2002B00F02D8102899107F7D501239E
:1099A000838140F2E93304E0013B9BB2002B00F0DD
:1099B00020810289D207F7D58389B36913B11A6868
:1099C0009B8813830F2003F06FFE73699F4A9342B5
:1099D00000F036819E498B4214BF082100211A886D
:1099E00022F040021204120C1A801A8892B222F05D
:1099F0003802114319801A8892B242F040021A804C
:109A0000012003F051FE934A70690123D3768F4BF6
:109A100098427FF49AAB3022FFF79CBB96F938301E
:109A200001337FF428AC0A2632202EF075FE4FF465
:109A3000FA7503F0EDFD044603F0EAFD001BB0F5F6
:109A40007A7FF9D3013DF4D107202EF0C7FC4FF403
:109A50007A7503F0DDFD044603F0DAFD001BB0F576
:109A60007A7FF9D3013DF4D1013EDDD1FFF746FB0A
:109A7000B6F93A30FFF7FBBBEFF3118188F3128898
:109A8000D0F808B00368DB0344BFCCF80060D0F81E
:109A900008B02368DCF80020C9B281F31188296876
:109AA0001A4407FB01F3A3EB0B03B3FBF1F307FB32
:109AB0000233ECE4EFF3118188F31288D0F808B098
:109AC0000368DB0344BFCCF80060D0F808B023681B
:109AD000DCF80020C9B281F3118829681A4407FB19
:109AE00001F3A3EB0B03B3FBF1F307FB023357E5E1
:109AF000EFF3118288F3128881680368DE0303D5CF
:109B00000123CCF8003081682368DCF80060D2B211
:109B100082F311882A6806EB030E07FB02F35B1A37
:109B2000B3FBF2F307FB0E3E1EE5EFF3118288F361
:109B3000128881680368DE0303D50123CCF8003066
:109B400081682368DCF80060D2B282F311882A6849
:109B500006EB030E07FB02F35B1AB3FBF2F307FB02
:109B60000E3E78E40CF040FEFFF73EBB0CF03CFEEE
:109B70007069FFF720BB0CF037FE3EE43146364BF0
:109B800041F80C3F00202FF085F8FFF7D2BA0021F2
:109B9000FFF73CBB0CF028FE43E50CF025FE706996
:109BA00066E50CF021FE7069FFF7FCBB0CF01CFEB3
:109BB00081E50CF019FE7069A4E50CF015FEBAE51C
:109BC0000CF012FE7069DFE50CF00EFEF5E50CF00E
:109BD0000BFE706918E60CF007FE2EE60CF004FE92
:109BE000706951E60CF000FE706901E50CF0FCFDB7
:109BF0008EE40CF0F9FDE0E60CF0F6FD70696EE421
:109C00000CF0F2FD59E60CF0EFFD70697CE60CF00B
:109C1000EBFD92E60CF0E8FD7069B5E60F4A516C79
:109C20000B435364FFF763BB0C4A116B0B43136385
:109C3000FFF75DBB094A116C0B431364FFF757BB79
:109C40000021CCE63022FFF77EBB00BF0038004089
:109C5000003C0040501F0020A5840008003802404E
:109C600008B5034B1B6803B1984772B6FEF722FC98
:109C7000A4580020084B10B507281B68C8BF14382B
:109C800018440C46007E0CF013FA20B12146BDE8C2
:109C900010400CF063BC10BD403A002038B50C4BAE
:109CA00007281B68CCBFA0F11404044623440546D2
:109CB000187E0CF0FDF950B128220134C471827174
:109CC0002EF028FB28460021BDE83840D2E738BDF9
:109CD000403A0020064A00235168814202F11C02EA
:109CE00004D00133102BF7D100207047D8B2704751
:109CF0002C06002070B50F4C0F4DC0EBC00004EBDC
:109D00008004286B26693043286382B09209667B01
:109D1000A1600025012101A863618DF804608DF820
:109D200005208DF806508DF8071027F0A7FF02B028
:109D300070BD00BF2C06002000380240074BC0EB6E
:109D4000C00030B403EB8000054C0569236B2B4346
:109D500023630176427630BC704700BF2C0600209A
:109D6000003802402DE9F04F534C54F8204083B0A6
:109D7000002C00F09C80256E002D00F09A80174684
:109D80004E4A9846064604F166032869226004F2AA
:109D900066226361A2614FF400736A68A160E360A8
:109DA0002361A265A24668B1FFF794FF721CD2B28C
:109DB0000C21FFF7C3FFA36DA9682A69626304330E
:109DC000E1636365E868A0B1FFF784FF721C814618
:109DD000D2B20B21FFF7B2FF2346EA7F384948464B
:109DE000FFF788FFA36DA968EA68A26304332164C2
:109DF000236594F865000CF05BF9814694F86400E3
:109E00000CF056F98346287F00284DD118F0080F32
:109E100036D1BA070DD5B9F1000F0AD00B22731C49
:109E200089F8062089F8073048466A7F22210CF01D
:109E300005FAFB0715D4E36B7BB995F82020A97FC1
:109E40008DF8063001A8930901228DF805308DF8B0
:109E500004108DF8072027F011FF504603B0BDE82D
:109E6000F08FBBF1000FE6D001360C238BF80760B2
:109E70008BF8063058466A7F22210CF0DFF9DAE7CA
:109E80000136F6B2B9F1000F04D00B2389F8076050
:109E900089F8063018F0100F484614BF022112212D
:109EA0006A7F0CF0CBF9C6E72EF016FAAEE7A246B1
:109EB000D3E7AA46D1E700BF203A0020504C04085F
:109EC000358D000800B97047F0B599B006462FF0FF
:109ED00031F9804DC36802682A600446002B00F007
:109EE000DE8030460CF0E4F87B4BD86118B12922B3
:109EF00000238271C371227A2A210CF09FF928680D
:109F000003F000FA2EF0E8F92E68338823F00103FD
:109F10001B041B0C33803046FEF7AAFF6F4A9042A9
:109F2000034600F2BE80002218A9DFF8D4E16C4F8E
:109F300021F85C2D304601326A4EB3FBF2F3032266
:109F4000B3FBF6F3002602939BB2B3FBF2F3AEF839
:109F500000305B003B80ADF80C60ADF806608DF81A
:109F60000E602FF09FF8E379ADF812606022990738
:109F7000ADF814600696ADF81C60ADF81E60ADF843
:109F80002060ADF82260ADF8102040F1948013F00D
:109F9000010F0CBF324608220423ADF81E20ADF895
:109FA0001430002304AA61792868069302F06EFD3C
:109FB000617928684C4E2FF045F82B68B3F844209F
:109FC0006FEA42426FEA524292B2A3F844201A88E2
:109FD00092B242F080021A80E2796079198C92077D
:109FE0004CBF04220122824092B289B221EA0201CE
:109FF0001984198C89B20A431A841A8892B242F0E1
:10A0000001021A80207D00222921FFF797FE60229D
:10A010003649207D0023FFF76DFEE068306027F0B1
:10A020005DFF3068036823F00103036027F056FFEB
:10A0300009A827F015FF2B6862792169306809911A
:10A0400034331A4440F22A330A920D934FF480625B
:10A05000274B0F920B9340224FF48053002709A9FE
:10A060000C9210934FF480424FF4403311920E97AC
:10A070001297139327F006FF637929681D480C2B6C
:10A080009CBF1D4A32F813708B8932689BB23B43E8
:10A090008B811368012143F010031360017019B024
:10A0A000F0BD00F1B77202F558521449B2FBF1F25B
:10A0B000013A92B238E713F0010F0CBF00210221E0
:10A0C00001224FF48073ADF81C10ADF81220ADF8EA
:10A0D000203066E7B4BE0020501F0020FF6BDC027A
:10A0E000AABE002000350C00B0BE0020118600087A
:10A0F00070480020ACBE0020446D0408006CDC02F7
:10A10000A8BE00200348D0F8AC3113B100F5D270DE
:10A11000184770472C0600200348D0F8903113B13F
:10A1200000F5C470184770472C0600200348D0F88B
:10A13000743113B100F5B670184770472C06002033
:10A140000348D0F8583113B100F5A870184770478C
:10A150002C0600200348D0F83C3113B100F59A706A
:10A16000184770472C0600200348D0F8203113B15F
:10A1700000F58C70184770472C0600200348D0F873
:10A1800004310BB1FC301847704700BF2C0600208B
:10A190000348D0F8E8300BB1E0301847704700BFF3
:10A1A0002C0600200348D0F8CC300BB1C43018473F
:10A1B000704700BF2C0600200348D0F8B0300BB128
:10A1C000A8301847704700BF2C0600200348D0F87D
:10A1D00094300BB18C301847704700BF2C0600201C
:10A1E0000248836F0BB17030184770472C0600206F
:10A1F0000248C36D0BB15430184770472C0600203D
:10A200000248036C0BB13830184770472C06002009
:10A210000248436A0BB11C30184770472C060020D7
:10A220000248836803B11847704700BF2C0600201E
:10A23000F8B584894FF6FF764FF47A7433B319B3C7
:10A240000F78013101E0B44218D00589013CAD0717
:10A25000A4B2F8D5BCB284814FF47A7402E0BCB2E7
:10A26000B4420BD00589ED0704F1FF37F7D5858996
:10A27000ADB20AB115700132013BDFE70CF0B4FA60
:10A28000003018BF0120F8BDFF27DEE70120F8BD30
:10A29000F8B50501684C694B625961199A4204EBA3
:10A2A000050704BF01230B730646387A2EF014F815
:10A2B0003B7A03F01F015B090122032B02FA01F232
:10A2C0006DD0042B66D0022B5CD06319013618794F
:10A2D0000BF0EEFEF6B2074610B11223C671837181
:10A2E000631958790BF0E4FE10B11323C671837122
:10A2F000631998790BF0DCFE10B11423C6718371D9
:10A3000066190A21F27938460BF098FF70790BF044
:10A31000CFFEF2790A210BF091FFB0790BF0C8FE65
:10A32000F2790A210BF08AFF6359454A934247D0DC
:10A33000444A934250D0414A934259D0424A9342B0
:10A3400062D0424A93426BD0414A93422CD02C4473
:10A35000227BE2B901200222198801F4415141F423
:10A3600045710A4302431A809A8B22F40062120458
:10A37000120C07219A8319821A8892B242F0400285
:10A380001A80F8BD334B596A0A435A629DE7002090
:10A390000246E1E72F4B19690A431A6195E72D4BF5
:10A3A000196A0A431A6290E702F564424FF40010FA
:10A3B000536A43F40013536227F098FC6359C6E7CD
:10A3C00002F584324FF48050536A43F48053536251
:10A3D00027F08CFC6359BAE702F500324FF4804055
:10A3E000136A43F48043136227F088FC6359AEE795
:10A3F00002F5FE324FF40040136A43F40043136247
:10A4000027F07CFC6359A2E702F582324FF400503A
:10A41000536A43F40053536227F068FC635996E78C
:10A4200002F568424FF48010536A43F4801353627C
:10A4300027F05CFC63598AE76C5C0020003C00401C
:10A44000003001400038004000340140005001401D
:10A450000054014000380240431C00F014812DE9F3
:10A46000F04F4FEAC00808EB00039B00DFF8F4A2AE
:10A470005AF803B087B00AEB0304BBF1000F00F0F9
:10A48000FF8014330AEB03010022DBF804704AF862
:10A4900003204A608A60CA600346A56801900133C0
:10A4A000D4F80C90DBB2002D00F0EE801522EB7199
:10A4B000AA71B9F1000F00F00081162289F8062078
:10A4C00089F807309BF80E002DF006FFBB8823F4B7
:10A4D00040731B041B0CBB8028460CF039F848461F
:10A4E0000CF036F8112128460BF02CFD11214846BE
:10A4F0000BF028FD0826642404E00A203CB103F098
:10A50000D3F8013C28460CF04BF80028F5D028463B
:10A510000CF018F80A2003F0C7F828460CF018F8D9
:10A520000A2003F0C1F8013EECD148460CF00AF8CD
:10A530000A2003F0B9F828460CF004F80A2003F0CA
:10A54000B3F828460CF004F80A2003F0ADF84846AA
:10A550000BF0FEFF019B08EB03040AEB8404284682
:10A56000637C002B0CBF1221322104220BF066FE0B
:10A57000637C002B0CBF12213221484604220BF0D1
:10A580005DFE704B9F4200F0B7806F4B9F4200F022
:10A59000BD806E4B9F4200F0A580BB8801996C4A3C
:10A5A0006C4C23F440731B041B0CBB803B88884419
:10A5B0000AEB880A9BB243F001039AF810103B8023
:10A5C000BD8802A8002918BF144627F09FFB049AF3
:10A5D0006148B2FBF4F325F03F05A0FB02122D0405
:10A5E000900C2D0C0543BD805C4C39884FF496725D
:10A5F00002FB00F284FB02409BB2D217002BC2EB9D
:10A60000A01221F0010108BF01230904013243F423
:10A610000043090C92B239803A84BB833B889BB2D9
:10A6200043F001033B803B8823F4816323F0020362
:10A630001B041B0C43F480634FF480423B803A813F
:10A640003B8823F080031B041B0C3B809BF81030DD
:10A650008DF808300024012302A88DF80B308DF806
:10A6600009408DF80A4027F009FB9BF80F308DF860
:10A67000083002A88DF809408DF80A4027F024FB25
:10A6800007B0BDE8F08F7047B9F1000F48D016222F
:10A6900089F8073089F806209BF80E002DF01CFE83
:10A6A000BB8823F440731B041B0C2846BB800BF0B3
:10A6B0004FFF48460BF04CFF18E79BF80E002DF0BB
:10A6C0000BFEBB8823F440731B041B0CBB80284685
:10A6D0000BF03EFF48460BF03BFF112128460BF0E4
:10A6E00031FC07E71E4A136A43F4000313624FF478
:10A6F000000027F003FB50E7194A136A43F40013E4
:10A7000013624FF4001027F0F9FA46E7144A136A6F
:10A7100043F4800313624FF4800027F0EFFA3CE724
:10A720009BF80E002DF0D8FDBB8823F440731B046A
:10A730001B0C4846BB800BF00BFF48460BF008FF94
:10A74000D8E600BF0054004000580040005C0040C4
:10A75000009F2400804F120083DE1B43D34D621004
:10A7600000380240503A0020F0B5C60033189B0074
:10A77000254DEA585468A28A83B092B20192019A98
:10A780002B4412F4706F1CBF01221A75019B13F445
:10A79000E06F07460CD1A38A3E4423F4706305EBB7
:10A7A00086051B041B0C0022A3826A7503B0F0BD52
:10A7B000238BA38823F480631B041B0CA380019BC1
:10A7C0009B05E8D423889805E5D42388D9050ED5C0
:10A7D0002388DA05FCD423889BB243F400732380DA
:10A7E00023889B05FCD43846FFF736FED3E7238841
:10A7F0009BB243F400732380A38823F440731B04AB
:10A800001B0CA380C7E700BF503A0020F0B583B00F
:10A81000441C8DF8073001D0032802DD002003B06E
:10A82000F0BDC700244E3B1806EB83035D68002D86
:10A83000F4D04900C9B2997501240021DA755C761B
:10A8400099761C765C751975A9880DF10702890542
:10A85000DA611A6214D42B88DA050CD44FF48054D0
:10A8600001E0013C1ED02B889B05FAD42B889BB2BB
:10A8700043F480732B80AB889BB243F44073AB806E
:10A88000074406EB87024FF4805401E0013C09D0F5
:10A89000537D002BFAD106EB87073C7D84F0010045
:10A8A00003B0F0BD054A138801339BB21380FFF754
:10A8B000D3FD2046B3E700BF503A0020703B002094
:10A8C0002DE9F04F85B090F855300190002B40F005
:10A8D000E486019A137C012B00F03887022B12D1F9
:10A8E000936913B11A689B885383019C6B2160693B
:10A8F000FEF7A0FA80216069FEF79CFAA36913B104
:10A900001A689B881383A74CA74DDFF8A492A74829
:10A91000DFF8A0E24FF0640A4FF0100C4FF47A76A3
:10A92000D9F80430C3F30803002B40F02686EFF378
:10A930001183002B40F021862168826800BF2368C4
:10A940009942F9D12F6806FB07F39B1AB3FBF7F383
:10A9500006FB013101270091D9F80430C3F3080345
:10A96000002B40F05984EFF31183002B40F0548406
:10A970002368816800BF22689342F9D1D5F800B0FE
:10A9800006FB0BF2521AB2FBFBF206FB0323009A02
:10A990009B1AB3F57A7FDFD3BAF1010AC0D1019ACD
:10A9A000137C012B00F0DC86022B12D1936913B1CA
:10A9B0001A689B885383019E68217069FEF73AFAF2
:10A9C00007217069FEF736FAB36913B11A689B88DC
:10A9D0001383DFF8DC91754EDFF8D8C14FF0640ABD
:10A9E0004FF010084FF47A77D9F80430C3F3080316
:10A9F000002B40F0DF85EFF31183002B40F0DA8568
:10AA00002168B26800BF23689942F9D1286807FB22
:10AA100000F39B1AB3FBF0F307FB01310120009117
:10AA2000D9F80430C3F30803002B40F01384EFF38C
:10AA30001183002B40F00E842368B16800BF2268A8
:10AA40009342F9D1D5F800B007FB0BF2521AB2FBD2
:10AA5000FBF207FB0323009A9B1AB3F57A7FDFD33F
:10AA6000BAF1010AC0D1019A137C012B00F0AF8624
:10AA7000022B12D1936913B11A689B885383019EEC
:10AA80006B217069FEF7D6F900217069FEF7D2F9E3
:10AA9000B36913B11A689B881383DFF81491434894
:10AAA000DFF810E14FF0640A4FF0100C4FF47A76A3
:10AAB000D9F80430C3F30803002B40F02485EFF3EA
:10AAC0001183002B40F01F852168826800BF236836
:10AAD0009942F9D12F6806FB07F39B1AB3FBF7F3F2
:10AAE00006FB013101270091D9F80430C3F30803B4
:10AAF000002B40F0CD83EFF31183002B40F0C8838F
:10AB00002368816800BF22689342F9D1D5F800B06C
:10AB100006FB0BF2521AB2FBFBF206FB0323009A70
:10AB20009B1AB3F57A7FDFD3BAF1010AC0D1019A3B
:10AB3000137C012B00F04286022B4DD1936913B197
:10AB40001A689B885383019B586940F2E93302E0FD
:10AB5000002B00F06C860289013B12F0020F9BB2C1
:10AB6000F6D06B23838140F2E93302E0002B00F042
:10AB70005E860289013B12F0010F9BB2F6D08389F9
:10AB800040F2E93302E0002B00F04D860289013BE0
:10AB900012F0020F9BB2F6D00123838140F2E93319
:10ABA0000DE000BF60BA002064BA002010E000E0B1
:10ABB00000ED00E05CBA0020002B00F03486028932
:10ABC000013B12F0010F9BB2F6D08389019B9B6978
:10ABD00013B11A689B881383DFF8B892AC48DFF88A
:10ABE000B8E24FF00F0A4FF0100C4FF47A76D9F814
:10ABF0000430C3F30803002B40F0A284EFF3118369
:10AC0000002B40F09D842168826800BF2368994230
:10AC1000F9D12F6806FB07F39B1AB3FBF7F306FB8A
:10AC2000013101270091D9F80430C3F30803002B48
:10AC300040F04B83EFF31183002B40F046832368F1
:10AC4000816800BF22689342F9D1D5F800B006FBB5
:10AC50000BF2521AB2FBFBF206FB0323009A9B1A7B
:10AC6000B3F57A7FDFD3BAF1010AC0D1019991F827
:10AC70004F200B7C042A34BF18261A26012B00F023
:10AC8000BA85022B12D18A6912B1136892885A834D
:10AC9000019F1B217869FEF7CDF831467869FEF7F0
:10ACA000C9F8BB6913B11A689B881383DFF8E49174
:10ACB0007748DFF8E4E14FF00F0A4FF0100C4FF443
:10ACC0007A76D9F80430C3F30803002B40F0E3830D
:10ACD000EFF31183002B40F0DE832168826800BF10
:10ACE00023689942F9D12F6806FB07F39B1AB3FB3F
:10ACF000F7F306FB013101270091D9F80430C3F3C3
:10AD00000803002B40F0FE82EFF31183002B40F08C
:10AD1000F9822368816800BF22689342F9D1D5F88F
:10AD200000B006FB0BF2521AB2FBFBF206FB032348
:10AD3000009A9B1AB3F57A7FDFD3BAF1010AC0D12A
:10AD4000019A137C012B00F04C85022B42D19369B0
:10AD500013B11A689B885383019B586940F2E93309
:10AD600002E0002B00F06D850289013B12F0020F1A
:10AD70009BB2F6D01C23838140F2E93302E0002B22
:10AD800000F05F850289013B12F0010F9BB2F6D003
:10AD9000838940F2E93302E0002B00F04E850289FE
:10ADA000013B12F0020F9BB2F6D01823838140F2D0
:10ADB000E93302E0002B00F040850289013B12F0EC
:10ADC000010F9BB2F6D08389019B9B6913B11A686E
:10ADD0009B881383DFF8BC902D48DFF8BCE04FF070
:10ADE0000F0A4FF0100C4FF47A76D9F80430C3F301
:10ADF0000803002B40F06B83EFF31183002B40F02E
:10AE000066832168826800BF23689942F9D12F6860
:10AE100006FB07F39B1AB3FBF7F306FB013101278F
:10AE20000091D9F80430C3F30803002B40F0878267
:10AE3000EFF31183002B40F082822368816800BF0A
:10AE400022689342F9D1D5F800B006FB0BF2521AF2
:10AE5000B2FBFBF206FB0323009A9B1AB3F57A7F41
:10AE6000DFD3BAF1010AC0D101990B7C91F84E6091
:10AE7000012B00F08884022B49D18B6913B11A6829
:10AE80009B885383019B40F2E932586909E000BF77
:10AE900010E000E000ED00E05CBA0020002A00F0C5
:10AEA000DA840389013A13F0020F92B2F6D01A2322
:10AEB000838140F2E93202E0002A00F0CC84038969
:10AEC000013A13F0010F92B2F6D0838940F2E932D1
:10AED00002E0002A00F0BB840389013A13F0020F5C
:10AEE00092B2F6D0B6B2868140F2E93302E0002B8E
:10AEF00000F0AD840289013B12F0010F9BB2F6D045
:10AF00008389019B9B6913B11A689B881383DFF8BF
:10AF1000CC92B048DFF8C0E24FF00F0A4FF0100CAF
:10AF20004FF47A76D9F80430C3F30803002B40F0CD
:10AF30009682EFF31183002B40F0918221688268A2
:10AF400000BF23689942F9D12F6806FB07F39B1ACB
:10AF5000B3FBF7F306FB013101270091D9F8043068
:10AF6000C3F30803002B40F00782EFF31183002B9B
:10AF700040F002822368816800BF22689342F9D1C1
:10AF8000D5F800B006FB0BF2521AB2FBFBF206FB3F
:10AF90000323009A9B1AB3F57A7FDFD3BAF1010A33
:10AFA000C0D101990B7C91F85060012B00F0E28335
:10AFB000022B12D18A6912B1136892885A83019FB9
:10AFC00019217869FDF736FF31467869FDF732FFC0
:10AFD000BB6913B11A689B881383DFF800927D4820
:10AFE000DFF8F4E14FF0640A4FF0100C4FF47A767A
:10AFF000D9F80430C3F30803002B40F0F882EFF3D4
:10B000001183002B40F0F3822168826800BF23681F
:10B010009942F9D12F6806FB07F39B1AB3FBF7F3AC
:10B0200006FB013101270091D9F80430C3F308036E
:10B03000002B40F0BE81EFF31183002B40F0B9816B
:10B040002368816800BF22689342F9D1D5F800B027
:10B0500006FB0BF2521AB2FBFBF206FB0323009A2B
:10B060009B1AB3F57A7FDFD3BAF1010AC0D1019AF6
:10B07000137C012B00F09983022B12D1936913B139
:10B080001A689B885383019E37217069FDF7D2FEB1
:10B0900010217069FDF7CEFEB36913B11A689B8861
:10B0A0001383DFF838914B48DFF82CE14FF00F0A9B
:10B0B0004FF0100C4FF47A76D9F80430C3F308033C
:10B0C000002B40F0B082EFF31183002B40F0AB82F5
:10B0D0002168826800BF23689942F9D12F6806FB76
:10B0E00007F39B1AB3FBF7F306FB0131012700912D
:10B0F000D9F80430C3F30803002B40F07781EFF355
:10B100001183002B40F072812368816800BF2268A0
:10B110009342F9D1D5F800B006FB0BF2521AB2FBFC
:10B12000FBF206FB0323009A9B1AB3F57A7FDFD369
:10B13000BAF1010AC0D1019A137C012B00F02D83D2
:10B14000022B12D1936913B11A689B885383019E15
:10B1500038217069FDF76EFE01217069FDF76AFE06
:10B16000B36913B11A689B881383DFF8708019499B
:10B17000194F4FF00F094FF0100E4FF47A70D8F8B6
:10B180000430C3F30803002B40F06982EFF311830E
:10B19000002B40F0648222688E6800BF23689A42C8
:10B1A000F9D1D5F800C000FB0CF39B1BB3FBFCF3FB
:10B1B00000FB023300930126D8F80430C3F30803E0
:10B1C000002B40F03081EFF31183002B40F02B81F6
:10B1D00006E000BF10E000E05CBA002000ED00E0F7
:10B1E0002368D1F808A000BF22689342F8D1D5F8AF
:10B1F00000B000FB0BFCACEB0A0CBCFBFBFC00FB47
:10B2000003C3009A9B1AB3F57A7FD5D3B9F101092C
:10B21000B5D105B0BDE8F08FEFF311888CF312883B
:10B2200081680368DB0344BFCEF80070816823683F
:10B23000DEF800205FFA88F888F31188D5F80080DE
:10B240001A4406FB08F35B1AB3FBF8F306FB023360
:10B25000FFF79DBBEFF3118E88F31288B168336856
:10B26000DB0344BFCCF80000B1682368DCF80020A1
:10B270005FFA8EFE8EF31188D5F800E01A4407FBC2
:10B280000EF35B1AB3FBFEF307FB0233FFF7E3BBDE
:10B29000EFF311888CF3128881680368DB0344BFE5
:10B2A000CEF8007081682368DEF800205FFA88F825
:10B2B00088F31188D5F800801A4406FB08F35B1A5E
:10B2C000B3FBF8F306FB023329E4EFF311888CF3A8
:10B2D000128881680368DB0344BFCEF80070816880
:10B2E0002368DEF800205FFA88F888F31188D5F823
:10B2F00000801A4406FB08F35B1AB3FBF8F306FB65
:10B300000233ABE4EFF311888CF312888168036891
:10B31000DB0344BFCEF8007081682368DEF80020AC
:10B320005FFA88F888F31188D5F800801A4406FB84
:10B3300008F35B1AB3FBF8F306FB0233F8E4EFF310
:10B3400011888CF3128881680368DB0344BFCEF850
:10B35000007081682368DEF800205FFA88F888F3BF
:10B360001188D5F800801A4406FB08F35B1AB3FB7A
:10B37000F8F306FB02336FE5EFF311888CF31288C4
:10B3800081680368DB0344BFCEF8007081682368DE
:10B39000DEF800205FFA88F888F31188D5F800807D
:10B3A0001A4406FB08F35B1AB3FBF8F306FB0233FF
:10B3B000EFE5EFF311888CF3128881680368DB03F3
:10B3C00044BFCEF8007081682368DEF800205FFA81
:10B3D00088F888F31188D5F800801A4406FB08F332
:10B3E0005B1AB3FBF8F306FB023338E6EFF3118880
:10B3F0008CF3128881680368DB0344BFCEF80070C9
:10B4000081682368DEF800205FFA88F888F31188E5
:10B41000D5F800801A4406FB08F35B1AB3FBF8F377
:10B4200006FB02337FE6EFF3118A8EF312888A68F7
:10B430000B68DB0344BF3E608A682368D7F800C00E
:10B440005FFA8AFA8AF31188D5F800A09C4400FBC1
:10B450000AF39B1AB3FBFAF300FB0C33D1E6EFF3CC
:10B4600011828CF3128887680368D90303D50123FE
:10B47000CEF8003087682368DEF80010D2B282F37D
:10B4800011882A68194406FB02F3DB1BB3FBF2F3B5
:10B4900006FB013160E5EFF311828CF312888768B7
:10B4A0000368D90303D50123CEF8003087682368E9
:10B4B000DEF80010D2B282F311882A68194406FB24
:10B4C00002F3DB1BB3FBF2F306FB013113E4EFF3F2
:10B4D00011828CF3128887680368D90303D501238E
:10B4E000CEF8003087682368DEF80010D2B282F30D
:10B4F00011882A68194406FB02F3DB1BB3FBF2F345
:10B5000006FB01318BE4EFF311828CF3128887681C
:10B510000368D90303D50123CEF800308768236878
:10B52000DEF80010D2B282F311882A68194406FBB3
:10B5300002F3DB1BB3FBF2F306FB0131FFF7D2BAD8
:10B54000EFF311828CF3128887680368D90303D55F
:10B550000123CEF8003087682368DEF80010D2B2ED
:10B5600082F311882A68194406FB02F3DB1BB3FB44
:10B57000F2F306FB0131FFF754BBEFF311828CF3BA
:10B58000128887680368D90303D50123CEF80030F9
:10B5900087682368DEF80010D2B282F311882A6827
:10B5A000194406FB02F3DB1BB3FBF2F306FB01318C
:10B5B000FFF7D0B9EFF3118288F31288B0683368CF
:10B5C000D90303D50123CCF80030B0682368DCF838
:10B5D0000010D2B282F311882A68194407FB02F3E3
:10B5E0001B1AB3FBF2F307FB0131FFF717BAEFF3B6
:10B5F00011828CF3128887680368D90303D501236D
:10B60000CEF8003087682368DEF80010D2B282F3EB
:10B6100011882A68194406FB02F3DB1BB3FBF2F323
:10B6200006FB0131FEE4EFF311828CF31288876888
:10B630000368D90303D50123CEF800308768236857
:10B64000DEF80010D2B282F311882A68194406FB92
:10B6500002F3DB1BB3FBF2F306FB013146E5EFF32C
:10B6600011868EF31288D1F808C00B68DA0303D56F
:10B6700001233B60D1F808C023683A68F6B286F32C
:10B6800011882E681A4400FB06F3A3EB0C03B3FBEE
:10B69000F6F300FB023300938DE51D09013D032DF8
:10B6A00003F00F0300F2B680734A32F8150040FA37
:10B6B00003F2D40740F1AE80012404FA03F3013B06
:10B6C000184037F0E3FE6D4B6D4A5B5D184412EB9A
:10B6D000C00500F09F8000232021EB71A97152F872
:10B6E0003000684A00F13F4303F57E039B0AD25CB9
:10B6F00002F01F035209032A04FA03F300F0B68094
:10B70000042A00F0AE80022A7FD0AB88029302A9FF
:10B710000023039326F03CFD01995B4B41F80C3F5D
:10B7200028462DF0B7FAAB88B3FA83F3C3F11F03B1
:10B73000012212FA03F33FF4CCA854490A681343D8
:10B74000019A0B60137C012B7FF4C8A8104680235C
:10B75000417D90F914006B22FFF758F8FFF7D3B83A
:10B7600010460723417D90F914006822FFF74EF838
:10B77000FFF72FB9084633461922497D90F9140086
:10B78000FFF744F829E4084633461A22497D90F928
:10B790001400FFF73BF8FFF7BABB10463822417D93
:10B7A00090F91400FFF732F8DFE410461023417DD2
:10B7B00090F914003722FFF729F872E410466B2243
:10B7C000417D90F91400FFF721F8FFF705BA104604
:10B7D0005346417D90F914006B22FFF717F8FFF7ED
:10B7E0005CB910461823417D90F914001C22FFF724
:10B7F0000DF8FFF7EFBA084633461B22497D90F952
:10B800001400FFF703F8FFF751BA214A516C0B43BC
:10B8100053647AE701991C4B41F80C3F00202DF04E
:10B8200039FAFFF756B80AF0DFFFFFF7CFB90AF091
:10B83000DBFF019B5869FFF7A3B90AF0D5FFFFF7BB
:10B84000C3BA0AF0D1FF019B5869FFF7A2BA0AF008
:10B85000CBFFFFF756BB0AF0C7FF019B5869FFF704
:10B8600035BB0B4A116B0B4313634EE7084A116C4F
:10B870000B43136449E700BF8C76040888760408FC
:10B88000A0B8002000750408A5840008003C014011
:10B89000003802402DE9F04F8A4A436983B0934251
:10B8A000019000F00D8188498B420CBF2821302186
:10B8B0001A8822F040021204120C1A801A8892B2DE
:10B8C00022F03802114319801A8892B242F04002E5
:10B8D0001A80012001F0E8FE019C2046FEF7F0FFEF
:10B8E000A36913B11A689B885383019B586940F27E
:10B8F000E93302E0002B00F0DB800289013B12F00B
:10B90000020F9BB2F6D06A23838140F2E93302E052
:10B91000002B00F0CD800289013B12F0010F9BB299
:10B92000F6D0838940F2E93302E0002B00F0C580B5
:10B930000289013B12F0020F9BB2F6D010238381E3
:10B9400040F2E93302E0002B00F0B7800289013BAE
:10B9500012F0010F9BB2F6D08389019B9B6913B152
:10B960001A689B881383594CDFF86CE1DFF86C91FF
:10B970005748584F4FF0640A4FF0100C4FF47A7547
:10B98000D9F80430C3F30803002B76D1EFF3118309
:10B99000002B72D12168826800BF23689942F9D1D7
:10B9A000DEF8006005FB06F39B1AB3FBF6F305FB1C
:10B9B000013101260091D9F80430C3F30803002BAC
:10B9C00040D1EFF31183002B3CD12368816800BF85
:10B9D00022689342F9D1DEF800B005FB0BF2521A4F
:10B9E000B2FBFBF205FB0323009A9B1AB3F57A7FA7
:10B9F000E1D3BAF1010AC3D1019B324A5B69934298
:10BA000007D0DFF8C4A0534514BF4FF0080A4FF029
:10BA1000000A1A8822F040021204120C1A801A88B6
:10BA200092B222F038024AEA020AA3F800A01A8869
:10BA300092B242F0400201201A8003B0BDE8F04FFC
:10BA400001F032BEEFF311888CF31288816803682D
:10BA5000DB0344BF3E60816823683A685FFA88F878
:10BA600088F31188DEF800801A4405FB08F35B1A9E
:10BA7000B3FBF8F305FB0233B6E7EFF311828CF367
:10BA8000128886680368D90302D501233B60866863
:10BA900023683968D2B282F31188DEF80020194495
:10BAA00005FB02F39B1BB3FBF2F305FB013180E7BF
:10BAB0000AF09AFE019B586934E70AF095FE4CE7BC
:10BAC0002821F5E600380040003C004060BA002024
:10BAD00010E000E05CBA002064BA002000ED00E055
:10BAE0000220FCF7C5BD0220FEF73EBE0120FCF798
:10BAF000BFBD0120FEF738BE0020FCF7B9BD002015
:10BB0000FEF732BE1549164B16480A6810B48C6809
:10BB10001549B2FBF4F203FB02F30360D1F888206D
:10BB2000124B134C42F47002C1F888201A680020AE
:10BB300042F001021A6098601A6822F0847222F4BE
:10BB400080321A605C601A684FF0006422F4802230
:10BB50001A60D8608C605DF8044B704700000020CC
:10BB600040420F00B0A4002000ED00E00038024089
:10BB700010300024044B4FF4F0700A21022283E8B5
:10BB80000700FFF7BFBF00BF0000002038B50B4C17
:10BB900023688BB15A68821A002A054604DA0CE041
:10BBA0005A68AA1A002A07DB9A68226018461A689F
:10BBB00090472368002BF3D138BD38BD78C10020F1
:10BBC0000B4B002210B4027203F59074032102E0C3
:10BBD000072A09DC9979890702D51979815401323C
:10BBE0009C4203F11803F3D15DF8044B704700BF8A
:10BBF000507504082E230370704700BF012310B452
:10BC000031213224102244704171C27003720370DA
:10BC1000037183705DF8044B704700BF2DE9F0415C
:10BC20000B78047BDB43DEB200F1100200F1380335
:10BC300042F8044F9342FBD1DFF89CC000F1600151
:10BC4000002243F8042F8B42FBD14FF0140E052144
:10BC5000002546FA01F303F00103002B1D4414BF35
:10BC60004FF019084FF00A0811F0010FEDB214BFA0
:10BC70002746002700220EEB02039BB200EB830352
:10BC8000013242455F61F6D1013A92B20132013987
:10BC90000EEB02034A1C9BB201D09E46D9E715F079
:10BCA000010F14BF19250A2500215A1892B200EB82
:10BCB00082020131A9425461F7D10B449BB21A1D93
:10BCC00000EB8202013300219BB25160ACF80030DE
:10BCD0000361BDE8F08100BF781F0020254B5B8821
:10BCE0000B332DE9F04F8A4601F1060B1FFA83F959
:10BCF0004FF00108002100271AF801EB3E464C46A0
:10BD00000122A4F10B039BB207E001339BB2B0F810
:10BD10000CC0C5F814C09C420AD000EB8305002A71
:10BD2000F3D100EB830501339BB29C426A61F4D1ED
:10BD3000231D00EB83030136092FF6B259600CD0A6
:10BD4000092E14D008FA07F313EA0E0F14BF0122CC
:10BD500000220C34A4B20137D3E709F17809DA459F
:10BD60001FFA89F9C7D1034B5980BDE8F08F002233
:10BD7000EFE700BF781F00202DE9F047DFF85C8077
:10BD8000B8F8043004338A461FFA83FC01F109092C
:10BD90004FF0010E1AF8017B64460026231F0EFAAD
:10BDA00006F29BB23A40BAB1818900EB83050133B8
:10BDB0009BB29C426961F6D101360434082EA4B2CC
:10BDC000ECD10CF1200CCA451FFA8CFCE2D1002307
:10BDD000A8F80430BDE8F0871146E6E7781F002098
:10BDE00010B5027B01681F2A4FF020030ED94C6862
:10BDF000203A93401C4216D00B4A4068002414702D
:10BE0000026822F001020260CB6010BD0C68934012
:10BE10001C4208D0044A406800241470026822F0D2
:10BE2000010202608B6010BDF1270020436A826925
:10BE3000D154436A0169826B01338B4228BF0023CE
:10BE40004362002A2FD0EFF31182502383F312882C
:10BE5000836B1968C9072CD470B45E686EB9456AE3
:10BE6000816A8D4217D084690C44DC600ED9691A4E
:10BE700059608562002180F85C10196841F0010169
:10BE8000D2B2196082F3118870BC70470469611ADC
:10BE900059608662EEE7012380F85C30D2B282F30B
:10BEA000118870BC7047826DD36843F08003D36003
:10BEB0007047D2B282F31188704700BF426B10B452
:10BEC00062B1C36CC2684469D11A013B615C5DF820
:10BED000044B08BF1346C364C8B27047016A436984
:10BEE000C4685B5C0131A14228BF114601625DF864
:10BEF000044BD8B2704700BF836B13B190F85C005D
:10BF00007047836A406A181AB0FA80F04009704797
:10BF1000416A836A99420AD3CB1A816B026961B183
:10BF20004968501E0B4483420AD2C01A7047026906
:10BF30001144CB1A816B0029F2D1501EC01A7047F0
:10BF400000207047436B43B1C26C5B6893422FBFC4
:10BF5000981AC0689B1AC0187047C269036A9A424F
:10BF60002FBFD01AC0688018C01A70470A4B30B56E
:10BF700003F1180493F900205D78072AC8BF143A2A
:10BF8000811804330D7313F8025C855413F8012CE7
:10BF90000A76A342EED130BD784C0408038A2DE91D
:10BFA000F0478589ADB21D4029D00F4606464FF0B7
:10BFB00000484FF00009B5FA85F328FA03F2D2439E
:10BFC00091B21B3B15403182042B16D8DFE803F0F9
:10BFD0003129211903007B6A002B32D003F1FF3A8B
:10BFE0001FFA8AFAC7F824903C6A34B123682046C5
:10BFF000514698476468002CF8D1002DDBD1BDE88C
:10C00000F0873868716B036889B29847002DD2D1E8
:10C01000F5E77868B16B036889B29847002DCAD1FB
:10C02000EDE7B868F16B036889B29847002DC2D17B
:10C03000E5E7F868316C036889B29847002DBAD1FA
:10C04000DDE7F36A1FFA83FACEE700BF30B5044696
:10C05000806D61718389A26823F400531B041B0C5B
:10C06000838185B0A379009213F0040230D04FF49D
:10C07000805213F00203ADF804205CD1ADF8063015
:10C080004FF480630022ADF8083011F00103ADF8E1
:10C090000C2028D1ADF80A3008238D07694648BF27
:10C0A000ADF80A3025F07AFEA279A36DD10724D429
:10C0B00012F0080F9A8A1BD122F008021204120C07
:10C0C0009A829A8992B242F400529A8105B030BDA8
:10C0D00013F00203ADF804202AD04FF400551346A4
:10C0E000ADF80650CEE70423ADF80A300C23D4E7B0
:10C0F00092B242F008029A82E3E710498B4215D0CF
:10C10000A1F548418B420FD001F580618B4209D0E7
:10C110000B498B42CCD105200121FDF7ABFDA27963
:10C12000A36DC5E70320F7E70220F5E70020F3E75A
:10C13000ADF80630A6E74FF400539FE7001001402A
:10C140000014014010B50446806DA160838923F47A
:10C1500000531B041B0C8381A37984B013F00402E9
:10C16000009135D04FF4805213F00203ADF8042053
:10C170005CD1ADF806304FF480636279ADF80830D9
:10C18000D1074FF00003ADF80A30ADF80C3045BFD1
:10C190000423ADF80A3008230C236946920748BFF0
:10C1A000ADF80A3025F0FAFDA279A36DD1071FD4AE
:10C1B00012F0080F9A8A16D122F008021204120C0B
:10C1C0009A829A8992B242F400529A8104B010BDC8
:10C1D00013F00203ADF8042025D04FF400511346AC
:10C1E000ADF80610C9E792B242F008029A82E8E779
:10C1F00010498B4215D0A1F548418B420FD001F573
:10C2000080618B4209D00C498B42D1D1052001219C
:10C21000FDF730FDA279A36DCAE70320F7E70220FE
:10C22000F5E70020F3E7ADF80630A6E74FF400533A
:10C230009FE700BF00100140001401401C4C08B5EE
:10C24000012102200AF092F9237803F00502052A61
:10C2500029D003F00903092B08D0002101200AF09E
:10C2600085F9002108460AF081F9FEE7114A124BD0
:10C2700011681A680B68114C23F001030B601388D6
:10C28000206823F001031B041B0C138018B12A2221
:10C2900000238271C37109224A2109F0CFFF20686F
:10C2A0000AF050F9D9E72BF041F92378D1E700BF24
:10C2B0001C3A0020FC27002000280020143B00200E
:10C2C000022828BF022010B4084C094B207000EB54
:10C2D0008002C0EBC20207495DF8044B013003EB5A
:10C2E0004203C0B20B6032F099BC00BFD0C6002040
:10C2F00074AF0020BC46002008B531F0D3FA0AF034
:10C30000C7FCBDE8084031F0B5BA00BF2DE9804850
:10C31000013085B0C3B203938B4D8C4F8C4C8D4E46
:10C320000A2302933220DFF830922CF0F5F94FF413
:10C33000FA7A4FF0100C4FF47A70D9F80430C3F346
:10C340000803002B40F0C180EFF31183002B40F075
:10C35000BC802968A26800BF2B689942F9D1D7F840
:10C3600000E000FB0EF39B1AB3FBFEF300FB013170
:10C370004FF0010E0191D9F80430C3F30803002BEC
:10C3800040F08780EFF31183002B40F082802B6810
:10C39000A16800BF2A689342F9D1D7F800B000FB2A
:10C3A0000BF2521AB2FBFBF200FB0323019A9B1A19
:10C3B000B3F57A7FDFD3BAF1010ABED1039B002B1C
:10C3C00040F0BD804FF47A7ADFF88C9150464FF000
:10C3D000100CD9F80430C3F30803002B40F092800E
:10C3E000EFF31183002B40F08D802968A26800BF15
:10C3F0002B689942F9D1D7F800E000FB0EF39B1AA5
:10C40000B3FBFEF300FB01314FF0010E0191D9F8AF
:10C410000430C3F3080303BBEFF31183EBB92B68BC
:10C42000A16800BF2A689342F9D1D7F800B000FB99
:10C430000BF2521AB2FBFBF200FB0323019A9B1A88
:10C44000B3F57A7FE3D3BAF1010AC2D1029B013B73
:10C4500002937FF467AFFCF751FEEFF311888CF382
:10C460001288A1682368DB0344BFC6F800E0A16816
:10C470002B6832685FFA88F888F31188D7F8008053
:10C480001A4400FB08F35B1AB3FBF8F300FB02331A
:10C49000D4E7EFF311888CF31288A1682368DB03DB
:10C4A00044BFC6F800E0A1682B6832685FFA88F8DC
:10C4B00088F31188D7F800801A4400FB08F35B1A50
:10C4C000B3FBF8F300FB023370E7EFF311828CF358
:10C4D0001288D4F808E02368D90303D50123336018
:10C4E000D4F808E02B683168D2B282F311883A6838
:10C4F000194400FB02F3A3EB0E03B3FBF2F300FBC2
:10C50000013135E7EFF311828CF31288D4F808E09B
:10C510002368D90303D501233360D4F808E02B68DE
:10C520003168D2B282F311883A68194400FB02F3F1
:10C53000A3EB0E03B3FBF2F300FB013164E71846F3
:10C540002BF04CFF3EE700BF60BA002064BA002029
:10C5500010E000E05CBA002000ED00E038B5484B88
:10C560005A899989914224BF00225A81198ADA890D
:10C57000914224BF0022DA81DA78CAB1072A414900
:10C580006AD091F85300404D012400210A282C70F4
:10C590009C70D9715DD00C2807D0002A6CD0DFEDDB
:10C5A0003B7A072A0ED00A2862D0DFED397A09E0FB
:10C5B000344A92F853000A2856D00C285BD1D97916
:10C5C000DFED347A344C9FED350AA278002918BF8C
:10C5D000F0EE407A062A04D8314901EB820191ED50
:10C5E000060A217979B1013A032A0BD8F7EE007ACD
:10C5F00087EE800A37F0FCFA2388984228BF184655
:10C60000208038BD38BD9B781F4A07EE103A11785C
:10C61000B8EEC77A67EE277A07EE101AB8EEC77A37
:10C6200027EE277AB4EEC70AF1EE10FAEADD80EEC3
:10C63000277AFDEEC77A17EE903A102BA8BF102389
:10C64000012BB8BF0123DBB28B4238BF0B461370FE
:10C6500038BDDFED147AA4E791F853000A2803D01F
:10C660000C28ACD0D9799AE7D979DFED0E7AA9E711
:10C67000DFED0D7AA6E7D979DFED047AA2E700BFF6
:10C6800090AC0020B4A40020205800206F12033981
:10C690006F12833A0AD7A3398C5D00206F120338DA
:10C6A000784C04085304E9380F506E3A2DE9F047EE
:10C6B000AA4FAB4E31F0F6F8BE421ED2DFF824830B
:10C6C000DFF824934446258862197DB14A450DD28E
:10C6D000052D0BD933886188C3F30B03994200F011
:10C6E000E080144625886219002DEFD1716830462C
:10C6F00014360AF059FABE42E4D39A4A1378A3F1E9
:10C70000170102290FD9984911F83300002840F089
:10C71000F780D8000144497829B1944911F83330A1
:10C720000BB918231370924B5A78022A00F2D98061
:10C730009049914802EB420201EB82011A780160B4
:10C74000022A00F2D78002EB82018C4BC2EBC102BD
:10C7500003EB4203998C5A8C894C9142236001D39C
:10C7600000225A84874B9A78042A00F0EA8032B972
:10C770001A88B2F5F07F84BF4FF4F0721A80824DB0
:10C78000FFF7ECFE2B68814A1A40002A00F0E28095
:10C79000D80700F1D180590400F1C9801A0700F1CF
:10C7A000B8809B0400F1BC8026F0C8F910B9784825
:10C7B00031F0CAFB4FF400700AF02CFA4FF48020DD
:10C7C0000AF028FA4FF000700AF024FA4FF0806067
:10C7D0000AF020FA2BF090FB002130226D4838F04F
:10C7E000C4F920682AF0D8FA6B4B256803F1500190
:10C7F00003E00433994200F081801A78002AF8D1CE
:10C800009C78D8788442F4D26449654B0A702846F3
:10C810001D602EF039FF634A63491079634A644B07
:10C820001160C822642111FB0021002259609A6026
:10C83000DA601A615A619A61DA6183F8202083F81C
:10C84000212021F007FA5B4B9FED5B5A1B885B4A66
:10C850009FED5B6A55795B4C5B495C48086006EE6E
:10C86000903AF8EEE66A1388C5EE265A07EE103ABB
:10C8700053881279C4ED005A07EE903AB8EEC77AA1
:10C88000534BF8EEE77A1D725A7227EE067A67EE7E
:10C89000867ABDE8F04783ED017AC3ED007A30F087
:10C8A000E9BF63799B077FF41CAF716894F804A01B
:10C8B00030460AF079F93388BAEB133F04D01436C6
:10C8C000BE42FFF4FFAE18E773887068AA1FC3F377
:10C8D0000B039A4204F10601A8BF1A4637F048F844
:10C8E000EDE700225A701A78234822490160022A93
:10C8F0007FF629AF00221A70204B2BE7012283E735
:10C90000D8000C186468002C7FF404AF172414704E
:10C9100000E730480AF07EF92B689B047FF544AFAE
:10C920002D480AF077F940200AF074F93CE72B48CB
:10C930000AF070F92B6831E729480AF06BF92B6887
:10C9400029E79A8AB2F57A7FBFF419AF4FF47A7269
:10C950009A8214E743F008032B6019E740060008A9
:10C9600090010008405C0020D06D04089C7D040804
:10C97000D0C60020DCC60020C046002074AF0020D6
:10C98000BC4600208C5D002018B100200960000228
:10C990003C980020B421002034C90020781D0020DC
:10C9A000E821002070B8002032580020EC20002040
:10C9B0001C400020C8260020C0C9FB48C424002019
:10C9C00017B7D138CC260020DCB200203661023DFA
:10C9D000B8B20020016000020940000209200002F4
:10C9E00008600002024000080080000808B530F02E
:10C9F00059FF0AF04DF930F03DFFFFF757FE0120D7
:10CA0000BDE8084032F00AB938B50C4C0C4DAC42C8
:10CA100006D26168204614340AF0C6F8AC42F8D356
:10CA2000084A094B094C1460002209491A705A70CF
:10CA300008480860BDE838401AF0AEB89001000818
:10CA400040060008BC460020D0C6002074AF00207D
:10CA5000C0460020DCC6002008B5FFF7D5FF30F047
:10CA600021FF0AF015F9BDE8084030F003BF054B7F
:10CA700010B59A68044C2178501C09B99A6010BD11
:10CA80000246F8E7781F0020F1270020F0B50C29B6
:10CA900034D8DFE801F0893333335E333333343352
:10CAA00033330700048C9689B2F802E01788734D7F
:10CAB00024F480542404240C0484038C8488818B03
:10CAC00023F4005321F4E6411B0409041B0C46EA3D
:10CAD0000E06090C43EA063341EA0721A8429BB23D
:10CAE000A4B289B200F09E8005F58065A84200F0EE
:10CAF000998092688480818302640384F0BD048CF1
:10CB00009589B2F802C0B2F800E05C4F24F480745A
:10CB10002404240C0484038C8688818B23F4007302
:10CB20001B0421F073011B0C45EA0C04090443EAC1
:10CB30000423090CB8429BB2B6B241EA0E015CD0A4
:10CB40004F4CA04259D0926886808183C26303848F
:10CB5000F0BD048C9589B2F802C0B2F800E0474EEF
:10CB600024F010042404240C0484038C8788018B93
:10CB700023F0200321F4E6411B0409041B0C45EAC1
:10CB80000C04090C43EA041341EA0E21B0429BB2A3
:10CB9000BFB289B25DD03A4CA0425AD09268878029
:10CBA000018382630384F0BD048C9789B2F802E0AC
:10CBB0001688324D24F001042404240C0484038CD0
:10CBC0008488018B23F002031B0421F073011B0CEA
:10CBD00047EA0E0709043B43090CA8429BB2A4B2E2
:10CBE00041EA060125D005F58065A84221D092686A
:10CBF0008480018342630384F0BDD589148A578AF7
:10CC000023F4006343EA05254FF6FF332B40958854
:10CC100026F440563C4343EA052346EA04169BB2F9
:10CC2000B6B290E7158A24F4804444EA8514A4B28D
:10CC30005FE7D689158A578A23F00803334324F423
:10CC4000407496883D4323F004032C433343A4B23D
:10CC5000CDE7D489158A568A23F0800343EA04136A
:10CC60004FF6BF741C40938827F44067354344EA6D
:10CC7000031347EA85079BB2BFB28FE7000001406C
:10CC8000000401402DE9F84FF02200219148924C18
:10CC9000DFF86892914D924E924FDFF8648237F040
:10CCA00064FF91489149DFF85CE2DFF85CC2002242
:10CCB0001359834200F0E980B3F1804F00F0E78020
:10CCC000AB4200F0F280B34200F0F180BB4200F0D2
:10CCD000F080734500F0EF80634500F0EE8043453F
:10CCE00000F0ED80DFF824A2534500F0EA800AF559
:10CCF000806A534500F0E7800AF5806A534500F0EA
:10CD0000E480AAF5983A534500F0E1800AF5806A7C
:10CD1000534500F097800AF5806A534508BF0D23FC
:10CD200000F091801832B2F59C7FC1D16A4EDFF8D5
:10CD3000E0A106F59C774FF003094FF0020803E0ED
:10CD40001836B74200F09F80B379002BF8D03379C2
:10CD50001C09013C032C03F00F03F1D8644A32F89C
:10CD6000140040FA03F2D207EAD5012505FA03F3CD
:10CD7000013B184036F08AFB5E4B1B5D18441AEBF2
:10CD8000C002DDD05AF830305B4C317A03F13F40BD
:10CD900000F57E00800A205C00F01F044009032893
:10CDA00005FA04F57BD0042873D0022804D14F483B
:10CDB000406C05434D484564B2F804E0BEFA8EF27B
:10CDC000C2F11F0292B2D00803EB800002F007020A
:10CDD000046A92000F25954024EA05040462046A5F
:10CDE00001FA02F22243002502624FF0010C2A46AA
:10CDF00003E0102A05F10205A2D00CFA02F030EA95
:10CE00000E0102F10102F4D11C6809FA05F1C943CF
:10CE10000C401C60D3F800B008FA05F444EA0B0497
:10CE20001C609C680C409C609C689C605C6824EA68
:10CE30000000586058685860D8680140D960D968C7
:10CE4000D960D6E70C2309EBC3034FF0010A1B7925
:10CE500003F01F0B5B09032B0AFA0BFA09D0042B12
:10CE60000CD0022B7FF45EAF4B6C4AEA03034B6499
:10CE700058E70B6C4AEA03030B6453E70B6B4AEA6F
:10CE800003030B634EE7BDE8F88F0023DBE70123C4
:10CE9000D9E71648006B0543144805638CE713482F
:10CEA000006C05431148056486E70223CBE70323A2
:10CEB000C9E70423C7E70523C5E70623C3E707231C
:10CEC000C1E70823BFE70923BDE70A23BBE70B231C
:10CED000B9E700BF2C910020507504080004004001
:10CEE00000080040000C00400000014000380240F3
:10CEF0008C7604088876040800750408606D0408C0
:10CF000000040140001000400014004000400140B7
:10CF1000A0B8002001490248FFF740B8F491002072
:10CF20000018004001490248FFF738B8CC910020B2
:10CF30000004014001490248FFF730B8CC910020BD
:10CF40000004014001490248FFF728B8A4910020DD
:10CF5000000C004001490248FFF720B87C910020F6
:10CF60000004004002494FF08040FFF717B800BFAF
:10CF70005491002001490248FFF710B82C9100207D
:10CF80000000014001490248FFF708B82C91002039
:10CF900000000140F0B504684B4DA30AAB4276D0C7
:10CFA00009D94A4DAB425CD00135AB4273D03B3D11
:10CFB000AB425AD0F0BDB3F5801F64D0023DAB4206
:10CFC00057D14FF0700E02264779B0004FEA970C08
:10CFD000002964D063460227A5899F4083190CEB82
:10CFE00043032F4303F1040C394DBFB245F823101E
:10CFF00045F82C20A781EFF31181502282F312888B
:10D00000821905EBC2021369002B33D0136204337B
:10D01000821905EBC202576917B11F6053690433C7
:10D02000821905EBC202976917B11F609369043337
:10D03000821905EBC202D76917B11F60D3690433A7
:10D040000027CAB21F6082F31188304405EBC0008C
:10D05000036A93B9A38923F001031B041B0CA3816A
:10D06000F0BD4FF0200E0026AEE74FF0E80E05268B
:10D07000AAE7F0BD05EB0E03CAE7A3899BB243F014
:10D080000103A381F0BD4FF0480E01269CE74FF04D
:10D09000980E032698E74FF0C00E042694E702236B
:10D0A000BF0803FA07F7A389094D9BB223EA0703D8
:10D0B00087190CEB470CA3810CF1040345F82C10E5
:10D0C00045F8232097E700BF030010004000100040
:10D0D0002C91002010B5036882480139834282B048
:10D0E00089B200F0CA80A0F58060834200F0C5805C
:10D0F00000F58040834200F0B78000F580608342F5
:10D1000000F0B28000F58060834200F0AD80764C84
:10D11000188824686408B4FBF2F4013CA4B282B21B
:10D12000B3F1804F0AD07148834207D000F5806088
:10D13000834203D000F58060834202D122F0700266
:10D1400092B26B48834200F0A18000F58060834278
:10D1500000F0A68022F4407200F56C4092B2834247
:10D160001A80D9621C854FD05E4A93424CD001226E
:10D170009A821A8892B242F001021A80B3F1804F6B
:10D1800000F09880594A934200F0968002F5806240
:10D19000934200F0938002F58062934200F0908009
:10D1A00002F58062934200F08D8002F58062934226
:10D1B00000F08A8002F57042934200F0878002F509
:10D1C0007052934200F0848002F58062934200F036
:10D1D000818002F5806293427ED0A2F5983293421C
:10D1E0007CD002F5806293427AD002F5806293424D
:10D1F00008BF0D2215D002A84FF0012340F8043DCE
:10D2000024F03CFD02B010BD0122002119869A8253
:10D210001A88384892B242F0010283421A80ADD196
:10D220000A46354B03EBC20301A85C798DF8044034
:10D23000012300228DF805308DF807308DF8062087
:10D2400024F01CFD1B2C08D02E2CDBD12B4B019382
:10D2500001A824F013FD02B010BD294B019301A8D1
:10D2600024F00CFD02B010BD1F4C18882468B4FBDC
:10D27000F2F4013CA4B282B252E71B4C1888246835
:10D28000B4FBF2F4013CA4B282B257E701201A8049
:10D29000D9621C8598821A8892B202431A8071E77B
:10D2A00001201A80D9621C8598821A8892B20243A2
:10D2B0001A8063E70122B4E70222B2E70322B0E753
:10D2C0000422AEE70522ACE70622AAE70722A8E778
:10D2D0000822A6E70922A4E70A22A2E70B22A0E778
:10D2E0000C229EE700040140B0A40020000400408E
:10D2F0000010004000000140606D04082C01000196
:10D30000190100012B4B98423CD0B0F1804F3BD02B
:10D31000A3F57C43984239D003F58063984237D017
:10D3200003F58063984235D003F58063984233D08B
:10D3300003F58063984231D003F5704398422FD0B3
:10D3400003F5705398422DD003F5806398422BD09B
:10D3500003F58063984229D0A3F59833984227D0EB
:10D3600003F58063984207D003F58063984208BFB5
:10D370000D2202D0002070470C220F4B03EBC2039A
:10D38000187970470022F8E70122F6E70222F4E755
:10D390000322F2E70422F0E70522EEE70622ECE79B
:10D3A0000722EAE70822E8E70922E6E70A22E4E79B
:10D3B0000B22E2E700000140606D04082DE9F04F08
:10D3C000013085B0C3B203930B4602918B4C8C4E57
:10D3D000002B00F09A8032208A4D8B4FDFF82C9280
:10D3E0002BF09AF94FF4FA7A4FF0100C4FF47A7050
:10D3F000D9F80430C3F30803002B40F0DE80EFF3CC
:10D400001183002B40F0D9802968A26800BF2B68E7
:10D410009942F9D1D7F800E000FB0EF39B1AB3FB59
:10D42000FEF300FB01314FF0010E0191D9F80430F9
:10D43000C3F30803002B40F08780EFF31183002B28
:10D4400040F082802B68A16800BF2A689342F9D11E
:10D45000D7F800B000FB0BF2521AB2FBFBF200FB54
:10D460000323019A9B1AB3F57A7FDFD3BAF1010A3D
:10D47000BED1039B002B40F0BD804FF47A7ADFF8D9
:10D480008C9150464FF0100CD9F80430C3F30803C8
:10D49000002B75D1EFF31183002B71D12968A2689D
:10D4A00000BF2B689942F9D1D7F800E000FB0EF3DA
:10D4B0009B1AB3FBFEF300FB01314FF0010E01910B
:10D4C000D9F80430C3F3080313BBEFF31183FBB99E
:10D4D0002B68A16800BF2A689342F9D1D7F800B041
:10D4E00000FB0BF2521AB2FBFBF200FB0323019A82
:10D4F0009B1AB3F57A7FE3D3BAF1010AC4D1029B38
:10D50000013B0293002B7FF466AF05B0BDE8F08FBE
:10D51000EFF311888CF31288A1682368DB0344BF02
:10D52000C6F800E0A1682B6832685FFA88F888F3D3
:10D530001188D7F800801A4400FB08F35B1AB3FB8C
:10D54000F8F300FB0233D2E7EFF311888CF3128873
:10D55000A1682368DB0344BFC6F800E0A1682B681C
:10D5600032685FFA88F888F31188D7F800801A4487
:10D5700000FB08F35B1AB3FBF8F300FB023370E720
:10D58000EFF311828CF31288D4F808E02368D903F2
:10D5900003D501233360D4F808E02B683168D2B298
:10D5A00082F311883A68194400FB02F3A3EB0E03DF
:10D5B000B3FBF2F300FB01317FE7EFF311828CF351
:10D5C0001288D4F808E02368D90303D50123336017
:10D5D000D4F808E02B683168D2B282F311883A6837
:10D5E000194400FB02F3A3EB0E03B3FBF2F300FBC1
:10D5F000013118E718462AF0F1FE3EE710E000E09E
:10D600005CBA002060BA002064BA002000ED00E09F
:10D61000204B5B68C3F3080330B4BBB9EFF311834D
:10D62000A3B91D4B1D4C1868A16800BF1A68904231
:10D63000F9D11B4B1C684FF47A7202FB04F3591AA0
:10D64000B1FBF4F130BC02FB00107047EFF3118224
:10D65000102383F3128811498C680B6813F4803F00
:10D66000104B02D0012018608C680B49D2B20D68B3
:10D67000186882F311880A4B19684FF47A722844AB
:10D6800002FB01F31B1B30BCB3FBF1F302FB0030C8
:10D69000704700BF00ED00E060BA002010E000E03D
:10D6A00064BA00205CBA00202DE9F84F8046FFF7ED
:10D6B000AFFF254E2549DFF8A0E0254A254D8446D9
:10D6C00010274FF47A740120DEF80430C3F3080306
:10D6D000D3B9EFF31183BBB90B68D2F808A000BF30
:10D6E000D1F800904B45F7D1D6F800B004FB0BF908
:10D6F000A9EB0A09B9FBFBF904FB0393A3EB0C03A9
:10D700004345E1D3BDE8F88FEFF3118A87F3128820
:10D71000D2F808B01368DB0344BF2860D2F808B021
:10D720000B68D5F800905FFA8AFA8AF31188D6F868
:10D7300000A0994404FB0AF3A3EB0B03B3FBFAF339
:10D7400004FB0933DAE700BF64BA002060BA0020A6
:10D7500010E000E05CBA002000ED00E02DE9F04FA1
:10D76000DFF830C1474A4849484E494D80461027A6
:10D7700018F1FF38C0F08480DCF80430C3F30803EC
:10D78000002B5CD1EFF31183002B58D10B68946808
:10D7900000BF08688342F9D1D6F800904FF47A7040
:10D7A00000FB09FEAEEB040EBEFBF9FE00FB03EE30
:10D7B000DCF80430C3F308034FF47A740120FBB99A
:10D7C000EFF31183E3B90B68D2F808A000BFD1F8DA
:10D7D00000904B45F7D1D6F800B004FB0BF9A9EB4C
:10D7E0000A09B9FBFBF904FB0393A3EB0E03B3F5A2
:10D7F0007A7FBDD2DCF80430C3F30803002BDFD0FE
:10D80000EFF3118A87F31288D2F808B01368DB03AC
:10D8100044BF2860D2F808B00B68D5F800905FFAD2
:10D820008AFA8AF31188D6F800A0994404FB0AF317
:10D83000A3EB0B03B3FBFAF304FB0933D5E7EFF3D8
:10D84000118487F31288D2F808901368D80303D59F
:10D8500001232B60D2F808900B682868E4B284F3A7
:10D860001188D6F800A04FF47A7400EB030E04FB85
:10D870000AF3A3EB0903B3FBFAF304FB0E3E97E7AD
:10D88000BDE8F08F10E000E060BA002064BA00202C
:10D890005CBA002000ED00E030B4EFF311831022F9
:10D8A00082F312880649074C0A68074801320025AE
:10D8B0000A602560DBB2026883F3118830BC7047D0
:10D8C00060BA00205CBA002010E000E00F4B1B881B
:10D8D000014643B90E4B0F4A1B7810680BB981F013
:10D8E000010108F03BBE0C4B5A691AB118B91A680D
:10D8F000106058747047094A18681188084A92FBEA
:10D90000F1F2012102605974704700BF38BA00205B
:10D910003ABA00203CBA002040BA002058BA002091
:10D9200020A1070038B5264B5C69636B73B1A36D0A
:10D93000A26BD2B1998A1A88C90592B201D5D207D1
:10D9400000D438BD4FF6F7721A8038BDA36D99899F
:10D950001A88890692B2EBD59206E9D5E26AD2B16D
:10D960009888216B80B29047E1E799891A880D0663
:10D9700092B2DFD51006DDD5A26A616A8A4219D05B
:10D98000A1692569885C98800132B2FBF5F105FB3D
:10D990001122A262CEE79B88E2696169DBB28B54F7
:10D9A000E269E068A36D0132B2FBF0F100FB1122E5
:10D9B000E261BDE7DA6822F08002DA60BAE700BF10
:10D9C000203A002038B5264BDC68636B73B1A36D39
:10D9D000A26BD2B1998A1A88C90592B201D5D20731
:10D9E00000D438BD4FF6F7721A8038BDA36D9989FF
:10D9F0001A88890692B2EBD59206E9D5E26AD2B1CD
:10DA00009888216B80B29047E1E799891A880D06C2
:10DA100092B2DFD51006DDD5A26A616A8A4219D0BA
:10DA2000A1692569885C98800132B2FBF5F105FB9C
:10DA30001122A262CEE79B88E2696169DBB28B5456
:10DA4000E269E068A36D0132B2FBF0F100FB112244
:10DA5000E261BDE7DA6822F08002DA60BAE700BF6F
:10DA6000203A002038B5264B9C68636B73B1A36DD8
:10DA7000A26BD2B1998A1A88C90592B201D5D20790
:10DA800000D438BD4FF6F7721A8038BDA36D99895E
:10DA90001A88890692B2EBD59206E9D5E26AD2B12C
:10DAA0009888216B80B29047E1E799891A880D0622
:10DAB00092B2DFD51006DDD5A26A616A8A4219D01A
:10DAC000A1692569885C98800132B2FBF5F105FBFC
:10DAD0001122A262CEE79B88E2696169DBB28B54B6
:10DAE000E269E068A36D0132B2FBF0F100FB1122A4
:10DAF000E261BDE7DA6822F08002DA60BAE700BFCF
:10DB0000203A002038B5264B1C68636B73B1A36DB7
:10DB1000A26BD2B1998A1A88C90592B201D5D207EF
:10DB200000D438BD4FF6F7721A8038BDA36D9989BD
:10DB30001A88890692B2EBD59206E9D5E26AD2B18B
:10DB40009888216B80B29047E1E799891A880D0681
:10DB500092B2DFD51006DDD5A26A616A8A4219D079
:10DB6000A1692569885C98800132B2FBF5F105FB5B
:10DB70001122A262CEE79B88E2696169DBB28B5415
:10DB8000E269E068A36D0132B2FBF0F100FB112203
:10DB9000E261BDE7DA6822F08002DA60BAE700BF2E
:10DBA000203A002070B4EFF31186502383F31288DB
:10DBB000836B1A68D20720D45D686DB9446A826AA3
:10DBC000944217D081691144D9600ED9A21A5A60C3
:10DBD0008462002280F85C201A6842F00102F1B2EF
:10DBE0001A6081F3118870BC704701698A1A5A6003
:10DBF0008562EEE7012380F85C30F3B283F311888D
:10DC000070BC704703685B6A03B11847704700BF78
:10DC100003681B6A03B11847704700BF2DE9F04F36
:10DC2000BC4B1E788BB0002E40F08180BA4BBB4CB1
:10DC30001D78BB4FDFF80CB305F00105A4F10A090C
:10DC400054F80A0CB8B14FF0CC0808FB069808F05D
:10DC50007FF880B154F80A0C08F072F814F8023C0E
:10DC6000024683B924283BD075B354F80A0C08F057
:10DC70006FF80028EED10136032E04F1CC04DFD179
:10DC80000BB0BDE8F08F012B2ED0022B33D0032B2D
:10DC900040D0042B00F06981052B00F05781062B42
:10DCA000E3D114F801ECBEF1000F00F0D881BEF111
:10DCB000010F00F01B8201360023032E04F8023C02
:10DCC00004F1CC04BCD1DBE7232A54F80A0C00F0A1
:10DCD0008281944B93F83A309342B8D1FBF70EFA15
:10DCE000012304F8023CC0E74D2800F067810023BF
:10DCF00004F8023CB9E700233C2804F8023C00F099
:10DD000057813E28B1D10122032304F8012C04F8E5
:10DD1000023CAAE7C028EAD80021042304F8050C35
:10DD200004F8040C04F8061C04F8023C9DE77E4B42
:10DD300018680028A4D008F097FEDFF80CA27B4DED
:10DD4000DFF8F891DAF8000008F002F8002897D020
:10DD5000DAF8000007F0F4FF09281BD03F2819D09B
:10DD60002B68002B67D1042800F0BA810C2800F042
:10DD7000CA807F28E6D0A0F12002D2B25E2AE1D884
:10DD80000BB92028DED05A1C09F803002A6033F0B2
:10DD900075FCD7E72C68002C5AD1654FA34607F5D0
:10DDA0001C78BBF1000F08BFBB4610374745F8D1C0
:10DDB000BBF1000F00F04E81103FDBF800003A6825
:10DDC000065D135D9E42204402EB040140F0408159
:10DDD000661E4E4422460BB9FD2A5CD906F8013F67
:10DDE00001322A6010F8013F11F801EF9E45F2D090
:10DDF0000AB15F4512D04F4833F048FC5F4508D365
:10DE00005BF8100B33F042FC092033F037FCBB45C4
:10DE1000F6D9494833F03AFC2A680024944291D25A
:10DE2000661E4E4416F8010F33F028FC2B680134AF
:10DE30009C42F7D386E70C2865D00A2834D00D28F9
:10DE400032D07F2800F0BE80FF2B3FF67BAF92E7F9
:10DE5000374E002706F51C78BB4602E010364645D3
:10DE60000DD022463168484609F05AF90028F5D10C
:10DE7000B346002FF2D1374610364645F1D13B4626
:10DE80005F469B46002B98D1002F3FF45BAF29489B
:10DE900033F0FCFBB4E7511C202009F80200296094
:10DEA00009F801300A46A4E733F071FC2321234826
:10DEB00036F072FE002800F01181A0EB0900286006
:10DEC00090B1431E19F80310202940F02C8109EB72
:10DED000030243B112F8011D202903F1FF304FD195
:10DEE0000346002BF6D12B604FF480720021484688
:10DEF00036F03BFE074B1B78002B3FF4C1AE0E48BB
:10DF000033F0C4FB1EE70E4833F0C0FB0A4833F081
:10DF1000BDFB17E7B5C600200C910020227C002035
:10DF2000781F00203C980020543E0020C03F002075
:10DF3000EC510408787F0408807F0408C03E00206C
:10DF4000887F0408AC4C0408BC3E002014F8063C52
:10DF500014F8051C99426FD814F8043C83427FF4EE
:10DF6000C6AE062304F8023C9BE614F8043C04F811
:10DF7000030C5A40052304F8042C04F8023C74E610
:10DF80002B606A4C002204F51C7809F8032002E09B
:10DF9000103444454CD02168484615F02DFD00282A
:10DFA000F6D0444544D2E368984700232B609BE7B2
:10DFB000032204F8013C04F8022C56E6022304F87C
:10DFC000023C52E6013B002259482B6009F803202D
:10DFD00033F05CFBB6E6574B5749DB78574ADFF81E
:10DFE00088E11060003318BF01230B70544B554A71
:10DFF000CEF80030544B3A614FF0400E012187F8C3
:10E0000018E0F86078617D765048197033F0ECFDC7
:10E010004F4833F03BFB4FF4006010F063FB4D4B77
:10E0200093F83A30232B3FF459AE14F8023C36E60D
:10E03000494833F02BFBB8E714F8041C08EB030045
:10E040005140013304F8041C04F8063C82720CE6CB
:10E050002246CDE64148103F33F018FBD0E69BE85E
:10E060000F000DF1280C0DF1080888E80F004CF89E
:10E0700024ED14F8053C14F803AC069462462344DE
:10E080004FF0010C414606A8ADF822E00793ADF829
:10E0900020A08DF824C005F093FD40B1029A304BCA
:10E0A00003924146A4F10A00029311F0EFF8DDF863
:10E0B0000480002304F8023CB8F1000F3FF4DBAD0C
:10E0C00054F80A0C11F0A4F9013654F80A0CC047B0
:10E0D000032E04F1CC047FF4B3ADD1E52868EFE65C
:10E0E000204814F0F1FB0BB0BDE8F08F14F8053CAC
:10E0F00014F8032C0694234407936E2A4FF0000370
:10E1000008930993ADF820207FF4D5AD06A809F057
:10E1100089F806A809F07AF806A809F077F806A8A1
:10E1200009F074F8C7E503462BE700BFEC5104087B
:10E13000B07F0408D0C600206C280020BC3E002020
:10E14000881F0020E5560108B5C60020B47F0408EA
:10E15000807F04083C980020947F0408787F04089E
:10E1600084CC0020C03E0020543E00202DE9F04722
:10E17000C44B1C6862072DED028B03D4BDEC028BEF
:10E18000BDE8F087C04D2B78002BF7D06E6846F2C3
:10E19000A713861B9E42F1D9DFF850936860B9F847
:10E1A0000070DFF84C83002F40F0A68198F806201D
:10E1B000AB689FEDB60ADFEDB60ADFF8F492013ADC
:10E1C000B3FBF2F307EE903AF8EE677AB7EE008A07
:10E1D00027EE800A35F0D4FDDFEDAE7A38EE400A46
:10E1E00020EE270A35F004FDB8F80830DFEDAA6A02
:10E1F00007EE103AEB68C01AB8EEC77A07EE900A3D
:10E20000A7EE668AB8EEE70AD9ED097AF8EEE77A62
:10E2100020EE080A67EEA67AA7EE270A35F0E8FC9A
:10E220009E4BC9F8240002461860A30740F1AA815A
:10E23000DFF8C0E29A4CDEED007A9FED9A5A216831
:10E24000F8EE677A27EE855A002900F0BB81964BDD
:10E2500007EE101AD3ED026AB8EEC77AF8EEE66A56
:10E2600086EE878A914991ED004AB8F80C10D5EDF9
:10E27000054ADFED895A95ED066A67EE847A06EE67
:10E28000901A67EE887A8A49B6EE004AF8EEE66A96
:10E29000F0EE643AE7EE843A66EEA56A91ED097A0B
:10E2A0007E49F7EE005A75EEE65AB8EEC77AA3EE4D
:10E2B000856A77EEA47A27EE257AC5ED057AF0EE29
:10E2C000477AE6EE267ABDEEE77AC5ED067A81ED6D
:10E2D000007A78490978122900F05B8100211960E1
:10E2E000596099602160CEF80010002F7FF446AF8E
:10E2F000E869EA61121A07EE102ADFED6F6A6F4BC8
:10E3000007EE906AB8EEC77AF8EE677A27EE267ABB
:10E3100040F2DC52C7EE276A0A21FDEEE67A17EEDC
:10E32000900A9042A8BF10469842B8BF184609F01C
:10E33000DBF9B8F80A309FED586AD5ED056A07EEAB
:10E34000103AB8EEC77AF7EE007AE7EE467A05EEB5
:10E35000900AF8EEE55A66EE866A67EEA57AE7EE71
:10E36000267AB0EE670AC5ED057A35F041FC052145
:10E37000064609F0B9F9524A5249B2F9004008601C
:10E3800084EAE473A3EBE473B3F5487F74DAB2F97B
:10E39000022082EAE273A3EBE273B3F5487F6BDA03
:10E3A000494B1B78002B40F01181484B3B4A1B68BE
:10E3B000126847489B1AB3F5FA7FA8BF4FF4FA7367
:10E3C0009842B8BF18460A2109F08EF9414B1C68E3
:10E3D000637A00FB03F00028B8BF7F30C211B2F5AA
:10E3E000967F3D4BA8BF4FF496729A42B8BF1A462B
:10E3F0003A48E37E076895ED087ADFED396A911BAC
:10E4000001FB03F3227F344E002B01FB0272B8BFE5
:10E410001F335B11B2F5C81F3249A8BF4FF4C812B1
:10E42000B3F5967FA8BF4FF496738A42B8BF0A46E9
:10E43000617F026007EE901A37EE087AF8EEE77A0D
:10E4400027EE267AB34267EE877AB8BF3346002AB2
:10E45000B8BF02F5FF52FDEEE77AB8BF1F3203EBFB
:10E46000623317EE902A962A6FF09501A8BF962284
:10E470008A42ACBF9F1A5F1A1B4A85ED088A176053
:10E480007CE600BF5C460020D41F0020089425379E
:10E49000B1DC423ED048874A6F12833A6046002082
:10E4A000F0B20020BD378635E0B200206CB8002005
:10E4B000E05B002038BB00200024744924FAFFFFF1
:10E4C0006846002064460020C4260020BC260020A8
:10E4D0000CFEFFFFBC460020D4FEFFFFB426002048
:10E4E0000000003B0000E7FFAC2600207ACC0020B3
:10E4F0001C560020ECB20020374998F806A00A68A4
:10E50000AB689FED360ADFED360A002A0AF1FF3AC2
:10E51000B3FBFAF39246B8BF02F1070AA2EBEA0294
:10E5200003EB020ABAF1000F5346B8BF0AF1070322
:10E53000DB1007EE903AF8EEE77AC1F800A027EE7C
:10E54000800A35F01DFCF7EE007A77EEC07A9FED79
:10E55000257A2B6967EE877A9A4518BF07F1FF3352
:10E56000FDEEE77A14BF9FB200274FF00003C5ED20
:10E57000037A18BFC5F810A0A9F800706B61AB61F1
:10E58000002252E69FED188ADFF870E0174C184B16
:10E590009FE695ED057AD5ED067ADFF864C0206830
:10E5A000996891FBF0F1BDEEC77AFDEEE77A17EEC0
:10E5B000100A17EE909AACF80200ACF80010ACF814
:10E5C00004908BE69FED088A094B4BE6094A0A4BFB
:10E5D00012681C680CE700BF1C0000200894253757
:10E5E000B1DC423ED048874A00000000F0B2002073
:10E5F000E0B20020C0260020BC460020ECB2002083
:10E600003CBB00202DE9F843304B1B685B0701D46D
:10E61000BDE8F8832E4C2F4D94F82490B9F1010FEA
:10E6200048D1EB69284698472B69284698472B6ABA
:10E6300004F12C0004F128019847274B276B9B79A4
:10E64000A668E06A07F101089845636B08BF84F883
:10E65000009003F1010208BF4FF00008032A1FD009
:10E660001E49626394F8382041F82300FAB904EB9C
:10E67000870704EB8803F863DA6BAB89C4F8308052
:10E68000B61A30440022A06084F82420002BBFD0AA
:10E69000134A0A2B1268B8BF0A231361BDE8F88336
:10E6A0000E4B01229860002384F83820636320F029
:10E6B00029FCDCE76B6928469847AB6928469847F0
:10E6C0000122EB8984F82420E0E700BF5C460020AB
:10E6D000D41F0020E05B00201C5600204061002079
:10E6E0003C560020F8B5534B1B681C0700D4F8BDFE
:10E6F000514C524E524D736804F1FC0107463046AE
:10E700009847B4F9FC00B4F9FE20B4F90031317E29
:10E71000286028466A60AB601FF01EFA494A1378E9
:10E7200059073ED4D4F80401474B1B7883B1474BBB
:10E730002968B3F90AC0B3F90CE0B3F90E606A684E
:10E74000AB68A1EB0C01A2EB0E029B1B85E80E004F
:10E750000028CCD03E4B381A98423FD9B4F9145116
:10E76000B4F91011B4F90871B4F90A21B4F91261BD
:10E77000B4F90C313548394432442B4401EBD171A2
:10E7800002EBD27203EBD3735B10491052100025D9
:10E7900041818281C381C4F80451BDE8F840FEF78D
:10E7A00025B92C4EB5F90000B5F90410A4F80801FC
:10E7B00023F0040313700022B5F90830A4F8100107
:10E7C000C4F804713260B280A4F80A11A4F81211DE
:10E7D000A4F80C31A4F814313846A5E7002007F05E
:10E7E000D5FA2B68B4F908219342B4F91021B8BFC7
:10E7F000A4F808319342C8BFA4F81031B4F90A2133
:10E800006B689342B4F91221B8BFA4F80A3193425D
:10E81000C8BFA4F81231B4F90C21AB689A42B4F91C
:10E820001421C8BFA4F80C319A42BFF660AFA4F817
:10E830001431F8BD5C460020D41F00204C5C002041
:10E8400000C70020B84600209C5C00203C580020F7
:10E850007FC3C901465800202DE9F047C74C6368C3
:10E8600020469847002800F0C380C54B1B78012242
:10E87000042B84F83C2000F0BD80B4F91610B4F9E4
:10E880001820B4F91A3021636263A363BD4B1B885F
:10E89000002B69D0BC4DD4ED0C7AD5ED004A95ED36
:10E8A000050A95ED015A95ED067AD5ED035A95EDD9
:10E8B000026AF8EEE76AD5ED047AA4EEA60AA5EEA0
:10E8C000267A67EEC07AA5EEC07AE6EE267A85ED66
:10E8D000057AC5ED067A35F08BF9D4ED0D6AD5EDE4
:10E8E000094A95ED0E0A95ED0A5A95ED0F7AD5ED88
:10E8F0000D7AD5ED0C5A95ED0B6A2063F8EEE66AB9
:10E90000A4EEA60AA5EE267A67EEC07AA5EEC07A36
:10E91000E6EE267A85ED0E7AC5ED0F7A35F068F9C8
:10E92000D4ED0E6AD5ED124A95ED170A95ED135AFE
:10E9300095ED187AD5ED167AD5ED155A95ED146A40
:10E940006063F8EEE66AA6EEA40AA6EE857A67EEA4
:10E95000C07AA0EE657AE6EE867A85ED177AC5ED87
:10E96000187A35F045F9A063884FA17F88481FF0D9
:10E97000F3F83B88002B40F08480864ED6F818517F
:10E98000854B1B685B0743D4B5F90070216B636B43
:10E99000A06B824A824E92ED026AD2ED006AD2EDFD
:10E9A000015AC91B2163B5F90270DB1B6363B5F91A
:10E9B00004703568C01B07EE900AB8EEE75A07EE00
:10E9C000901AB8EEE77A07EE903AF8EEE77A36EE6C
:10E9D000056A36EE877A77EEA57A0135A06382ED77
:10E9E000026A82ED007AC2ED017A3560BDE8F087F7
:10E9F000BDE8F0876B4BB4F91600B4F91810B4F900
:10EA00001A2018802063598061639A80A2633DE7D1
:10EA1000B6F82821322A00F08880002A66D196F8BC
:10EA20004631002BB0D06048D6F838215F4980FBD2
:10EA30000273D217C2EB23122A80D6F83C2180FB46
:10EA40000273D217C2EB23126A80D6F84031A78A2C
:10EA500080FB0302DB17C3EB2213DB1BAB8000231D
:10EA6000CB6086F846312EF01DFF08F011F92EF02C
:10EA700001FFFDF71BFE012030F0D0F8D6F8185149
:10EA800082E7444E226BD6F81851B3F5C87F4FF099
:10EA9000000323632B80398818BFD6F81C01B7F810
:10EAA000008008BF0020B1F5C87F18BFD6F820311C
:10EAB000616B02440B440020B8F5C87F6063C6F860
:10EAC0001C21C6F82031688052D0D4F838E0D6F83E
:10EAD0002411A0637144B8F1010FA880C6F8241175
:10EAE00068D008F1FF38A7F8008049E7D6F8380168
:10EAF000236B00210344C6F8383121632980D6F8FE
:10EB00003C01636B61630344C6F83C316980A36BCD
:10EB1000D6F84001A1630344012AC6F84031A98018
:10EB200075D0013AA6F8282179E72B8820491F489B
:10EB3000276BA6F82C310023B5F802E0B5F804C025
:10EB4000C0684B608B602363C6F838712B80616BA3
:10EB5000C6F83C1163636B80A16BC6F84011A363D8
:10EB6000A6F82EE1A6F830C1C6F83401AB80D8E78C
:10EB7000A36BC6F82431A063A880B2E770460020DA
:10EB800038BB0020185D00201C5D00207CCC0020DC
:10EB9000A0460020D41F0020B4AC0020ACB200205E
:10EBA000A8B200203CBB00201F85EB512C58002050
:10EBB0000C210020DFF88CC0DFF884E0C8328CFB29
:10EBC00002A9C833D217C2EBE9128CFB03A9DB17E9
:10EBD000C3EBE913C8316B802A808CFB013CA28A0D
:10EBE000CB17C3EBEC139B1AAB80CEF80C002EF0C6
:10EBF00059FE08F04DF82EF03DFEFDF757FD40465A
:10EC000030F00CF8B7F80080D6F8185169E70B20FF
:10EC100086F8441186F845212FF0DAFED6F818510F
:10EC2000074BB6F82C21B6F82E71B6F83001D6F89D
:10EC300034112A806F80A880B6F82821D96070E747
:10EC40002C5800201F85EB512DE9F04F2DED028B44
:10EC50009F4BA04A1C7897B000F59C41203181461B
:10EC600009911160002C00F004859B4A12689042C3
:10EC700040F28380994A089216689949994ADFF8C8
:10EC8000A0A20791013C04921C7006F48056002E4D
:10EC900040F08180944B1B78022B00F05187042BAD
:10ECA00000F04087012B00F0F486904B99459AF8CC
:10ECB000023000F2B283002B40F0B3838C4B0993F7
:10ECC000089B1E6816F4805740F0A184DFF8549228
:10ECD000049BB3F90610079B5C8BA142B4BF0024D0
:10ECE0000124844B1B6813F080535ED0099A12787C
:10ECF00012F001025FD00798408C884241F33580C2
:10ED0000002C5ED17C4D95F8D411002959D17B4857
:10ED10007B49006890F82D0000250D604D608D60E6
:10ED2000784900284ED10870002A4FD0F1064DD501
:10ED3000754A1278D20649D4002F47D1002B45D10D
:10ED4000750243D4714B1B78002B01F0AA86704BDF
:10ED50009B78002C41F050873BB16E4A6E4B126895
:10ED60001B689B1A002BC1F22C871020624D2FF0DC
:10ED70002FFE012385F8D53128E0584B08931E68F3
:10ED8000574A584B079206F480560493DFF890A137
:10ED9000002E3FF47FAF0021564808F077FF00288F
:10EDA0007FF478AF15F006FC74E770029ED4099AE0
:10EDB000127802F00102504D002185F8D411002C88
:10EDC000A5D0504901200870002AAFD1534B1A78C2
:10EDD000002A40F0B3800799049D488BB5F9007074
:10EDE000898BB5F902508742CCBF8026002646F0B9
:10EDF00040038F42A8BF33469B0843F080068542FC
:10EE0000C8BF3346049F43F040068D42B8BF334627
:10EE10009B08B7F90450B7F9066043F080078542B4
:10EE2000C8BF3B4643F040078D42B8BF3B469B08F6
:10EE300043F08007304D8642C8BF3B4643F0400751
:10EE400095F8D6E18E42B8BF3B469E4501F0B281AF
:10EE5000A5F8D82185F8DA212C4985F8D6310E7825
:10EE6000002E01F0C3805F2B01F04D816F2B01F06C
:10EE70008D81099B1B78DB0760D495F8DA11002996
:10EE80005CD1B5F9D831322B58DD95F8D621012067
:10EE9000572A85F8DA0101F09F84089B1B685C07FC
:10EEA00040F1E7875A2A40F0E48795F84531002B76
:10EEB00041F0078695F8DC3183F0010385F8DC31F9
:10EEC000002B41F0A5860C202FF082FD01F02FB918
:10EED00074C100207CC0002070C10020B4AC0020B0
:10EEE0001098002084900020DEC00020404B4C0091
:10EEF0000C910020E4570020D41F0020BC460020C5
:10EF0000C85B002064260020B8460020781D002041
:10EF10004C58002060BA0020D43F002077C7002062
:10EF20001C40002084C900200F202FF051FDB5F8AF
:10EF3000D83185F8DA41FA3BA5F8D831089BB34AB5
:10EF40001B680692B24C5F0700F17A840DF1500BFA
:10EF5000DFF8E4820A940023CBF80430454614938A
:10EF6000192740F6330340F28336049C02E004354F
:10EF70004D4524D0A878E978884217FB006EF6D278
:10EF800095F801C00CF1040C17FB016034F91C105A
:10EF90009942A8BF1946B1F5617FB8BF4FF46171BE
:10EFA0008E45E4DA8842E2DB29782729DFD8584603
:10EFB0000435059308F05AFE4D45059BDAD1954B73
:10EFC000954A1B780A9C9BE8030082E80300002B0B
:10EFD00040F01781914B1F78002F00F0BB83012177
:10EFE0008D4808F053FE002840F04A819AF803301B
:10EFF000002B40F0458123881DB225F00105AEB2FB
:10F00000B342268000F0C185854D02270E204FF0C7
:10F0100014094FF0FF082F7085F8019085F80280E1
:10F020002FF0D6FC39467C48268808F02FFE0028B1
:10F0300041F03A8026F002039BB2B34223800AD00B
:10F04000774B1421FF2202250E201D7059709A70F3
:10F050002FF0BEFC2688DFF8E4A1DFF8E4B19AF8CF
:10F060000010DBF80400B50708BF81F00201C1F30E
:10F07000400107F073FA2421674808F007FE30B911
:10F08000099A1378590744BF23F004031370069BB1
:10F090001B6813F00A0F1DD005215F4808F0F6FD2C
:10F0A000002800F0388625886F0740F1B4875A4859
:10F0B000062108F0EBFD002800F01A866E0640F1EC
:10F0C000A2870721544808F0E1FD002840F0B885E8
:10F0D000069B1B689D0600F10E8326884E480C2176
:10F0E00008F0D4FD002800F0E68046F48073B342B7
:10F0F000238009D04A4B02251421FF220E201D70C7
:10F1000059709A702FF064FC464B1B78082B00F066
:10F11000DE800E2B00F0DB80089B1B685D0548D568
:10F12000414B1B79002B00F08F8014213A4808F0E6
:10F13000ADFD002840F08D801BF02AF901202FF052
:10F1400051FB002835D0DFF8FC8000254FF0CC09BA
:10F1500002E0DDB2022D2CD809FB05F76B1C58F834
:10F160000760002EF5D1032290F902300296019239
:10F17000C2782E4951F82220009218463246334672
:10F1800001212EF025FF034605EB450000EB0010A2
:10F19000059353B1314608EB8000CC2235F0E5FCF5
:10F1A000059B48F807300135EDB223F0CFFF00286A
:10F1B000D0D1099B1B78D80740F19C809AF80010A9
:10F1C0001B4A1C4DDBF80000012301F00101137004
:10F1D0002B7007F0C3F9069B1B685A0700F1FE80ED
:10F1E00017B0BDEC028BBDE8F08F98F8022098F8BC
:10F1F00003309A42C0F0328608F10408A8453FF473
:10F20000E9AE98F800102329F6D1EEE75C4600201D
:10F2100046460020B05D0020E4570020B5C600201F
:10F22000583E0020405C002044BC0020D068040808
:10F23000D02600200D91002034C9002028BA0020DB
:10F240002CBA0020187C0020099B1B78D9077FF579
:10F2500073AF4FF40F7020F03FF80028A9D010F0E2
:10F26000CBF94FF40F701FF0CFFF0028A1D010F0A2
:10F27000C3F94FF40F701FF0C7FF0028EFD198E7D4
:10F28000069B1B689A077FF5B6AE2688F3073FF505
:10F29000D1AE46F001039E4223803FF4CBAEB54B86
:10F2A0001421FF2202250E201D7059709A702FF034
:10F2B0008FFB2688BEE626F480739BB2B342238080
:10F2C0007FF418AFAC4B1B78082B7FF422AF228859
:10F2D00022F040039BB29A4223803FF41DAFA54B1E
:10F2E00002251421FF220E201D7059709A702FF0F4
:10F2F0006FFB11E7A14B1E78002E65D1A04B1B6858
:10F30000002B61D0DFF8C482DFF8C49218F8030C38
:10F3100099F804704146A8F1030528F051FD002832
:10F3200000F03B85002F40F08C8505F108016879DD
:10F3300028F046FD002841F097839249A87A28F0EA
:10F340003FFD002800F03C85022F41F071838E497B
:10F35000E87B28F035FD002841F066838B49287D45
:10F3600028F02EFD002800F03C85042F41F08C830E
:10F370008749687E28F024FD002841F08183854973
:10F38000A87F28F01DFD002800F03C85062F41F0E5
:10F390007383814995F8230028F012FD002841F07D
:10F3A00067837E4995F8280028F00AFD002800F0C0
:10F3B0003C85082F41F04983794995F82D0028F0C4
:10F3C000FFFC002840F03C85764B01221A7033F098
:10F3D00093F9069B1B685A077FF502AF032028F0BC
:10F3E00027FD002800F0FE86238813F008047FF430
:10F3F000F7AE08200FF05EF9049E6B486B4D6C4928
:10F400006C4A6D4BF68800682E80086014601C60A2
:10F4100017B0BDEC028BBDE8F08F13B901238AF859
:10F420000230664B09931B201D789AF8214028F082
:10F43000FFFC012C05F00108814600F07F8605F0F5
:10F44000020305939AF820305D4EDFF888B15D4FD6
:10F45000052B00F2CF80DFE813F0BF00820006002A
:10F46000FD00FF00F200012C04BF05238AF82030C4
:10F47000B8F1000F12D0079B3088B3F918100022A2
:10F48000134661F30F0260F31F4261F30F03049808
:10F4900061F31F4303600323426005934A4DDAF88A
:10F4A00014202B689A4280F0918547F23052032352
:10F4B000CAF81C208AF8203002200FF013F915F04A
:10F4C00079F82A68DAF81C3013440422CAF8183094
:10F4D0008AF82020012C40F0CB862B68DAF818201F
:10F4E0009A4280F087809BF8000018B928F0A0FCB1
:10F4F00000287FD13B6823F002033B602A687388B1
:10F50000642101FB03234FF480600022CAF810300D
:10F510008AF820208AF803200FF0B4F89AF82030F7
:10F5200096E728F08BFC012807D1274D73882A68BD
:10F53000642101FB0323CAF81030B9F1000F02D097
:10F54000B379002B7DD1012C54D01F4DDAF8102057
:10F550002B689A42C0F0948601238AF82030012C4F
:10F560006DD0F379012B79D028F0E8FB9AF82030A0
:10F570006EE700BF583E0020405C00200D91002047
:10F5800010910020243E0020293E00202E3E002025
:10F59000333E0020383E00203D3E0020423E002009
:10F5A000473E0020D026002060460020B0260020E4
:10F5B000BC260020B4260020AC2600200C910020A0
:10F5C00070B80020B446002060BA00201A3E002027
:10F5D0001C000020781D0020B8F1000FA1D14FF4CD
:10F5E0008060B9F1000F00F0EE820FF063F80023A5
:10F5F000CAF81030059B002B3FF462AB18462FF081
:10F60000E7F9089B1E6816F480573FF45FAB1D2195
:10F610009E4808F03BFB00287FF458AB9C4B03F15D
:10F62000500903E00433994500F0E1851A78262A51
:10F63000F8D19978DA789142F4D2FFF749BB954D29
:10F640005CE728F07BFB03224FF47A738AF82020D2
:10F65000CAF81C308F4D2FE78E4D3BE728F06EFB2C
:10F66000032240F6B8338AF82020CAF81C30894DAE
:10F6700022E7894F3B78002B01F00C81874BDFF8A4
:10F680005082DFF850B2DFF850A2079345465E463D
:10F69000049099460EE019F804109847032C28DCD2
:10F6A00088B93B782AF8020F01349C4205F1040521
:10F6B00080F21881072CE1B23046DBF80430EADD35
:10F6C000984700B2EDE738F824206B88801A4FF491
:10F6D0007A719B1A01FB00F040F6CA0290FBF3F02E
:10F6E0000844904240F2EE23A8BF10469842B8BFAB
:10F6F000184600B2D5E76A4B1B78980704D5694DC8
:10F700002B7D042B00F2EE85268816F0300F3FF497
:10F71000E5AC10200EF0B6FF20200EF0B3FF624BD8
:10F72000268800221A70614A6148624F624D0021AA
:10F730001160624A39600023296041608161036081
:10F7400083604361C3611360516093605361916151
:10F75000D361C3E4DFF884B1DFF88481584D0BF145
:10F760005A064FF0010959461BF8010C28F028FBF6
:10F77000F8B19BF804009BF802309BF803E000EB23
:10F78000400105EB8101013BD1F8E42103EB430388
:10F79000434493420DD095F8102281F8E0E109FA34
:10F7A00000F022EA0000C1F8E431C1F8E87185F800
:10F7B00010020BF1060B5E45D5D14249354A424B4A
:10F7C000424D09681B78D2F800900A910593A5F57F
:10F7D000F07B00266B6863B31F7857B3AA68A9EB68
:10F7E0000202002A0ADB9BF810220121B14022EA22
:10F7F000010209F5FA718BF81022A960059AC2B1CD
:10F800002A7859780432D2B2002940F0B48207999C
:10F810000498098B30F9122001F1C800824240F3AC
:10F82000F8849BF810129A7841FA06F3D80740F151
:10F8300097850136042E05F10C05CBD1FFF7CFBB20
:10F840001F4D95F8DC315BB1099B1B78DE0707D5AE
:10F85000049BB3F90620079B5B8B9A4200F36F85EC
:10F8600011210A4808F012FA002800F06C8295F87D
:10F8700044312BB995F8453113B93223A5F8283115
:10F88000012385F84431FFF761BB00BFE457002036
:10F8900034C9002060BA0020F8C900201098002068
:10F8A000B846002050610020584200204443002008
:10F8B000F4420020382600202C2700201C43002082
:10F8C000D41F0020C046002010400020B42100209A
:10F8D00010CA002018C700201A210020313D002046
:10F8E000BC4C0408DDF81090B84AB9490892126877
:10F8F000A1FB091B42F2010111404FEA9B1B0F9132
:10F9000000F01E82B34DB448B44CB5492E7800784F
:10F91000267008701EB1B2490E7886F00106B14D0E
:10F920000F2185F86C11002B00F09283AE4B079CE1
:10F930000E93B4F824E0B4F826C0079CCDF82CC090
:10F940001846248B0078A94B1294A94C0D9004946E
:10F950000446A3FB00035B0803EB4303E31ADBB29B
:10F9600095F86D810A9302F4805205F5B8700BF595
:10F970009673119597F800A0DFF8BCC29C4C0C91CF
:10F980007546DDF83CE01392002106930596CDF80C
:10F990004090059B002B00F09282964B33F911307A
:10F9A0001FFA83F9A9454FEA410203D30B9EB145E3
:10F9B00040F2C9825CF821309B4580F08982A35EC9
:10F9C000BEF1000F40F09E8201315145A35200F17B
:10F9D0000600DEDB0C9A119D874B85F86C210F2AFF
:10F9E0000CBF01220022DDF8409085F86D811A706D
:10F9F00000F035837848DFF844A279497F4D012231
:10FA0000027004200A700EF06DFE2B68DAF8081000
:10FA1000DAF80420CAF80C305B1A934284BF002342
:10FA20008AF821303C78089B1E68002C00F048873B
:10FA3000079A734DB2F824E0178B6D4916F480567F
:10FA4000284640F0428332460EE0437803EB8303BE
:10FA500003EB830303F2EE239BB20132A24221F8AF
:10FA6000023B00F102000ED015F81230002B00F01E
:10FA70006E82022BE9D001320B8821F8023BA242B0
:10FA800000F10200F0D10E9A137801331370FFF7E2
:10FA9000FEB8544DD5F8D031A9EB0303002BFFF687
:10FAA00004A9584A584B527C079933F812308A7D82
:10FAB000DFED566A9FED566AC97D9BB207EE102AAC
:10FAC00007EE903AB8EEC77AF8EEE77A27EE267A94
:10FAD00067EE867A099AC5F8D021C7EE876A40F2A8
:10FAE000FF32FCEEE67ACDED057ABDF81430934294
:10FAF00028BF134609B1D31A9BB24648464D017838
:10FB0000464C35F81160226825F81130921B1344D9
:10FB10000131434D236001F00F021B0902702B805D
:10FB2000FFF7C3B8FDF774FD3E4B3F4A1B68C31A8D
:10FB300093427FF7BAA83A4B00221A80FFF7B5B874
:10FB4000079A0499537DD27D013B31F913301AB1E4
:10FB5000C3F53B6308331BB2A3F57A7307EE903A03
:10FB60009FED327A2E4AF8EEE77A40F2FF3167EEE7
:10FB7000877AFCEEE77ACDED057ABDF814308B423A
:10FB800028BF0B461380FFF790B80221284808F0E1
:10FB90007DF800283FF44EAA2580B7073FF55BAA01
:10FBA00046F00203B34223803FF455AA214B0220C2
:10FBB0001421FF2218700E2059709A702EF008FF41
:10FBC0002688FFF748BA0EF05DFD10E5B4AC0020C2
:10FBD000D34D621058C00020681D00201040002046
:10FBE000691D0020D41F0020E9C80020ABAAAAAAE2
:10FBF000849000201C21002086C7002060BA0020CD
:10FC000044CA0020B0BA0020D0BA00200000C84288
:10FC100000008044DFC00020E4C00020E0C00020DD
:10FC200044460020D824002060E316006F12833F72
:10FC3000E4570020583E0020ECC800201C40002063
:10FC4000CD4AB2F90030002BB8BF5B42B3F5E17F7B
:10FC5000BFF63EAAB2F90230002BB8BF5B42B3F543
:10FC6000E17FBFF635AAC54B93ED057AD3ED077A50
:10FC7000D3ED096A93ED030A77EEA67A30EE070A10
:10FC8000F7EE000AB0EE007AE7EEC70A30EE000A9F
:10FC900007F048FDB6EE008A20EE488A9FEDB80ACC
:10FCA00038EE000AFDEEC07A17EE903A2033402B72
:10FCB00040F253839FEDB30AB34DDFEDB27A85ED89
:10FCC000000ABDEEC87AC5ED017A17EE103A20336E
:10FCD000402BC5ED027A00F29E85B0EE480A07F08F
:10FCE00097FC0A2085ED030A2EF072FEFFF7F0B9AB
:10FCF00025F040039BB2AB4223803FF4E2A9A34B23
:10FD000002251421FF220E201D7059709A702EF0CA
:10FD10005FFEFFF7D6B9238823F00405ADB2AB42EE
:10FD200025803FF4C4A9994B02251421FF220E20FF
:10FD30001D7059709A702EF04BFE2588FFF7B7B9E9
:10FD400093490E78E6E595F84531002B3FF4FEA87F
:10FD5000099B1B7813F001037FF4F8A8012285F8B2
:10FD6000453185F84621FFF7F1B88A4D012185F824
:10FD7000D411FFF726B8012900F0F0849BF8102277
:10FD80000123B34001361343042E8BF8103205F1E2
:10FD90000C057FF41FADFFF722B908F10501687962
:10FDA00028F00EF800283FF4C8AA012F40F05C8626
:10FDB00005F10D01A87A28F003F8002840F03886F4
:10FDC0007549E87B27F0FCFF00283FF4C7AA032F02
:10FDD00040F02A867149287D27F0F2FF002840F084
:10FDE00053866F49687E27F0EBFF00283FF4C7AACF
:10FDF000052F40F045866B49A87F27F0E1FF0028DA
:10FE000040F03A86684995F8230027F0D9FF00288A
:10FE10003FF4C7AA072F40F02B86644995F82800C5
:10FE200027F0CEFF002840F01086614995F82D009C
:10FE300027F0C6FF00283FF4C7AA092F3FF4C4AA41
:10FE40000926334603EB83031D445A4B6978AA788D
:10FE500089F8046019705A70FFF7B6BA564807F06F
:10FE600015FF00283FF4B6A814202EF0B1FDFFF7CF
:10FE7000B1B85D2A00F079825B2A00F01D855E2A08
:10FE800000F05E85562A00F06E85972A00F0E18525
:10FE9000A72A00F04985494C23889B0740F0148528
:10FEA000A2F1B703072B00F28A82DFE813F0820287
:10FEB0008802880288027C0288026E026E02002D8F
:10FEC0003FD05CF821309B454FEA4102FFF477AD0B
:10FED0003B4B3B4E9B5C06EB0209002B00F0D780AE
:10FEE000022B47D199F8013003EB830303EB830323
:10FEF00003F2EE239BB2032933DD1BB2BEF1000FE8
:10FF00003FF462AD0A9E20F81630B8F1000F03D11D
:10FF10000D9E022E7FF658AD4388B0F80090B0F8E1
:10FF200004804B449844274B0FFA88F883FB0863FE
:10FF3000254EA3EBE87326F802801BB24FF00108B0
:10FF400042E52B464A00069E4CF8216038E5D3B2C4
:10FF5000022B04D9032B7FF48EAD73467DE53B461F
:10FF60007BE5012606FA01F90C9E26EA09061BB27A
:10FF70000C9625E5A35ABEE7684600200817002026
:10FF8000DB0FC93F00000000A0000020583E002009
:10FF900010400020D41F0020293E00202E3E0020CB
:10FFA000333E0020383E00203D3E0020423E0020EF
:10FFB000473E002014910020E457002046460020D0
:10FFC00044CA0020565555558C210020B24B1B7851
:10FFD000002B7FF46AAAB8F1000F3FF466AA012C47
:10FFE0007FF408AB9AF82030FFF732BA3146AB48BD
:10FFF00007F04CFE002800F0A58085F8DB6114F0C6
:020000040801F1
:1000000009FFFEF736BF45F04003AB4223807FF483
:1000100076AEFFF756B845F004039D4223800AD020
:100020009F4B02251421FF220E201D7059709A70DB
:100030002EF0CEFC25889B4B9B4AB3F904309B499C
:1000400082FB0302DB17C3EBA2030B80FFF72FB881
:10005000974B984A0E9201221A70974B04931B21DA
:100060008E4807F013FE00287FF4C4ACDFF870A2BE
:10007000924DDAF80C202B68CAF808309B1AC82B6E
:1000800000F20C84089B1E6806F48056FBE4CBB299
:10009000022B40F26083032B7FF46CAF129B139E04
:1000A000002E08BF2B4626E726F001039BB2B34281
:1000B00023803FF472AD0E202F7085F8019085F8F3
:1000C00002802EF085FC268867E500220FE0437849
:1000D00003EB830303EB830303F2EE239BB20132B2
:1000E000A24221F8023B00F102003FF4CCAC15F82B
:1000F00012301BB1022BEAD00B88F0E7D3B2032BEE
:10010000FAD83B46EBE7B2F5FA7FFEF617AF95F863
:10011000DA31002B7EF412AF099B1B78012213EA1F
:10012000020485F8DA213EF4FFAE14F043FA644B82
:100130000693089B634C1B68FEF705BF00230593DD
:10014000FFF780B9099B604A1B781060D8077EF5DD
:1001500094AE5E4B1B78002B3EF4F0AE9AF8033061
:10016000002B7EF4EBAE95F8DB310133DBB2032BD1
:1001700085F8DB317EF6E2AE554B5B7813B9002C87
:100180007EF4DCAE14F016FAFEF773BEB2F5FA7F19
:10019000FEF6D4AE95F8DA21002A7EF4CFAE099BA4
:1001A0001B78012185F8DA11D90700F16A8314F070
:1001B00031FEBCE7474A48491068B5F9D821C669FD
:1001C00081FB06018911F617701A00F5FF407F3098
:1001D00082423EF741AE891B0A4412B2A5F8D821EB
:1001E000FEF73ABE08200EF04DFAFEF7F9BF3B4A83
:1001F000079BD488049A1B8BB2F906101A1B9142F4
:1002000040F39A8023449942B4BF00240124FEF7AE
:1002100068BDC8398A4280F282809BF810129A78B1
:1002200041FA06F3D9073FF504AB524201200B9285
:100230002EF0F4FC7B1E0B9A162B00F22A81DFE8CD
:1002400013F022023802090261024E027502DC013B
:10025000C701B00199018201280161026D01750297
:10026000DC01C701570141012B011601FE00E80026
:100270002A68DAF81C301344CAF81830FFF7BAB904
:1002800027F05CFD032240F6B8338AF82020CAF834
:100290001C30FFF711B900BF54260020E45700209E
:1002A000583E00206846002067666666644300206A
:1002B00086C70020E9C800208490002060BA002092
:1002C0005C46002046460020D83F00201040002019
:1002D0004C5800203C560020D34D621054B80020EA
:1002E0001C4000200A2027F0A3FD2688074600288E
:1002F00000F09582F10640F18983CA4D95F8187295
:10030000002F7EF4EBAE0D202EF062FB012385F86A
:1003100018322688002F7FF406AAFEF7DFBE9BF86E
:1003200010320122B24023EA020309F5FA728BF877
:100330001032AA60FFF77DBA0124FEF7D2BC00217B
:10034000B94807F0A3FC00287FF48AAA322385F875
:10035000DC01A5F82831FFF783BA07F059F9ABE4BF
:10036000002A0CBF0120022061E7B04B00220120CF
:10037000AF49B04C0B60B04B227006932EF04EFC90
:10038000089BAE4C1B68FEF7DEBDAD4AAD49A94BDC
:10039000116002225A70A84B069327F0ADFD089B0E
:1003A0001B68FEF7D0BDA64AA7491160A14B0022E9
:1003B000F0E7A34AA54911609E4B0122EAE7792A9A
:1003C00000F0EB837A2A00F0E2839E2A00F0D883C3
:1003D0009D2A00F0CE83AE2A00F0C483AD2A00F03F
:1003E000BA83EF2A00F0B483FD2A00F09F83FB2A32
:1003F00000F01484FE2A00F00E84F72A00F0DE8359
:100400007B2A00F0D083089B8B4A1B680692FEF77C
:100410009ABDDBF81402DFF8388290F8361098F8AD
:10042000023011446429A8BF642121EAE17180F8F7
:100430003610002B40F0FB8326F00EFE9EE4DBF826
:100440001402DFF80C8290F8371098F8023011444B
:10045000FE29A8BFFE2121EAE17180F83710002BA8
:10046000EAD0162027F02EFDDBF81402E4E70A9804
:10047000DFF8DC8141781144B1F5967FA8BF4FF4D5
:10048000967121EAE171417098F80230002B40F03A
:10049000C883DBF81402CFE7DBF81402DFF8B08181
:1004A00081781144C829A8BFC82121EAE17181706F
:1004B00098F80230002BBFD0142027F003FDDBF8A2
:1004C0001402B9E7DBF81402DFF8848141781144A3
:1004D000C829A8BFC82121EAE171417098F802300B
:1004E000002BA9D0132027F0EDFCDBF81402A3E7C2
:1004F000DBF81402DFF8588101781144C829A8BF3D
:10050000C82121EAE171017098F80230002B93D0E4
:10051000122027F0D7FCDBF814028DE7DFF83081DA
:100520000A9898F80230417911446429A8BF6421DF
:1005300021EAE1714171002BABD00E2027F0C2FC03
:10054000DBF8140278E7DBF81402DFF80481017AA3
:1005500098F802301144C829A8BFC82121EAE171E6
:100560000172002B3FF468AF0B2027F0ABFCDBF8E7
:10057000140261E7DBF81402DFF8D480C17998F83F
:1005800002301144C829A8BFC82121EAE171C17114
:10059000002B3FF451AF0A2027F094FCDBF8140243
:1005A0004AE7DBF81402DFF8A880817998F8023076
:1005B0001144C829A8BFC82121EAE1718171002B2B
:1005C0003FF43AAF092027F07DFCDBF8140233E753
:1005D000DBF81402DFF87880417998F80230114492
:1005E000C829A8BFC82121EAE1714171002B40F060
:1005F0002283112F7FF454AF1EE7DBF81402DFF8DB
:100600005080017998F802301144C829A8BFC82148
:1006100021EAE1710171002B40F0E382102F7FF499
:1006200055AF09E7D41F0020E457002074AF002025
:10063000BC460020D0C600205C4600204646002074
:10064000C0460020F4C60020DCC60020E8C600201A
:1006500094B000200A99DFF8D0840F791744642FF2
:10066000A8BF642727EAE7770F7127F045FC98F8C1
:100670000230002B3FF40DAF0320394627F022FC57
:10068000DBF81402D8E60A98DFF89C84017811445C
:10069000FA29A8BFFA2121EAE171017098F8023025
:1006A000002B3FF4F6AE012027F00CFCDBF814021F
:1006B000C2E60A98DFF87084817811446429A8BFE3
:1006C000642121EAE171817098F80230002B3FF437
:1006D000E0AE022027F0F6FBDBF81402ACE60A9845
:1006E000DFF84484C17998F80230114481F308019D
:1006F000C171002B3FF4CDAE052027F0E3FBDBF802
:10070000140299E60A9BDFF82084997998F8020090
:1007100011446429A8BF642121EAE171997100287C
:1007200040F091820D2F7FF4FBAEB2E6DBF81402AD
:10073000DFF8F483C17898F802301144C829A8BFC3
:10074000C82121EAE171C170002B40F042820F2FD5
:100750007FF4D2AE70E6129BFFF7CDBB049931F95E
:1007600012209978B2F5617F4FF4966393FBF1F311
:100770006CDB40F633019142A8BF11460C2FA1F566
:10078000617191FBF3F100F05E81182F7FF4F6AAFE
:10079000C9B2C8290B46A8BFC823DBF81402C27D22
:1007A000DFB297423FF4EAAA9A1ADFF87C83C77552
:1007B00048BF0732D71098F802300137FFB23BB973
:1007C000002F3FF4DBAA38462EF028FAFFF7D6BAFE
:1007D000182027F077FBF3E7BE4BBF491A684FF4A8
:1007E0007A73B3FBF2F3C3EB431203EB8202089B71
:1007F0001B68D2001F06A1F8A82000F1A580B74A07
:100800000692126855077EF59DABB54AB54C0A2194
:100810001180FEF798BBB0EE670AFFF762BAF206E6
:1008200000F1E6800B2027F003FB002840F0AA80AF
:10083000B30600F10181AC4D95F81832002B3FF45E
:1008400062AD002F7EF46FAFFEF748BC0C2F40F076
:10085000D78000273946A54B0B915B78BB423FF40C
:100860008DAADFF8C482384615F0E4F898F8023013
:100870000B991BB1C9B20C2027F024FB0137FFB242
:100880009EE79B49089B0A60944A1B680692954C18
:10089000FEF759BB974A0792FFF726B8964A089B7E
:1008A0001E68136823F004031360012306F48056C6
:1008B0008AF82130FFF7E7B8904B0122022057E574
:1008C00006F48056FFF7DFB80023BB2A149300F02C
:1008D000E580B72A00F0DE80BE2A00F0D980BD2A6C
:1008E0007FF46DAD4FF6FE71854A7C48D68906903F
:1008F0009089334401449181D3812CF0D3FF06F0D9
:10090000C7F92CF0B7FFFBF7D1FE01202EF086F9D6
:10091000B5F8D821089BFA3A00211B68A5F8D82120
:1009200085F8DA11FEF70FBB7649089B0A786B4809
:100930001B68069042F004020A706A4CFEF703BB83
:10094000714B0222032013E56E4A127896077FF559
:1009500056AF6E4A127D042A7FF651AF16F0ACF9FD
:10096000089B1B684BE72CF09DFF06F091F92CF0DB
:1009700081FFFBF79BFE01202EF050F995F8D62160
:10098000FFF783BA624A634B528993ED007A07EE10
:10099000902AF8EEE77AB0EEC77AB4EEE77AF1EE95
:1009A00010FA7FF545AF93ED017AB0EEC77AF4EE19
:1009B000C77AF1EE10FA7FF73BAFB3063FF53BAFD6
:1009C00020200DF077FE95E80C0053490A60084698
:1009D00041F8043F2AF002FE504B01221A70424DAA
:1009E00095F81832002B00F004812688FEF79BBE94
:1009F00010200DF047FE494B26881F70012711E794
:100A0000182F7FF4BBA900210B46C6E610200DF07D
:100A100051FE20200DF036FE4149081F2AF0DEFD70
:100A20003E4B02221A70DAE703263346FFF70ABA72
:100A300002263346FFF706BA20200DF023FE374B7F
:100A400000221A70CBE7CFB205E708263346FFF73E
:100A5000F9B92249334A089B06914FF4C8711B68C3
:100A60001180204CFEF76FBA01263346FFF7EAB932
:100A700007263346FFF7E6B906263346FFF7E2B905
:100A800005263346FFF7DEB904263346FFF7DAB909
:100A9000022129E719464FF6FE7325E7194602237E
:100AA00022E7002C3EF461A90F4D95F8D531002BBB
:100AB0003EF48CA92DF070FF002385F8D531FEF7A8
:100AC00085B9064B85F8451185F846010693054C16
:100AD000FEF7B7BEA4AC0020B4A400205C46002002
:100AE0007ACC002046460020D41F0020D0C600202B
:100AF000D83F002010980020B4460020C2AF00204C
:100B00002C580020B846002010B000205061002072
:100B1000E842002054BC0020BC24002058420020A1
:100B2000504200207CCC002094B000200021012005
:100B300014F0B4FEB5F8D821089B46491B6806910D
:100B4000963AA5F8D821002285F8DA21FEF7FBB9FC
:100B500000210846ECE7FF21002021F064FB95F816
:100B6000D6213EE40121002021F05DFB95F8D6213D
:100B700034E40021FF2021F056FB95F8D6212AE429
:100B80000021012021F04FFB95F8D62120E4324AC4
:100B9000137A43F00103137235E42F4A137A23F0DA
:100BA000010313722FE44FF4FA61022014F076FE71
:100BB000284B0693089B1B68FEF7C5B9002104204B
:100BC000B6E7264D13F0F6FC002385F8D531FEF785
:100BD000FDB80F200B9227F075F9DBF814020B9A81
:100BE000B5E510200B9227F06DF9DBF814020B9A93
:100BF00014E50127FFF787BB002B3FF455AF1849D9
:100C0000184A09684FF47A7000FB031313604BE72E
:100C10000B20FEF759B90021032089E700210220AB
:100C200086E7152027F04EF9DBF8140204E41720BC
:100C300027F048F92DE411200B9227F043F9DBF857
:100C400014020B9AD5E40D200B9227F03BF90B9A76
:100C500068E500BF5C46002070430020D41F0020E0
:100C600060BA0020D43F00202DE9F0478C4B1B7860
:100C7000DB07074644D58B4B8B4D1C788B4E012CE4
:100C800059D01CD3022C07D189498A4A0988128875
:100C9000914201D901241C70EB7AE3B12B89D3B1C5
:100CA000854B1B78BBB10EF0E3F8002800F09B8069
:100CB0002B7B83422CBF0121002131700CE07C4949
:100CC0007E4A098810886A7B801A8842E2DAEB7AC9
:100CD0000024002BE2D131782A79632A06D8022C2D
:100CE000774E00F0BA803378002B5DD1754AAB7A2D
:100CF0008C4238BF0C461470002B4CD1BDE8F087F5
:100D00006B4B694D19885B88E878CB1A83EAE372EC
:100D10008142A2EBE3721DD32B788B421AD3614B35
:100D20001C78E01E012861D96749097802294FD053
:100D3000012C5E4EA5D15F4A5D491288687B098807
:100D4000121A914239DD5D4A12888A42A4D20024E7
:100D50001C70A1E7B1EB400FE1DC524B1C78E11EA7
:100D6000012940F29480022ADEDC57494F4E087870
:100D7000DFF84481DFF844C1DFF838E100210324C3
:100D8000022834701C7088F80010ACF80010AEF81F
:100D9000001081D11FE0012C71D0022C0BD1072053
:100DA000BDE8F0472DF014BE7068381A474B9842E2
:100DB00058DD72709AE7BDE8F08702241C706BE77B
:100DC000022AD2DD4049097802294FF0040464D197
:100DD0003949364E09783E48022ACCBF002201220A
:100DE000C28081804BE70221317075E7022A9BDCCB
:100DF00095F800C091FBFCFC0CF1010CBCF1080F54
:100E0000DFF8B4A0304EA87895F801E096F800809D
:100E10002A4CDFF8A090254EA8BF4FF0080C8AF8A6
:100E200000C01FFA8CFA10FB0AF01EFB0AFE80B20B
:100E3000DFF88CA02080A9F800E000244FF0640EB9
:100E4000B8F1020F34701C70CAF804408AF801E04F
:100E50007FF439AF0FFA8CF1BDE73078A0B90123E8
:100E600077603370C2F164021A4B00FB02F083FB1F
:100E70000023C017A0EBA3506430707036E7082041
:100E8000BDE8F0472DF0A4BD7368F81A8EE7032C77
:100E900096D10D49097802299AD0044EFCE600BF8C
:100EA0000C910020E82700204C460020EE2700206F
:100EB0003CBC0020EC27002052BC0020EA27002088
:100EC000942600201940002038BB00207F9698000F
:100ED0003CBB00206BCA5F6B2DE9F04F2DED028B00
:100EE00095B0064619F054FA9E4B1D7825B115B001
:100EF000BDEC028BBDE8F08F9B4B1B685805F6D507
:100F0000DFF8B092D9F80020002A00F02781974C32
:100F1000D4F8283103F5F43348339E42C0F01E81E3
:100F2000934F94F82C113B68C4F82861013184F880
:100F30002C11990701F1798713F0140F41F01787ED
:100F400013F0080F94F82C3140F0C28113F0070819
:100F500001F0BA85282B874B029302F0B1805E2006
:100F60009047854B1B78002B6BD0804C834AD4F87C
:100F70003431F31A934201F24384DFF83CA29AF829
:100F80000080B8F1000F33D1DFF80092D9F80000EB
:100F900004F0DEFEC0B201280ED90228784F42F0DC
:100FA0004F813B78002B42F02A82D4F83C31F31A6F
:100FB000B3F57A6F82F0D58272480768002F40D06F
:100FC0009AF80030BBB9704BD9F800001B689B78C9
:100FD0001E3B012B4FF0020142F26882043019F0EF
:100FE0008FF8012200238AF8002084F8483126E097
:100FF000644807682FB3D4F8443140F6B732F31A87
:1010000093421ED994F84031002B02F00F81013B2E
:10101000DBB284F84031002B01F0978717F8011BF1
:1010200094F84821076094F8493158480A4401333C
:10103000006884F8482184F8493104F08DFEC4F832
:101040004461534A029B12781B68012A03F1010391
:101050000C9301F0FF824F4B1B787BB1DFF85C9162
:10106000D9F8003053B1414C029BD4F85C21D3F83D
:1010700000B0ABEB0202632A01F21A82DFF8408172
:1010800098F800A0BAF1020F01F03A873C4F97F8A8
:101090007430032B01F0DC843F4B1B7873B13F4D60
:1010A0002B685BB1314CFCF7B3FAD4F8683103908C
:1010B00044F61F62C31A934200F26081384B1B78DA
:1010C000002B7FD1374B1B7843B1284CD4F8B83272
:1010D00003F50043E8339E4281F03283324B1B78A4
:1010E000002B3FF404AF214E304C314D06F2C127A6
:1010F000206804F02DFE00283FF4F9AE206804F0CB
:101100001FFE2B7880465A1E33B120682A7004F0E7
:101110001FFE0028F2D1EAE603223946781E33F09A
:101120000AFD96F8C03296F8C12286F8C38283F48D
:101130007F4383F0FF039B1A1FFA88F89BB2B8EB3A
:10114000132FD5D196F8C222DBB29A42D0D1781EA5
:1011500029F002FB2B7818442870C9E7054B02934D
:10116000FFE600BFB5C60020B4AC0020F02100208F
:101170005C46002060BA00206E4700203F0D03004F
:1011800024000020D4460020D0460020CC46002079
:101190006F4700207C4700208447002088470020BC
:1011A000F4470020054800208E4700209447002087
:1011B00098470020DC460020D846002010BE0020C2
:1011C000B2C80020604C2278002A41F03A82DFF851
:1011D000A49199F80040002C40F0AB805B4D28783A
:1011E000002842F08C805A4C5A4DD4F8B02229780D
:1011F000594B93FBF1F313449E42FFF463AF94F811
:10120000B432564AC4F8B062D75CFB0702F174826C
:10121000B80702F1E981790702F12A823A074CD531
:101220004F4BDFF854810D930DF15009A3F13D02AE
:1012300049F8202D0021A3F1400203F8401C0223AD
:101240001121517093704846D8F8001005F0FAFF4C
:101250004846D8F8041005F0F5FFB8F80E304149BB
:1012600003EBC3039B00053381FB0321DB17C3EBB7
:10127000A10189B2484605F0FDFFB8F8103003EB34
:101280008303590089B2484605F0F4FF364B1B78BA
:101290009B0743BFB8F8081001F57A7189B24FF483
:1012A0007A71484605F0E6FF0C9B98F81420591C0B
:1012B0000C9148461A7019F011F894F8B432297854
:1012C000013393FBF1F201FB123384F8B432F9E6F7
:1012D00013F0030A7FF43AAE5E209047D9F800304D
:1012E00014209847214B1F4AB3F9043082FB0312A4
:1012F0004FEAE378C8EBA2080FFA88F85FFA88F0A3
:1013000018F052FFC8F3072018F04EFFD9F800304C
:101310005E209847D9F800301C209847504618F0B6
:1013200043FF504618F040FF94F82C31D9F80020C4
:101330000CE60F4D2F6E002F41F09D86044B89F86F
:101340000070C3F8B062BDE660470020FC47002093
:10135000F021002004480020A08601000048002061
:101360002047002067666666B84600206846002071
:101370000C480020FD4700205061002094F86E3199
:10138000002B41F0EA85DF4B1B6803F00802002ABE
:1013900048F603414AF60B404BF60F4249F6074721
:1013A00004BF02460F4613F0040F4FF0190118BF97
:1013B00017469B0684F86E1103D547F4804747F023
:1013C00020070DF047FDC7F30909002842F0D2823B
:1013D000CD4B9B79002B42F09F82984664204FF0C2
:1013E000FF3A4FF0000C0C970D97ADF83CC0CDF8CC
:1013F00042C0CDF846C0CDF84AC0CDF83890ADF81F
:101400003E80ADF840A08DF84E000CAF0FCFDFF856
:1014100008E384F805C0AEE80F0097E80F00AEE8D7
:1014200007002EF8023B71464FF0010C1B0CFE2703
:101430001F20C82201F81E39A770A27184F807C0C6
:10144000E07094F87E01207180F0F10383EA0313C9
:10145000DAB2130983F0E70343EA022383EAC20303
:101460001BB283EA0312D2B2C3F3072383EA121337
:1014700043EA022383EAC2031BB283F0C80282EA72
:101480000212D2B2C3F3072383EA121343EA022300
:1014900083EAC2031BB283EA0C0787EA0717FFB28D
:1014A000C3F3072282EA171242EA072200EB0C0379
:1014B00082EAC7070EEB0C0084F87E31278011F812
:1014C000013B7B4083EA0313DBB21A0982EA17224D
:1014D00042EA032282EAC3031BB29FB28142278001
:1014E000EDD183F07C0383EA0313DBB24FEA131ED2
:1014F0008EEA172E8EEA032E8EEAC30E0FFA8EFEA8
:101500001FFA8EF9DFF814C2A4F800905FFA8EFE7D
:101510004FEA192984F8289084F827E00CF5D3784D
:1015200004F1220ADCF80000DCF80410DCF80820E2
:10153000DCF80C3047460FC70CF1100CD445B84608
:10154000F0D1DCF800003860704F9CF8043088F867
:10155000043007F1270884F8CDE184F8CE9117F81C
:10156000011F286804F0F8FBB845F8D194F86F2102
:10157000002A41F05E856649029B08781B680A21B3
:1015800084F86F11002801F09A86DFF894E10128B1
:10159000BEF80010059142F2EE820228BEF80280E9
:1015A00002F00082BEF804100491032802F0DD82EC
:1015B0000428BEF806A002F0D3820528BEF8087001
:1015C00002F0C7820628BEF80AC002F0BF820728D0
:1015D000BEF80C1001D0BEF80E2094F87EB10C932A
:1015E0008BF0300383EA0313DBB24FEA131E494842
:1015F00084F804B08EF07A0E4EEA032E00888EEA4C
:10160000C303DFF820E1C0EB00208EFB009E864480
:10161000C0171BB2C0EB6E200690C3F3072E83EAFF
:101620000310059BC0B24FF0000963F30F098EEA67
:10163000101305934FF0000E049B68F31F4967F3E6
:101640000F0E4FF00008002763F30F0861F30F0738
:10165000059BCDF834906CF31F4E62F31F474FF09B
:10166000000C9DF81820CDF83CE06AF31F48CDF837
:10167000388010978DF844C08DF8452043EA002348
:101680000DF1300883EAC007B8E80F003FB287F0D9
:10169000C80989EA0919DFF880E084F805C05FFA13
:1016A00089F9C7F30727AEE80F0087EA191747EA59
:1016B000092398E8030083EAC9031BB283F02307D8
:1016C0004EF8040B87EA0717FFB2C3F3072282EA3A
:1016D0001712704642EA072282EAC70720F8141957
:1016E0000BF1010B4FF0230CFE211622C82384F8C6
:1016F0007EB1278084F807C00EF1020EA170E2705F
:10170000A37111E05C4600204C4600209723002086
:1017100018C7002044460020F8210020F2210020B4
:10172000849000200308208010F8013B7B4083EA6E
:101730000313DBB21A0982EA172242EA032282EA81
:10174000C3031BB29FB270452780EDD183F0F40331
:1017500083EA0313DBB24FEA131E8EEA172E8EEADA
:10176000032E8EEAC30E0FFA8EFE1FFA8EFCD64FA2
:10177000A4F800C04FEA1C295FFA8EFE84F81EE030
:1017800084F81F907968BA683868FB6807F5D37CDD
:10179000ACE80F0038697969BA6904F2C518ACE899
:1017A000070004F2A71784F8C59184F8C4E117F87C
:1017B000011F286804F0D0FAB845F8D194F87231C6
:1017C000002B41F04684C14F3B681922980684F8EB
:1017D000722140F10E83BE4BDFF800831B7899071E
:1017E00041F1868798F81430042B8CBF4FF0030921
:1017F0004FF00209FBF70CFFB8F81030B8F80820DA
:101800000C9003EB83035B00ADF84A304FF47A7021
:10181000D8F800308DF84C900E93B8F80E1098F868
:1018200014E0D8F804308DF84DE000FB02F24FF0E0
:10183000000A4FF0FF300DF13009CDF834A01092BE
:101840000F93ADF848101190CC46BCE80F00DFF8BC
:1018500090E2AEE80F009CE80F00AEE80700724689
:10186000182122F81C39E17194F87E1184F805A042
:1018700081F0780383EA0313D8B2030983F0F603F7
:1018800043EA002383EAC0031BB283EA0310C0B219
:10189000C3F3072383EA101343EA002383EAC00358
:1018A0001BB283F0C80080EA001C5FFA8CFCC3F313
:1018B000072080EA1C1040EA0C2080EACC0000B22D
:1018C00080F0180383EA0313DBB2C0F3072080EA39
:1018D000131040EA032080EAC30301F1010CFE204B
:1018E0004FF01E0A4FF0C80BA0700EF1020E2171CE
:1018F00084F87EC1238084F803A084F806B01846DB
:1019000012F8011B414081EA0111C9B20B0983EAB7
:10191000102343EA012383EAC10109B288B2724568
:101920002080EDD181F0180181EA0111C9B20A09C4
:1019300082EA102383EA012383EAC1031BB29AB22D
:1019400061492280DBB2120A04910692059384F861
:10195000272084F826308E4601F5D37B04F1220A35
:10196000DEF80000DEF80410DEF80820DEF80C30A7
:10197000DC46ACE80F000EF1100ED645E346EFD181
:10198000DEF80000CCF800009DF81430DFF854A118
:1019900084F8CC319DF8183084F8CD31D3461BF84B
:1019A000011F286804F0D8F94A4B5B45F7D1FBF7D3
:1019B0002FFED8F800103B68B8F808200591D8F839
:1019C0000410069113F0140F4FF47A7101FB02F129
:1019D00041F074850F4694F87EB10C908BF06A004C
:1019E0003D4BDFF804E1B3F90420109780EA0010C2
:1019F000C0B2030983F0D50343EA002383EAC0039E
:101A00001BB283EA0310C0B2C3F3072383EA1013A7
:101A100043EA002383EAC0031BB28EFB020E059843
:101A20000D90D2174FF00008C2EBAE0206980E9050
:101A300083F0C80C0F91ADF84A20ADF84480ADF8A2
:101A40004680ADF848808CEA0C1CCE465FFA8CFCD0
:101A5000C3F30727BEE80F0087EA1C1747EA0C27E5
:101A600087EACC07DFF878C084F804B03FB2ACE86E
:101A70000F0087F021039EE8070083EA0313DBB21F
:101A8000C7F3072787EA13170BF1010E47EA03276D
:101A90008CE8070087EAC30384F87EE14FF0210B4E
:101AA0004FF0FE0E1C27C8220CF10C0C84F80580A8
:101AB00084F807B084F802E0ACF11C01E770184626
:101AC000A271238012E000BFF22100205C460020BA
:101AD000B8460020BD230020684600205061002049
:101AE000F8210020972300206766666611F8012B15
:101AF000424082EA0212D2B2130983EA102343EA77
:101B0000022383EAC20212B290B261452080EDD175
:101B100082F0680282EA0212D2B24FEA121B8BEA0A
:101B2000102383EA022B8BEAC20B0FFA8BFB1FFAFE
:101B30008BF3DB4F23805FFA8BFB1B0A059384F842
:101B4000253084F824B007F5D37C04F122083868E6
:101B50007968BA68FB68E646AEE80F00103747457B
:101B6000F446F4D13B88AEF800309DF81430CD4FE8
:101B700084F8CAB1D04684F8CB3118F8011F286820
:101B800004F0EAF84745F8D194F87EC1C64A84F8D3
:101B900004C08CF0EB0383EA0313D9B20B0983F082
:101BA000C50343EA012383EAC1031BB283EA03109E
:101BB000C0B2C3F3072181EA101141EA002181EA92
:101BC000C00109B20CCA81F0C80787EA0717FFB243
:101BD0004FF0000EC1F307210D93CDF838E081EAF4
:101BE00017130C9299E8070043EA072383EAC70317
:101BF0000FFA83F8AD4B84F805E088F0310783E8ED
:101C0000070087EA0717FFB2C8F3072383EA171311
:101C100043EA072383EAC703277A607AA27AE17A44
:101C200094F80CE094F811801BB25F4087EA071724
:101C3000FFB2C3F3072383EA171343EA072383EAB8
:101C4000C7031BB2584080EA0010C0B2C3F3072399
:101C500083EA101343EA002383EAC0031BB25A400D
:101C600082EA0210C0B2C3F3072282EA101242EAEB
:101C7000002282EAC00212B2514081EA0111C9B2C7
:101C8000C2F3072383EA111343EA012383EAC10362
:101C90001BB28EEA030E8EEA0E1E5FFA8EFEC3F3AF
:101CA000072383EA1E1343EA0E23677BA07BE17BB5
:101CB000227C83EACE031BB25F4087EA0717FFB29C
:101CC000C3F3072383EA171343EA072383EAC7030F
:101CD0001BB2584080EA0010C0B2C3F3072383EA66
:101CE000101343EA002383EAC0031BB2594081EA80
:101CF0000111C9B2C3F3072383EA111343EA012395
:101D000083EAC1031BB25A4082EA0212D2B2C3F381
:101D1000072383EA121343EA022383EAC2031BB2B6
:101D200088EA030888EA08185FFA88F8C3F30723EB
:101D300083EA181343EA082383EAC803A17CE27C00
:101D4000DFF874811BB2594081EA0111C9B2C3F3B3
:101D5000072383EA111343EA012383EAC1031BB279
:101D60005A4082EA0212D2B2C3F3072383EA121363
:101D700043EA022383EAC2031BB283F0270787EA00
:101D80000712D2B2C3F3072787EA121747EA0227DE
:101D900087EAC2073FB20CF10103BAB25FFA87F9D2
:101DA0004FF0310CFE200C2184F87E31C8234FEA1D
:101DB000122E228084F807C0A070E170A37184F80D
:101DC0001490049F84F815E07968BA68FB68386855
:101DD000B7F810C0A8E80F0028F803CB84F8BBE1DF
:101DE00084F8BA911AF8011F286803F0B5FFD045AE
:101DF000F8D194F87671002F41F026812C4B94F89D
:101E00007E81B3F90010B3F90220B3F904309FEDDD
:101E1000296A677107EE103A029B1B680C9388F0E1
:101E20006A0383EA031306EE901AD9B20B0983F012
:101E3000D50343EA012383EAC1031BB283EA0311FA
:101E40005242C9B207EE902AC3F3072383EA111363
:101E500043EA0123F8EEE77AF8EEE66AB8EEC77ACD
:101E600083EAC1031BB267EE867A66EE866A27EEC6
:101E7000067A002083F0C80ECDED0E7ACDED0D6A06
:101E80008DED0F7A1090119012908EEA0E1C0DF1CC
:101E900030095FFA8CFCC3F3072EB9E80F000DE0A0
:101EA000F2210020BB2300204C420020F82100201A
:101EB0006846002088C3E43A982300208EEA1C1E5E
:101EC0004EEA0C2E8EEACC0EDFF888C40FFA8EFE96
:101ED000ACE80F008EF01E0799E8070087EA071AA2
:101EE0005FFA8AFACEF3072787EA1A1747EA0A2722
:101EF0008CE8070087EACA071C214FF0050A4FF05B
:101F00001E094FF0FE0EC82208F10103E17084F8AB
:101F100076A184F8079084F802E0ACF11001A27178
:101F20000CF10C0C84F80480278084F87E3111F8C1
:101F3000013B7B4083EA0313DBB21A0982EA1722D2
:101F400042EA032282EAC3031BB29FB261452780A3
:101F5000EDD183F0270383EA0313DBB21A0982EA87
:101F6000172282EA032282EAC3031BB21FFA83FC10
:101F7000DFF8E483A4F800C05FFA83FE4FEA1C2C6C
:101F800084F825C084F824E008F5D37904F1220A06
:101F9000D8F80000D8F80410D8F80820D8F80C3089
:101FA0004F460FC708F11008D045B946F0D1E04FB1
:101FB000B8F80030A9F8003007F1240884F8CAE125
:101FC00084F8CBC117F8011F286803F0C5FEB84597
:101FD000F8D194F877A1BAF1000F41F02F80D54BDA
:101FE0001B68052284F877219A0641F17281D24A52
:101FF000DFEDD27AD18907EE101AB8EEC77A13F066
:10200000140F27EE277A01F0F984CD4BDFEDCB6A70
:10201000D3ED007AF8EEE77A67EEA67A94F87EC1FF
:10202000C84BC94AB3F90410B2F90620C74FC848D3
:102030008DED0D7A8CF0220383EA03135FFA83FEA1
:102040004FEA1E1383F0590343EA0E23B2F5FA6FE9
:1020500083EACE031BB2A8BF4FF4FA6283EA0318E7
:10206000B2F57A7F5FFA88F8C3F3072EB8BF4FF452
:102070007A72A2F57A728EEA181E642303FB02F3C9
:102080004EEA082E87FB03278EEAC80EDA17C2EB4A
:10209000A71280FB01300FFA8EF7CB174FF0000B21
:1020A000C3EBA00387F0C8080DF13009CDED0E7A1F
:1020B000ADF84220ADF84030CDF830B0CDF83CB0AE
:1020C000CE4688EA0818BEE80F005FFA88F8C7F322
:1020D000072787EA181747EA082787EAC8089D4FA5
:1020E000DEF800E084F804C00FC70FFA88F888F023
:1020F0004A0383EA0310C0B2C8F3072383EA10132C
:102100003A460CF1010143EA002383EAC00342F896
:1021100010E900204FF04A084FF0FE0C4FF0140E6B
:1021200084F87E11C82160712380043784F8078009
:1021300084F802C084F803E0A171184612F8011B6C
:10214000414081EA0111C9B20B0983EA102343EA35
:10215000012383EAC10109B288B2BA422080EDD1DD
:1021600081F0140181EA0111C9B24FEA111E8EEA11
:10217000102E8EEA012E8EEAC10E774B0FFA8EFEDC
:102180001FFA8EFC1F464FEA1C2B5FFA8EFE84F866
:102190001DB084F81CE0596838689A68DB68A4F8B8
:1021A00000C007F5D37CACE80F0038697969B7F84F
:1021B00018800497ACE8030004F2A717ACF800807D
:1021C00084F8C3B1B84684F8C2E104F2C31B18F81E
:1021D000011F286803F0C0FDC345F8D15F4B604A7A
:1021E0001B781278013B12F00100DBB214BFC02152
:1021F0004021172B03D85B4A134493F814A05A4B81
:102200001A8893071ABF002341F01001012312F42A
:10221000027F18BF022312F0100F18BF062312F01E
:10222000200F18BF1023002841F091814FF00308C0
:1022300094F87EC10C938CF0460383EA0313DAB260
:10224000130983F0920343EA022383EAC2031BB219
:1022500083EA0310C0B2C3F3072282EA101242EAF3
:10226000002282EAC00212B282F0C80E8EEA0E1E6E
:1022700000235FFA8EFE0320C2F307228DF834A0FC
:102280008DF8378082EA1E128DF835308DF83610C1
:102290008DF8380042EA0E2899E8070088EACE0E49
:1022A0000FFA8EF8DFF8ACA0E37188EA0819AAE803
:1022B00003005FFA89F9C8F3072888EA191848EA81
:1022C000092181EAC90994F808808AF800200FFAE8
:1022D00089F988EA090282EA02185FFA88F8C9F3E4
:1022E000072282EA181242EA0822607AA17A94F858
:1022F0000B90637182EAC80212B2504080EA00106B
:10230000C0B2C2F3072282EA101242EA002282EA35
:10231000C00212B2514081EA0111C9B2C2F30722D0
:1023200082EA111242EA012282EAC1021EE000BFE3
:10233000972300205C460020506100200AD7233CF0
:10234000604600206846002084900020D34D621033
:1023500067666666F8210020F2210020405C0020BC
:102360000C910020044D04084646002012B289EA70
:10237000020989EA09195FFA89F9C2F3072282EA98
:10238000191242EA092294F80C80607BA17B84F840
:1023900004C082EAC90212B288EA020888EA081870
:1023A0005FFA88F8C2F3072282EA181242EA08228A
:1023B00082EAC80212B2504080EA0010C0B2C2F3F2
:1023C000072282EA101242EA002282EAC00212B216
:1023D000514081EA0111C9B2C2F3072282EA111207
:1023E00042EA012282EAC102E17B94F8109013B222
:1023F00081EA030282EA0212D2B2C3F3072383EA1C
:10240000121343EA022383EAC2031BB289EA0302DE
:1024100082EA0212D2B2C3F3072383EA121343EA19
:10242000022383EAC2031BB283F0320282EA021261
:10243000D2B2C3F3072383EA121343EA022383EAE7
:10244000C2031BB29AB24FF0FE085FFA83FE092066
:10245000C8210CF1010C84F802804FEA1228E070C8
:10246000A17184F87EC1228084F8128084F811E082
:10247000049B186859689A68B3F80CB00AF5CC7CCC
:10248000ACE807000AF5D47A8CF80290ACF800B0FA
:1024900084F8B88184F8B7E117F8011F286803F0C1
:1024A0005BFCBA45F8D1039BC4F86831FEF706BE61
:1024B000DFF83C83BF4FDFF83CA3412028F0CCFB82
:1024C000B8F9022087FB0230D217C2EBA00080B21D
:1024D00028F0A6FBB8F9002087FB0230D217C2EB28
:1024E000A00080B228F09CFBB8F9042087FB0230E2
:1024F000D217C2EBA00080B228F092FB9AF800102D
:10250000D9F8000003F028FC94F8608118F0010766
:1025100000F02885A84F3A68910640F18180A74ACB
:10252000DFF8D4821278920740F1C48798F814201B
:10253000042A8CBF032302230393472028F08CFB3B
:10254000D8F8000028F038FBD8F8040028F034FB55
:10255000B8F80E209A49D9F80000A1FB0232C2F364
:1025600047121146049203F0F7FB9AF8000039680D
:10257000049A11F0140F82EA00028AF8002040F059
:10258000BA86B8F80820642000FB02F028F014FB9B
:1025900098F81470039BD9F8000043EA8707FFB24C
:1025A000394603F0D9FB9AF80020D9F800005740CB
:1025B00039468AF8007003F0CFFB94F86081B8F1D7
:1025C000000F2DD17F4F4F2028F046FB386828F0B0
:1025D000F3FA786828F0F0FA404628F0EDFA012185
:1025E000D9F8000003F0B8FB744A9AF8007012782A
:1025F000D9F8000002F00108414687F001078AF887
:10260000007003F0A9FB9AF80020D9F8000088EACE
:10261000020211468AF8002003F09EFB94F86081C4
:10262000694AC4F85CB108F10103DBB2A2FB0312F2
:10263000D20802EB8202A3EB420384F86031FEF77A
:102640001DBD624B6249186803F04EFB00232370E6
:10265000FEF7BDBD5F4F386800283EF4FCAC4FF07C
:10266000000ADFF898815C4CAB46554603F070FBDE
:10267000F8B1F5B94FF00109AA46386803F060FBDC
:1026800083B27E2B00F0518498F80120002A49D1B2
:1026900094F84C11B1B11B2B84F84C2100F01E842E
:1026A0000D2B45D0386888F8019003F051FB0028C5
:1026B000E3D1AA4650460CAA48495D4617F0DCF91A
:1026C000FEF7C9BC7D2B00F0F08594F8502122B1B3
:1026D00080F02003DBB284F8501194F84B21062AD5
:1026E00010D8B4F84E1138681944A4F84E11A11846
:1026F000013281F8543184F84B2103F029FB002882
:10270000BBD1D6E7B4F84E2188F8019013449BB2B0
:102710001A0A52FA83F3FF2BA4F84E31386802D11B
:102720002F4DA3E7386803F013FB0028A5D1C0E7BD
:102730003868A4F84E2103F00BFB00289DD1B8E7C0
:1027400094F8BC32C4F8B862012B40F2738594F857
:10275000BD222449981801EB8001013202F00102E8
:10276000CF6A84F8BD22BFB11F4D0D950DF1500900
:10277000123DA52349F8205D802284F810311523ED
:102780003146484684F8112184F81231B8470028B0
:1027900040F0D18494F8BC32144A013382FB031216
:1027A000A2EBE37202EB42029B1A84F8BC32FEF702
:1027B00095BC00BF676666665C460020B846002090
:1027C0001F85EB514C420020CDCCCCCCF8470020EB
:1027D00020470020C8460020F02100203A23002096
:1027E00044230020044D0408152300205655555558
:1027F0006846002014BE0020506100202400002004
:102800009E4A9F4B92F80BE0029AD4F83811106858
:102810001B889C4A401A4FF47A71DFB201FB0EF11B
:102820001B0A9777177588424FF00007D3775375C7
:102830009770177180F0EA84934BDFF870C21B68C1
:102840009249934F0868DFF8689289683F688CFB6B
:10285000038EDB17C3EB6E1303F5FA739BB293760B
:102860001B0AD37689FB00A389FB01A9C017C917EE
:10287000C0EBA300C1EBA90107F5EA43DFF834E29E
:1028800010773033001282F8201009121B12DFF883
:1028900028829EF800E0507782F821108CFB079088
:1028A000F917C1EB601182F823307A4B98F814A025
:1028B00083F81AA0783130371EF0020F82F8241006
:1028C00082F8227000F09F84D8F800E0724AD8F8AD
:1028D0000400DFF8E8B182FB0E714FEAEE77C7EB38
:1028E000A151039182FB0092C117C1EBA25203993F
:1028F0000BFB01E101EB410149000F460BFB020B11
:102900000497B9460BEB4B0B644F4FEA4B01059113
:1029100087FB099B87FB01194FEAA949CDF81C9059
:10292000B8F80E900399B8F8088002EB820209EB20
:10293000C90902EB8202089201EB81074FEA890282
:102940000599039207EB8707049A0697CF17C10FE3
:102950000991049852494FEAAB4BD2174FEADE7EF9
:1029600083F809E0ABEB020E01FB1E020798069903
:1029700008F5FA78BAF1050F1FFA88FAA0EB0708F4
:10298000059F474883F815A04FFA8EF909EB810996
:10299000414600FB18789DF8240098730898414F31
:1029A000DFF81CE149B201EB80018CFB020B4FEA1E
:1029B000E2720492039ABEF800E08CFB08C087FB29
:1029C00002C74FEAE27C049AC2EB6B120392364ACA
:1029D0001FFA89F91288ADF8102083F80A90039A3B
:1029E00083F813E089B24FEAE8784FEA112BC8EB7D
:1029F0006010CCEBA7174FEA1A284FEA192C4FEAC0
:102A0000222A9DF80C2083F810B04FEA202983F881
:102A10000BC0D973C7F3072C4FEA1E2134BF4FF008
:102A2000320B4FF0330B1A739DF8102083F80DA072
:102A3000587483F8129083F81680DF7183F808C009
:102A4000197583F81BB01A77C4F83461FEF795BA8C
:102A5000DFF87090D9F8000003F06AF900283EF41E
:102A60001BABD9F80000012103F05EF9022200231C
:102A700087F8742088F80030FEF70EBB44BC0020B5
:102A80003CBC00209C47002060460020844400207D
:102A900064460020C84700206BCA5F6B83DE1B437F
:102AA00040420F00D34D62109C4200201F85EB5125
:102AB00067666666B846002050610020806967FF3F
:102AC000C4460020D0C900205E209047D9F80030CD
:102AD00002209847FF2027F0C5FD0378FF2B00F068
:102AE000998490F901304FEAE3785FFA88F8D8B218
:102AF00017F05AFB404617F057FBD9F800305E201C
:102B00009847D9F8003003209847FF2027F0AAFD06
:102B10000378FF2B00F07984B0F90830D8B2C3F302
:102B2000072817F041FB404617F03EFBDA4B1B78B5
:102B3000042B7DD0DFF88CB3B4F82E119BF8002065
:102B4000DFF884A391FBF2F302FB13139BB2BAF8F4
:102B50000010A4F82E314FEA03181FFA88F86423F6
:102B600003FB01235200B3FBF2F348EA0328C3F34B
:102B700003225E20D9F800301FFA88F848EA0208DC
:102B80009847D9F80030062098475FFA88F017F088
:102B90000BFB4FEA182017F007FBC049B4F82E21B1
:102BA0004B7ABAF800A00132012BA4F82E2100F0D4
:102BB0000C874A7B0AEB8A031FFA83FA002A40F04B
:102BC000C084D9F800305E209847D9F800303A2008
:102BD0009847B34BA3FB0A384FEA58181FFA88FBF3
:102BE0005FFA8BF017F0E0FA4FEA1B2017F0DCFADF
:102BF000D9F800305E209847D9F800303B2098473C
:102C0000642303FB18A39BB2A648053380FB032073
:102C1000DB17C3EBA000C0B217F0C6FA002017F014
:102C2000C3FADFF8A88298F80630002B40F05184F0
:102C30003B689F0640F11282DFF894A29AF80030B8
:102C4000980700F1EA83DFF88C820027BB46D9F8A9
:102C500000305E209847D9F8003001209847584648
:102C600017F0A2FA384617F09FFAD9F800305E2024
:102C70009847D9F8003009209847002017F094FAB7
:102C8000002017F091FAB8F8123098F814B0B3F5A4
:102C9000967F0AD994F82C2102F00F02072A04D853
:102CA00042F20F7B9B4528BF9B46D9F800307B4FF3
:102CB0005E209847D9F80030052098473B7A002BD2
:102CC00000F06685ABF1200307EE903A9FED767A2F
:102CD000F8EEE77AF6EE006A67EE877ABEEE007AE3
:102CE000F5EEC07AF1EE10FA58BFB0EE667A77EEE4
:102CF000877AFDEEE77ACDED027ABDF908B05FFA8A
:102D00008BF017F051FACBF3072017F04DFA9AF831
:102D10000020002392070A930B9300F1658394F837
:102D20003031012B00F06083B7F90030DFED5F6ACE
:102D300007EE103AB7F9023007EE903AB8EEC77ACC
:102D4000F8EEE77A27EE267A67EEA67ABDEEC77A26
:102D5000FDEEE77A0CA88DED0C7ACDED0D7A17F02B
:102D600045FA94F82C31D9F80020FEF7F3B85E202C
:102D70009047D9F80030302098474D4BD3F8008069
:102D80005FFA88F017F010FAC8F3072017F00CFA72
:102D900094F82C3113F003087EF4C8AA454AD4F8FD
:102DA0002811454B9142186840F28F8380EAE07306
:102DB000A3EBE0733A4A1BB282FB03124FEAE37AB9
:102DC000CAEB621A4FF0640808FB1A380FFA88F849
:102DD0000FFA8AFA5FFA88FB5FFA8AF2C8F30728CB
:102DE000CAF3072AD9F8003002925E209847D9F832
:102DF000003010209847029A104617F0D5F9504637
:102E000017F0D2F9D9F800305E209847D9F8003091
:102E100021209847584617F0C7F9404617F0C4F9E3
:102E20003B68D9F80020FEF78BB8DFF8AC809FED47
:102E3000238A4FF0240A5E2090475046D9F800308C
:102E400098471F4BF8EC016A9B8A07EE103AF8EEA0
:102E5000E66AB8EEC77A0AF1010AC6EE877A5FFA27
:102E60008AFA67EE887AFDEEE77ACDED027ABDF94F
:102E700008B05FFA8BF017F097F9CBF3072017F043
:102E800093F9BAF1270F02D0D9F80020D3E73B68B5
:102E9000D9F80020FEF750B81940002044BC0020AB
:102EA0001F85EB5167666666E4380E3F0050C347E6
:102EB000644600203F4B4C006046002000007A44EE
:102EC0007046002052BC00203CBC00204C46002034
:102ED000B846002050610020A0460020386802F06B
:102EE00037FF00287FF4DEAB386884F84A9188F811
:102EF000019002F02DFF00287FF4BFABFFF7D9BB94
:102F0000FAF786FBD14B1B68A0EB030B40F6B833F6
:102F10009B4500F2BF81CE4B1A793A2A00F04284D9
:102F2000002388F80030FEF7B7B8386884F84AA163
:102F300084F84BA184F84C9188F801A002F008FFB6
:102F400000287FF49AABFFF7B4BB94F8481194F8CB
:102F50004931C0484A1CFEF76AB8013B84F86E311B
:102F6000FEF704BBBC4A1288D30513D4D00600F187
:102F7000E682910600F11D85530600F13C8510079D
:102F800000F15485D10700F1588512F0020F0CBFF3
:102F900004270C27B149B24A0B78D27803F0010319
:102FA0000AB143F002035320039327F055FEAD4AC4
:102FB000128802EB820202EB8202900080B227F0BC
:102FC0002FFE002027F02CFEA74AA8491288D9F826
:102FD0000000C2EBC212520081FB023111444FEAE1
:102FE000E278C8EB61285FFA88F8414602F0B4FE47
:102FF0009AF80020039BD9F800001F4388EA0208D2
:1030000000218AF8008002F0A7FE3946D9F80000B6
:1030100002F0A2FE9AF80020D9F800007A40D2B25D
:1030200011468AF8002002F097FE94F86081FFF7BD
:10303000C6BA013A84F86F21FEF7C0BB0AF1FF3A25
:1030400084F877A1FFF72FBA013F84F87671FEF775
:10305000C0BF013B84F87231FEF7CBBE1B077FF582
:1030600080AE834B93E803000CAB83E80300184663
:1030700017F0BCF875E60024DFF8108227464FF001
:10308000500A02E0DBB283F3118815F804B0601C2B
:103090005946284427F08EFC002840F025810BF18A
:1030A00001031C44EFF311838AF312882A6E9442C1
:1030B000E8DB0022DBB22A6683F31188FEF73EB913
:1030C0004FF0000A5E201F6884F82CA19047D9F8C1
:1030D0000030DFF8BC8117209847504617F064F89D
:1030E000644BA3FB07239B0BA8FB03125209C2EB03
:1030F0000212A3EB8203D8B217F056F8D9F80030C9
:103100005E209847D9F80030182098475A4BA3FB07
:1031100007239B09A8FB03125209C2EB0212A3EB7F
:103120008203D8B217F040F8504617F03DF8D9F8AE
:103130000020FDF714BF0C9EAE424FF000014FD9A6
:1031400041F2210015F8013B81EA03235A0013F4F0
:10315000004F80EA020192B289B208BF11464A00CC
:1031600080EA020311F4004F99B293B218BF0B46E4
:10317000590013F4004F80EA010289B292B208BFED
:103180000A46530012F4004F80EA03019BB289B251
:1031900008BF19464A0080EA020311F4004F99B2B1
:1031A00093B218BF0B465A0013F4004F80EA020195
:1031B00092B289B208BF11464B0011F4004F80EA69
:1031C00003029BB292B208BF1A46530080EA030181
:1031D00012F4004F9BB289B208BF1946B542B1D173
:1031E000484604F06DF825490C9D25486D1A152DAB
:1031F000A8BF15252A4630F0BBFB224A94F8BC3202
:103200001570FFF7C9BA2D22DA761DE41E4B02991C
:103210001B780968C4F83811013B012B3FF60CAB51
:103220001021022391701371FFF706BB16F09EFF69
:10323000FDF705BF0E4A02EB8302D76AFFF793BA88
:1032400016F084FF01233B70FDF7B6BEB8C800201E
:10325000A0C80020CC460020464600200C9100204B
:103260001C4000203CBC0020444600200308208075
:10327000044D040873B2E745D34D621000230020CB
:1032800088BF00209DBF00201940002011A3020824
:1032900089888888C44AB2F8623100210133A2F8D3
:1032A000623188F80010FDF7F7BE386884F8509155
:1032B00002F04EFD00287FF4E0A9FFF7FAB90146BD
:1032C0008446074682460490804605900246FEF7F3
:1032D00084B99FEDB67A13F0140F08BFF0EE477A69
:1032E0007EF493AEFEF79ABE41463A2027F0BEFA2E
:1032F0000743FFB2D3E6AE4A1068FFF747B9AD49BE
:10330000AD4B0093A1F13F07AC4BAD4A0B9101F8D7
:10331000404C0CA8AB490A9704F0AAF80A9F7B1C02
:103320000A933C700A9B2922591C0A911A700A9B25
:10333000EA22591C0A911A700A9BC822591C0A9148
:103340000CA81A702FF0A8FB00F101080CA9424646
:103350000A9830F00DFB0A9A02EB080301330A9336
:1033600002F808400A9B5A1C0A921C700A9B5A1CBD
:103370000A921C700A9B5A1C0A921C700A9B5A1CC7
:103380000A921C700A9B5A1C0A921C700A9B5A1CB7
:103390000A921C700A9B5A1C0A921C700A9B5A1CA7
:1033A0000A921C700A9B5A1C0A921C700A9B5A1C97
:1033B0000A921C700A9B5A1C0A921C700A9B5A1C87
:1033C0000A921C700A9B0122991814A80A911A707B
:1033D00050F8283DDB1B3B7016F080FF724B2C70C1
:1033E000C3F8B062FDF76EBE98E80C0001210AA890
:1033F00084F830110A920B9316F0F8FEB1E4C4F889
:103400003C6187F80080FDF7D7BD4FF000084046CB
:10341000FFF787BB4046FFF76BBBDFF8C081D9F8E9
:103420000030694F5E209847D9F800301120984746
:10343000B8F80E204FF4F36B0BFB02F287FB023758
:10344000D217C2EB6737F8B216F0AEFEC7F307200B
:1034500016F0AAFED9F800305E2098471920D9F856
:1034600000309847B8F80E30584A0BFB03F382FB44
:103470000301DB17C3EB611382FB0321DA17C2EBF5
:103480006112642101FB1233D8B216F08DFE0020C8
:1034900016F08AFE9AF80030B8F8087099077FF5A0
:1034A000D4AB5FFA87FB3F0AFFF7D1BB02F03CFCCD
:1034B000FDF797BD01230393FFF73FB83C4B1F680F
:1034C00007EB87077F00FEF786BAC346C24642462F
:1034D00088E4D9F80030DFF808B1DFF808A15E20F1
:1034E0009847D9F8003028209847DBF800308AFB4D
:1034F000032ADB17C3EBAA0A5FFA8AF016F054FE20
:10350000CAF3072016F050FED9F800305E20984725
:10351000D9F8003004209847B8F80830002B40F064
:103520004B82DBF8083083F310085FFA88F016F05E
:103530003BFEC8F3072016F037FEFFF779BB3427B0
:1035400028E59BF800309AFBF3FAFFF73ABB204AD4
:10355000D278002A0CBF4FF004084FF00508FEF7A0
:1035600067BE0123D9F800003B7002F0E9FB074673
:10357000D9F8000002F0E4FB7F067DF41DAD8A2837
:1035800000F043828E287DF417AD9AF80030002BAE
:103590007DF42EAD0F48104B03602D2384F840318D
:1035A0000768FDF70DBD00BFF021002000000000FE
:1035B0006046002020470020D6C60020088004086E
:1035C000108004081C80040889B5F8141F85EB518D
:1035D0001C400020D44600209C4700205061002061
:1035E0008444002067666666CF4AD04B0D920DF189
:1035F0005008A2F13D0048F8200D1988DFF85493D7
:10360000A2F1400300204FF00A0E02F8400C0822FD
:1036100083F801E040469A7003F02CFED9F80030A0
:10362000C349DA1781FB0313C2EBA30399B24046E7
:1036300003F020FE0BF01CFCD9F808900C9B4FEA1D
:103640001942591C0C911A700C9B4FEA1922591CF3
:103650000C911A700C9B5A1C0C9283F800900C9BD6
:103660005A1C0C921870404616F038FEFDF7D3BD78
:10367000AD4B0D93A3F1400900222121A3F13D0A96
:1036800003F8402C89F8021089F80120CDF830A009
:1036900024F0C0FBA74BA84A1B88A84900280ABFF2
:1036A00011464FF003084FF004085A0500F19F81BE
:1036B000D80700F1BE8103F00203A14A002B1CBF12
:1036C0004FF00308114642469E4830F051F90AEB8C
:1036D000080314A89C4A013340F8203D9B1A00229D
:1036E0000AF8082089F8013016F0F8FDFDF796BDBC
:1036F0004FF00109FEF77EB8DFF86C929FED938AD8
:10370000B9F90230884A0D9207EE903AF8EEE77A5E
:103710000DF1500867EE887AA2F14003FDEEE77ADA
:10372000A2F13D0148F8201D02F8400C0822CDED21
:10373000027A5A701E229A70BDF80810404603F0B3
:1037400099FDB9F9003007EE903AF8EEE77A404675
:1037500067EE887AFDEEE77ACDED027ABDF80810C3
:1037600003F088FDB9F9043007EE903AF8EEE77AF5
:10377000404667EE887AFDEEE77ACDED027ABDF835
:10378000081003F077FD404616F0A8FDFDF740BD98
:103790005FFA8BF016F008FD4FEA1B2016F004FDCF
:1037A000FFF7B5BA9978039318462DF0F3FB00287C
:1037B0007FF4B6AB5D49664F664A09886648674C38
:1037C000F961DFF8A891116803689268F962B4F8AA
:1037D0006211C7F86CB0FB63FA64D9F80000F965B0
:1037E000F8F7B0FB834600287DF451AC5146D9F878
:1037F000000002F099FA039B94F86421DB780493AB
:10380000642A4FF0040387F8743040F0198194F86B
:103810006531072B08BF84F865B194F86521504BDA
:10382000079207EB021A0393DAF804100691084690
:103830002FF032F9DAF8083005935FFA80FA18466B
:103840002FF02AF95FFA80FB454B079A06990AEB9D
:103850000B000830D87122F00F00987202F00F02AE
:103860000BEBCA005A739873524603F10F0030F005
:103870007FF8059B19463B4B0AF1090018445A464C
:1038800030F076F83648C37903F1010ACBB1013B39
:103890005FFA83FC0CF1080CDFF8D4E084440023C9
:1038A000073010F8012B5A409300D10883EA4203F5
:1038B00001F0180153404EFA01F253408445DBB247
:1038C000EFD1284A04980AF802302FF0FFFF94F84D
:1038D00065310022013384F8653184F86421039B4B
:1038E000DDF80CA09B785BB11AF80510D9F8000040
:1038F00002F032FA01359AF80230EDB2AB42F3D859
:1039000094F864310322013384F8643187F8742019
:1039100088F80020FFF79EB80E4B8046B3F900A050
:103920006420FDF75EBD00BF204700203CBC0020A6
:103930006766666646460020EC7F0408F47F04084C
:1039400004800408E3460020E146002058A08B4193
:10395000240000208444002060460020F021002044
:103960008C7300209273002068460020D0C900208C
:103970000007090E854B864A1B88927903EB830367
:1039800003EB83034FEA83081FFA88F8002A40F00C
:10399000FA804FF0FF330FFA83FA0BF069FA40B266
:1039A000FDF71FBD11469446174692460492FDF757
:1039B00014BE2427FFF7EEBA0BF05AFA16F0F4FB08
:1039C000002016F0F1FBFFF733B9D9F800305E2084
:1039D0009847D9F80030392098475FFA8AF016F0F6
:1039E000E3FB4FEA1A2016F0DFFBFFF71AB94FF09E
:1039F0000308684967E61027FFF7CCBA138907EE7A
:103A0000903AF8EE677AFEF709BB634B1B6898069D
:103A10007DF5D2AA9AF80030002B7DF4E9AA5F4820
:103A20005F4B03602D2384F84031B9E52027FFF771
:103A3000B1BA5C494FF0040845E60827FFF7AABA77
:103A400097F8753058481A0704BF0133DBB2072BCB
:103A500028BF01234FEA031B07EB0B025FFA8BFA27
:103A600092F810E0514A039200EB0E010022087A0E
:103A70004E498A7201F10D0207EB0B014AEA0E0E64
:103A8000012882F800E0C96802F1010C0DD9023862
:103A9000C0B200F1020E9644624602F8011B724564
:103AA0004FEA1121F9D101308444BB4421F0600276
:103AB00001339BF81110DBB20A43082B8CF800206D
:103AC0000CF1010249D04FEA031B07EB0B00384908
:103AD00090F810E034487044511A007A01EB000C61
:103AE0000AF1100ABCF1130F5FFA8AFAC4DDC9B2F9
:103AF0008A1DD2B2039842F0400E80F807E002F12E
:103B0000010ADFF8B8E0CAB105315FFA81FB0BF1B9
:103B1000080B83440EF1010C00221CF8010B5040ED
:103B2000820082EA4002C1084240224801F01801A6
:103B300040FA01F14A40E345D2B2EED104980AF8C6
:103B40000E2087F875302FF0C1FEC8E61146FDF74C
:103B500044BD11469446FDF740BD1549511AC6E7CC
:103B6000114694461746FDF738BD11469446174650
:103B70009246FDF732BD114694461746924604928E
:103B80009046FDF72ABD0C4B1B6804E73CBC0020A7
:103B90004C460020F87F04085C460020D4460020F4
:103BA000C8470020FC7F0408044D04088C730020E3
:103BB000997300200007090E8444002092730020AE
:103BC0002DE9F047B0F908500D81EDB2442D8CB0CD
:103BD0000C46164600F02C82074642D9812D00F093
:103BE0006A8200F29580542D00F0CC8040F2BD81B5
:103BF0006E2D00F0EB81802D40F0D080BB4B93F810
:103C0000009009F1020919F0FF0900F09480B84B07
:103C1000B84FB94EDFF828A3994403F101080A25EB
:103C200016E0322D00F0DB82A5F13C00C0B2132873
:103C300040F2DB8200232268511C2160157022684B
:103C4000C84502F101012160137074D018F8015BBE
:103C50000A2DE6D1BAF80030FF2BA8BFFF23DBB254
:103C6000E9E7052D00F0D2811FD8022D00F08280F7
:103C700040F26881032D00F0A081042D40F08E8079
:103C80009E4920462A4603F0D3FA0021204603F03D
:103C900017FB22680021531C0125236028462B4670
:103CA000117063810CB0BDE8F087242D60D040F224
:103CB000D480282D00F0C481382D6FD10A68904B34
:103CC0000125511C216015702268052150192060C2
:103CD000117022680A215019206011702268002199
:103CE00050192060117022681978501920601170E5
:103CF00022685978501920601170226899785319F8
:103D000023602B461170284663810CB0BDE8F08714
:103D1000A02D17D040F2BF80B82D00F0CA81FE2D33
:103D20003CD1784D05F1080635F8021B204603F01A
:103D3000C7FAB542F8D101252B46284663810CB05D
:103D4000BDE8F087704B0846196803F0A1FA6F4B85
:103D50002046196803F09CFA6D4B1968204603F061
:103D600097FA01252B46284663810CB0BDE8F08701
:103D7000684BF2E7042268492046012503F058FA0F
:103D80002B46C0E70B6800215A1C2260197022687C
:103D90000125531923602B461170B4E721462846AC
:103DA00009F0C0FB01460028C5D1742D00F0FB804E
:103DB000772D09D13B687A689A4240F0E681574AEC
:103DC00020462AF0E9FFB6E7F52D01F00783762DAE
:103DD00000F0DF817A683E68292DA2EB060300F02F
:103DE0007C8240F25982392D01F0D082532D40F06F
:103DF0008D82721C3A603078032800F22A85411EB9
:103E0000C9B2474D474A01EB410105EB4101107032
:103E1000497800288FD0013BDBB28B4240F01985F6
:103E20000021C2F80610C2F8021091725BB1581C52
:103E30003B681044013201333B6013F8011C02F867
:103E4000011F9042F7D1384B1B78002B3FF473AF22
:103E500001251FF069F92B4655E7202D9ED10B68EF
:103E6000324D591C6A7821601A7023682A78591CCF
:103E700021601A702368AA78591C21601A70298958
:103E8000204603F01DFA23686A79591C21601A70D4
:103E90002268A979FFE6822D80D10B68244A254D3E
:103EA0001178224A581C206019701189204603F0AD
:103EB00007FA214B22681B88FF2B02F10101A8BFE2
:103EC000FF2321601370A96881F3100189B2204695
:103ED00003F0F6F9296801F30F0189B2204603F0D7
:103EE000EFF9164B22681978D5E600BF19BB002000
:103EF000404D04086766666698270020D6C60020F5
:103F00005FAF00203CBB0020107AFF1F147AFF1F18
:103F1000187AFF1F18B10020888004083DDF0308CD
:103F20004C4E040878980020EF2700204C460020D3
:103F300052BC0020844400203CBC002019400020DA
:103F4000C0270020012D7FF429AF0B680022591CE7
:103F500021601A7023685A1C22601D702268252176
:103F6000531C23602B461170CDE6522D7FF416AF03
:103F70000A68B64E531C0321236006F10C0711702A
:103F80003346062001212268551C256011702268E5
:103F9000BB4202F101012160107000F0D3809979D9
:103FA000D8790633EFE73B687A689A4240F0E980B7
:103FB000A74A20462AF0F0FEBDE60B685A1C0A60AC
:103FC0001D700B685A1C0A601D7062E6A14B0A68DE
:103FD0001B88A14DFF2BA8BFFF23511C216013702C
:103FE000A96881F3100189B2204603F069F99B4B5F
:103FF0002046198803F064F9296801F30F0189B29A
:104000002046012503F05CF92B467CE60B229449FF
:10401000204603F00DF908229249204603F008F9E2
:10402000012507229049204603F002F92B466AE653
:10403000002A3FF480AE8D4B136001252B4662E6CB
:104040000B68DFF850828A4E591C022221601A70D8
:10405000236806275A1C22601F7023680A22591CF5
:1040600021601A70236801255A1922601D70B8F862
:104070000010204603F024F9B8F80210204603F09F
:104080001FF923685A1922601F702368502259199A
:1040900021601A7023680022591921601A70318832
:1040A000204603F00DF97188204603F009F92B46EC
:1040B00029E6704B51E6704B1E78033616F0FF066A
:1040C0003FF439AE6D4B6E4F1E4403F101094FF0C2
:1040D0000A081FE0B8F1500F7FD0B8F1320F00F09E
:1040E0009980A8F13C00C0B2132840F296800025C8
:1040F000294623685A1C2260204683F8008003F07A
:10410000DFF82946204603F0DBF84E453FF413AEB6
:1041100019F8018BB8F10A0FDCD15A4B9D68196868
:1041200005EB85054FF6FF736D009D42A8BF1D4648
:104130009942A8BF194625EAE57521EAE171ADB2B9
:1041400089B2D6E7504B21681A78481C20600A7063
:10415000002A3FF4F0AD013AD2B202EB420206EB84
:1041600042025578002D3FF4E6AD01351D44013380
:10417000226813F8011F501CAB4220601170F7D168
:10418000D9E55A1C3A60197812E75A1C3A60197836
:1041900015E63B685A1C3A601B78002B01F07881C9
:1041A000102B01F080810D462268501C2060137096
:1041B000204603F06DF82946204603F069F8334B9A
:1041C0002046196803F064F82046002103F078F8CF
:1041D0000021204603F074F85BE52D4B9EE7338801
:1041E000FF2BA8BFFF23DBB225E526F03BFA002812
:1041F0003FF420AD03780A2B25D8B0F9023087FBB5
:104200000312DB17C3EBA2039BB2FF2BA8BFFF2354
:10421000DBB210E597E8220082E726F023FA0028B7
:104220003FF465AF03780A2B3FF661AFB0F9043075
:10423000B0F9061003EB830383F3500521EAE17123
:10424000ADB289B255E70023E2E700BF4C4E040847
:10425000A9DF03083CBC0020844400204446002021
:10426000908004089C800408A880040869D2010892
:1042700080270020243D002019BB0020504D040859
:10428000902700204C27002078980020BC26002092
:10429000842700201C580020212D37D13346721C62
:1042A0003A60184D13F8022B6A703B6073782B70DC
:1042B000F31C3B60B378AB70384602F0A7FF3B6855
:1042C0002881591C1A46396012F8021B69713A603C
:1042D0005B78AB7101252B4615E5731C3B60337889
:1042E0000A2B01F0DA80502B40F03F86384602F06E
:1042F0008DFF054E3080384602F088FF0125708022
:104300002B4600E54C460020802700200B3DEF2D7A
:1043100000F29F8201A050F825F000BF1B53010856
:1043200053480108534801085348010853480108FD
:1043300053480108534801085348010853480108ED
:1043400053480108534801085348010853480108DD
:1043500053480108534801085348010853480108CD
:1043600053480108534801085348010853480108BD
:10437000534801085348010853480108814D01087A
:104380005348010873530108534801085153010869
:10439000534801085348010853480108F3520108E3
:1043A000534801089952010853480108FD4C01087F
:1043B00053480108D34C010853480108C14C010877
:1043C000534801086D4C010853480108C54F0108C6
:1043D000534801085348010853480108534801084D
:1043E000373D010853480108994F01085348010817
:1043F000534801087F4F010853480108214F010825
:10440000534801085348010853480108534801081C
:10441000534801085348010853480108534801080C
:10442000E14E010853480108934E01085348010822
:1044300053480108554E01085348010853480108E4
:1044400053480108534801085348010853480108DC
:1044500053480108F14D010853480108C1510108B2
:10446000534801085751010853480108B550010845
:1044700053480108435001087B5201083552010896
:10448000534801085348010853480108534801089C
:10449000534801085348010853480108534801088C
:1044A000534801085348010853480108534801087C
:1044B000534801085348010853480108534801086C
:1044C000534801085348010853480108534801085C
:1044D000534801085348010853480108534801084C
:1044E000534801085348010853480108534801083C
:1044F000534801085348010853480108534801082C
:10450000534801085348010853480108534801081B
:10451000534801085348010853480108534801080B
:1045200053480108534801085348010853480108FB
:1045300053480108534801085348010853480108EB
:1045400053480108534801085348010853480108DB
:1045500053480108534801085348010853480108CB
:1045600053480108534801085348010853480108BB
:1045700053480108534801085348010853480108AB
:10458000534801085348010853480108534801089B
:10459000534801085348010853480108534801088B
:1045A000534801085348010853480108534801087B
:1045B000534801085348010853480108534801086B
:1045C0005348010853480108534801085152010853
:1045D00053480108574C01082D4C01085348010865
:1045E000534801085348010853480108534801083B
:1045F000534801085348010853480108534801082B
:10460000534801085348010853480108534801081A
:10461000D14B01087F4B0108434B01085348010867
:10462000A74A01088D4A0108714A01085348010848
:10463000574A0108F14901088349010871490108F5
:104640001749010853480108E9480108534801087F
:1046500053480108C74801089948010885480108DE
:104660005D4801083548010813480108E74701087B
:10467000CF4701085348010853480108534801082F
:10468000534801085348010853480108534801089A
:10469000534801085348010853480108534801088A
:1046A000534801085348010853480108B547010819
:1046B00053480108534801085D4701085348010861
:1046C0005348010853480108F746010853480108B8
:1046D0005348010853480108DD460108B34B1B78D5
:1046E000DB0700F1B6800125F7F706FEF7F7DEFFDE
:1046F0002B46FFF708BB384602F088FD3B68ADF853
:104700000C001A46591C396012F8021B3A608DF8E9
:104710000E105A788DF80F20DA1C3A609A788DF8CE
:1047200010201A1D3A60DA788DF811205A1D3A606F
:104730001B798DF8123003A80023ADF8143002F075
:10474000BFFC9B4A9B4B1268801A4FF0010561F138
:104750000001C3E906012B46FFF7D5BA731C3B6085
:1047600033780F2B75D8B21C3A60C3EBC303924A5F
:104770007178D154F11C39601344B2785A70321DEB
:104780003A60F2789A70721D3A603279DA70B21D2E
:104790003A6072791A71F21D3A60B2795A7106F173
:1047A00008023A60F2799A7101252DF011FF2B462B
:1047B000FFF7A9BA384602F029FD804EF08138464D
:1047C00002F024FD0125B0812B46FFF79CBA384644
:1047D00002F01CFD7A4A00EB8000430001251380A3
:1047E0002B46FFF790BA3246731C3B60754B12F8AC
:1047F000021B19703A6072785A70F21C3A60B278F3
:104800009A70321D3A60F278DA7001252B46FFF774
:104810007ABA384602F0FAFC6B4E3082384602F023
:10482000F5FC7082384602F0F1FC0125B0822B467F
:10483000FFF769BA3346721C3A6013F8020B3B600B
:10484000F31C71783B60B27816F044F900287FF4CD
:1048500072AA4FF0FF352B46FFF755BA3346721C4C
:104860003A605A4A13F8021B11703B60534A73783E
:104870009370F31C3B60524BB2789A7001252B4623
:10488000FFF741BA524B534918684E2201252FF0C9
:104890006FF82B46FFF737BA3246731C3B604E4B1E
:1048A00012F8021B19703A6072785A70F21C3A6062
:1048B000B2789A70384602F0A9FC484B0125D8809E
:1048C0002B46FFF720BA384602F0A0FC434E30805A
:1048D000384602F09BFC7080384602F097FC0125B8
:1048E000B0802B46FFF70FBADFF8FC8098F8003055
:1048F000002B3FF420AA3A4E0025384602F086FCF1
:1049000022F000FD98F80030A6EC010A01359D4226
:10491000F3DBFFF710BA0D2B9BD1731C3B6035788E
:10492000072D96D8DFF8C48038460C2602F06EFCBE
:1049300006FB05F608EB0605A880384602F066FC83
:10494000E880384602F062FC3B6828811A46591C10
:10495000396012F8021BA9723A605B78EB72384634
:1049600002F03CFC012548F806002B46FFF7CBB9C6
:10497000384602F04BFC1B4B012518802B46FFF7F5
:10498000C2B9731C3B603078060600F14686074BBF
:104990001B78DD073FF5CFA9032828BF002001259C
:1049A000F7F78EFC2B46FFF7AEB900BF0C91002045
:1049B00060BA0020B8240020383C00202C58002089
:1049C0003C580020484000208C5D002090AC002026
:1049D000BC460020B07404082458002054B80020BD
:1049E0009C3E00206443002019BB0020783B00203F
:1049F000731C3B60384696F8009002F0EFFB80464F
:104A0000384602F0EBFB0546384602F0E7FB064667
:104A1000384602F0FBFB384602F0F8FB384602F05D
:104A200001FCB9F1000F00F0BA85B9F1100F7FF465
:104A300082A9BF4BC3F804809D600EB1BD4B1E60C0
:104A4000BD49BE4B0222081F01251A7026F0C6FD83
:104A50002B46FFF758B9BA4B1B78D8073FF56BA91F
:104A60000125F7F7F9FFF7F721FE2B46FFF74BB9C2
:104A7000B34B1B78DA073FF55EA9B24A13780125DC
:104A800043F0040313702B46FFF73DB9AC4B1B7882
:104A9000D9073FF550A9AC4B4FF4C87201251A80D5
:104AA0002B46FFF730B9092B7FF7D3AEDFF8CC8266
:104AB0003346721CD8F800503A6013F8022B2A7063
:104AC0003B607378AB70F31C3B60B378642BA8BF7A
:104AD0006423321D6B713A60F378642BA8BF6423A2
:104AE000721DAB713A603379EB71B31D3B60737922
:104AF000642BA8BF6423F21D2B723A60B379EB706C
:104B000006F108033B60F3792B71384602F07EFB17
:104B10007A683B686881D11A00290CDD591CD8F8E5
:104B200000003960521A002A1978417203DD9A1C7C
:104B30003A605B784370012523F0DEF92B46FFF7DE
:104B4000E2B8824B1868F31C02462136991E396080
:104B500013F8031C1170591E396013F8021C5170B0
:104B60003B6013F8011C91700333B34202F103025E
:104B7000ECD1012522F070FA2B46FFF7C4B8731C64
:104B80003B6033786F4A002B00F0F684137843F0D3
:104B90000203B11C13706E4D396073782B75384663
:104BA00002F01CFB2860384602F018FB68603846AB
:104BB00002F02CFB2881384602F028FB654AE88188
:104BC0001378012543F0020313702B46FFF79BB8BF
:104BD000C3F34705122D3FF63CAEBDB10CAB0DF152
:104BE0000A0803EB45094646A9F12609384602F0B2
:104BF0000DFB26F8020F4E45F8D1574B38F8022F1F
:104C000023F8022F4645F9D1112D09D8534A6B00DC
:104C1000023B13440021223223F8021F9A42FBD1A7
:104C20004F4A01231D461370FFF76DB8731C4D49A1
:104C30003B600A783378002A40F0A38404220A708B
:104C4000494A9B001380F8F7E3FC394B01251862B1
:104C50002B46FFF758B8454E00233846336002F024
:104C6000BDFA012530602B46FFF74DB8731C3B6041
:104C700033780E2B3FF6EDADB21C3A607078032806
:104C80003FF6E7AD3A49062202FB03F28B18F51C0A
:104C900058713D60B0788854321D3A60F2785A708D
:104CA000721D3A6032799A70B21D3A607279DA7088
:104CB000F21D3A60B2791A7101252B46FFF723B82D
:104CC000731C3B602B4B32785A7501252B46FFF73E
:104CD0001AB8721C3A6035781F2D3FF6BAAD052B15
:104CE0007FF4B7AD384602F079FA234B43F825003C
:104CF000012511F051FF2B46FFF705B81E4D05F1B8
:104D00004006384602F082FA3B68A5F88000591C3C
:104D10001A46396012F8021B85F882103A605B78F7
:104D200085F883300435AE42EBD1FFF704B800BFFD
:104D3000B8240020BC260020C024002058420020B7
:104D40000C910020B84600207CCC0020BC460020FE
:104D50005061002056420020BEC70020C0C700207E
:104D6000E4C70020DEC0002044460020243D00208F
:104D7000303D0020109800209C440020C0460020B8
:104D8000731C3B6035780191132D3FF662ADB31C67
:104D90003B6070782AF03AF800283FF45AADB34BE4
:104DA000027803F82520F21C3A6003EB8505B278FF
:104DB0006A70321D3A60F278AA70721D3A603279D8
:104DC000EA7003F15000019902E00433834207D0F6
:104DD0001A78002AF9D19D78DA789542F5D2012126
:104DE000A34B81F00101012519702B46FEF78BBF03
:104DF000A04B1B68002B3EF49EAF26F0E7FCFF287B
:104E00003EF499AF384602F001FA3F2840F2DC83C5
:104E1000994E002535703B687A68B080D21A012A15
:104E20007EF789AF1A46591C396012F8021BB1701F
:104E30000CA83A6000225D7800F8242D26F098FC3A
:104E40009DF80C30AB423EF476AF284626F0B4FC19
:104E5000FEF771BF894B1B78012B3EF66CAF731CBC
:104E600031463B60DFF8448211F8023B88F802309B
:104E7000F31CD21A3960012A70783B6040F3B18389
:104E8000384602F0C3F90125A8F800002B46FEF7CA
:104E90003ABF731C3B6096F80080B8F1110F3FF6E3
:104EA000D8ACB31C3B60764D737805F818303846A3
:104EB00002F0ACF940F6CA039842A8BF184640F287
:104EC000EE23984205EB4801B8BF18460125A0F231
:104ED000EE222B46192092FBF0F24A70FEF713BF28
:104EE0003346721C674D3A6013F8022B2A713B60FF
:104EF00073786B71384602F089F93B6828805A1C38
:104F00003A601B78AB71384602F080F93B686880E4
:104F10005A1C3A601B78EB7101252B46FEF7F3BE55
:104F2000731C3B60584B3278DFF884811A70002381
:104F3000C8F80030384602F051F93A68D8F8003025
:104F40005249534D0343501CC8F800303860137861
:104F50000B72384602F05AF92860384602F056F9CA
:104F60006860384602F052F9A860384602F04EF9FF
:104F70000125384602F04AF92B46FEF7C4BE454BE0
:104F800006F1080201363E6016F8011C03F8011F05
:104F9000B242F7D1FEF7CFBE3346711C39603E49AD
:104FA00013F8020B88703B607078487093423EF4AF
:104FB000C2AEF31C3B60394BB2781A7401252B4604
:104FC000FEF7A1BE0722B3FBF2F2C2EBC2015B1AED
:104FD0007FF43FACD2B202F1FF395FFA89F9002ABF
:104FE0003EF4A9AE09F101091D46731C3B6096F918
:104FF0000060304629F0BAFB0135804600283FF4B6
:1050000028AC8670384602F001F93B68A8F8000029
:105010001A46591C396012F8021B88F803103A60CE
:105020005A7888F80420DA1C3A609A7888F80620C2
:105030001E1D3E60DB7888F80530A945D5D1FEF706
:105040007ABE3346721C3A60154A13F8021BD170BF
:105050003B60144A73785371F31C3B60124BB27877
:10506000DA7001252B46FEF74EBE00BF34C9002082
:10507000781D0020109100201491002092B0002093
:1050800044CA002070B80020405C00201098002026
:10509000C83A00200F9800204C580020B824002067
:1050A0002C5800201C5600203C58002094B00020B2
:1050B00018B10020384602F0A9F8384602F0A6F8E8
:1050C000384602F0A3F8384602F0ACF83B68B84D19
:1050D0001946581C2A68386011F8020B82F82C0017
:1050E0003960597882F83610D91C39609B7882F87B
:1050F0003730384602F096F8384602F093F83846D2
:1051000002F090F838462E6802F080F87087384632
:105110002E6802F07BF83B687A683087D11A012943
:105120000ADD591C2A6839601B7882F82E3038460F
:1051300002F078F83B687A68D31A032B09DD384609
:105140002E6802F063F8708638462E6802F05EF82A
:10515000B08628680DE5731C3B60954DDFF87882BA
:10516000337888F8053038462E6802F04FF83084DE
:1051700038462E6802F04AF87A683B68F083D11A04
:10518000072900F37282D11A032900F36182D21A2F
:10519000002A05DD591C2A6839601B7882F8263000
:1051A000F7F7DCF91EF05CFA824B1B68002B00F06D
:1051B000B9812868012521F07FFB2B46FEF7A3BDAE
:1051C0003346721C3A60DFF8108213F8022B88F81D
:1051D00002203B60784A73781370F31C3B60774D74
:1051E000B3782B71331D3B60F378092BA8BF0923DB
:1051F0003846AB7002F00AF83B687A682880D11A0A
:10520000012905DD384602F001F83B687A68E8813B
:105210009A4240F0F381F7F7A1F93B687A689A4225
:105220003EF489AD5A1C3A601B78EB7001252B4681
:10523000FEF769BD731C3B603378002B00F0A6813C
:105240004FF40040012509F04DFA2B46FEF75BBDF7
:105250003346721C3A6013F8025B3B60F31C7078B3
:105260003B60B178002D00F0D281012D7EF463AD5A
:1052700010F0C4FB2B46FEF746BD514B1B7813F0D4
:1052800001017FF4E6AA731C3B603078012510F021
:1052900005FB2B46FEF737BD731C4A4D3B60337848
:1052A0002B72384601F0B2FFA883384601F0AEFFFA
:1052B0002883384601F0AAFF3A686883531C3B6094
:1052C0001278EA747A68D31A032B00F336813B68AC
:1052D000D11A052900F3AC81D21A002A7EF72BAD32
:1052E0005A1C3A601B7885F8213001252B46FEF7C1
:1052F0000ABD731C3B60344930780870D21A002A0A
:105300007EF719ADB31C3B607378003318BF0123DF
:1053100001254B702B46FEF7F6BC2C49102B4FF0A5
:10532000000228BF10230A604A608A60CA600A74BB
:10533000002B3EF400AD3A680139134401323A6063
:1053400012F8010C01F8010F9342F7D1FEF7F3BCFC
:10535000384601F05BFF1E4E3060384601F056FFC4
:105360007060384601F052FF0125B0602B46FEF711
:10537000CABC184E00233360384601F02FFF336853
:105380000125034333602B46FEF7BDBC731C3B6015
:1053900033780A2B00F08C80384601F043FF384602
:1053A00001F040FF384601F03DFFFEF7C4BC00BFEE
:1053B000BC4600203C5C0020205800208C5D002072
:1053C0000C91002010980020405C0020085800201C
:1053D000C83A002018B1002090AC00203B687A68E1
:1053E0009A4276D1AC4BFF221A704FF00009AB4DB8
:1053F0000FF0A4F849462022A94885F800902FF024
:10540000B4FB8DF80C909DF80C30072B00F28880CF
:10541000DFF8CC82A24F4A469DF80C3003EB4303E1
:1054200008EBC3035B7CE3B19DF80C3003EB430353
:1054300008EBC30320215B699BB19DF80C3003EBA3
:10544000430308EBC303586947F8220000F0C2FF8A
:105450002B7857F8230001F07BF82A780132D2B27A
:105460002A709DF80C300133DBB28DF80C309DF8BA
:105470000C30072BD0D92368591C21601A70002EDC
:105480003EF459AC874B336001252B46FEF73BBCFD
:10549000854A92E82200FEF787BE384601F0B6FE44
:1054A000824EFEF727BF7C4A51689568FEF77CBEA6
:1054B000B31C3B607E4B72781A70F21C3A60B27873
:1054C0005A70321D3A60F2789A7001252B46FEF729
:1054D0001ABC5A1C19463A606F4811F8022B027028
:1054E00039605B784370042A03D9FF2A7EF4D1AB7C
:1054F0007BE770490978994205D8022A7EF4C9AB46
:10550000FF2B7EF4C6AB236801255A1922601D705B
:10551000002E3EF410AC684B33602B46FEF7F3BB15
:105520004A46A8E765486649664A674B0360012515
:105530000B6013602B46FEF7E6BB384601F066FEB3
:10554000A884384601F062FE3B687A68E884D11A84
:1055500003297FF7BDAE1A46591C396012F8021BA9
:10556000A9773A605B7885F82030384601F04EFE26
:105570003B687A686884ABE6137803F0FD03FFF7B5
:1055800008BB042A7EF4D7ABFFF75ABB4F4A136817
:10559000012523F4004313602B46FEF7B4BB424BB6
:1055A0001020C3F800805D6009F06CF8484A137859
:1055B00043F001031370002E3EF4BDAB454B0125B3
:1055C0001E602B46FEF79FBBC50800F007030135A0
:1055D0000133EDB2404E28461946737024F0ACFFFB
:1055E00018E43E4BB1781A88012512FB00F22B46D5
:1055F00092FBF1F2A8F80020FEF785BB5A1C3A6036
:105600001B78003318BF012388F8073003E6012513
:1056100021F0A6FB2B46FEF776BB00F07F000328A7
:1056200028BF0020012510F005FA2B46FEF76BBBC2
:105630005A1C3A601B78EB72384601F0CFFD3B688C
:10564000E8605A1C3A601B782B743B687A6843E622
:10565000384601F0DBFDA8F80E00384601F0D6FD13
:105660003B687A68A8F8100091E5384601F0CEFD55
:10567000A8F80A00384601F0C9FDA8F80C00384621
:105680002E6801F0C3FD708438462E6801F0BEFD1F
:105690003B687A68B08476E5B8240020513E00204B
:1056A000BCC800209D1302084C4200201C5800205A
:1056B0005FAF002019BB002075D20108F8B20020AE
:1056C0004CB300204CB70020215B0108B4460020F9
:1056D000B8460020BC260020149100204A56002025
:1056E000F4AD002003682DE9F041DF691FB13B46AE
:1056F000BDE8F0411847002A164611DD04460D4664
:105700000E4400E023689B68204698470028F9D0A3
:10571000236815F8011B1B6820469847AE42F1D15B
:10572000BDE8F08100232522027043708370C370AE
:105730007047152303701623C370172383713A2310
:1057400083703B2343713C2303727047002870B57C
:105750001EDB0928044620DD012303EB83035B00E5
:10576000B0FBF3F2092AF8D87BB10E4EB4FBF3F08C
:105770000928CCBF57223022A6FB03E5024403FBD5
:105780001044EB0801F8012BF0D100230B7070BD21
:105790002D230B7040420131DBE7303001F8010B63
:1057A000F3E700BFCDCCCCCC884230B44FF001043D
:1057B0002ED301FB04F4B0FBF4F58D42F9D284B191
:1057C000AAB901E0B0FBF4F5092DCCBF5722302275
:1057D0002A4404FB150003F8012BB4FBF1F4002C60
:1057E000F0D100221A7030BC7047B0FBF4F5092DDF
:1057F000CCBF372230222A4404FB150003F8012BCA
:10580000B4FBF1F4002CF0D100221A7030BC7047C8
:105810000546002AEBD1D7E72DE9F04714461D468F
:10582000064600234FF47A72204629462DF0DEFD0D
:10583000DFF840814B4A4C4F88FB00310144C317CD
:1058400082FB002EC3EB611188FB012887FB002738
:105850008644464AC3EBEE2EC1EB011C82FB0E29A7
:10586000A0EB8C0C0744424A86F806C0C3EB2747DE
:105870004FEAEE7C08EB010ACCEBA90C82FB078215
:105880004FEAE1780CEB4C0CC8EB6A18AEEBCC0E8F
:10589000C8EB0818DFF8E0C086F804E0A1EB880147
:1058A00071718CFB0010F917C1EBE21240F2B55197
:1058B00001FB1272C3EBE050B2F5896F4FEA80072B
:1058C0003CDA40F2DA239A4242DCB2F5B77FB4BF49
:1058D0004FF0000C4FF0010C4FEA4C09DFF89C80B0
:1058E00009EB0C0308EBC3031FFA8CFED88A09EB03
:1058F0000C0108EBC10116310B2301E031F8020D58
:10590000824218DA013BF9D1CC44012338F83C003B
:10591000B37007F2B2770132121ABE44F270A6F8E1
:1059200000E0204629464FF47A7200232DF05EFDF8
:105930003281BDE8F0870133DBB2E9E74FF0030EB7
:10594000F44640F29650DFF834804FF00609CEE777
:105950004FF0020EDFF82480F44640F229404FF069
:105960000409C4E7C5B3A29107452EC2ABAAAA2A6F
:1059700073B06D1689888888792D0311604D0408ED
:1059800003685A1C02601970704700BF2DE9F04788
:10599000089C2578002B804689460CBF4FF0200AD2
:1059A0004FF0300A661C35B3002A29DD334601E08A
:1059B000024698B113F8011B501E0029F8D1971E1A
:1059C00060B13D46013D51464046C8476B1C002B27
:1059D000F8DC257827EAE770013055B1041B294629
:1059E0004046C847301916F8015B002DF7D1BDE8D5
:1059F000F087BDE8F087002A04DC2846BDE8F08780
:105A00000020EBE7571EDCE783684268D0ED037A9D
:105A100000EB83010133934281ED040A836004BFEC
:105A20000023836000EB830393ED047A036870EE38
:105A3000277A9A42C0ED037A77EEC77AC0ED037AEF
:105A40000CDA013307EE103AF8EEC76AB7EE007AC7
:105A500087EEA60A036030EE070A704707EE102AA9
:105A6000B8EEC77A87EE870A704700BF90ED057AD7
:105A700090ED004AD0ED066AD0ED014AD0ED047AEF
:105A800090ED035AD0ED025AA4EE007AB0EE406ACF
:105A9000B0EE470AB0EE667AA6EE247A67EEC07AD8
:105AA000A0EE457AE6EE257A80ED057AC0ED067A1D
:105AB000704700BFD0ED057A90ED013AD0ED003A85
:105AC000D0ED064A90ED024A90ED077A90ED035A28
:105AD00090ED086AD0ED045AC0ED067AF0EE406A07
:105AE00027EE830AC0ED056AA3EEA60A80ED087AC8
:105AF000A4EE240AA5EE470AA5EEC60A80ED070A21
:105B0000704700BFD0ED007A90ED017A30EE670A61
:105B1000E7EE007AB0EE670AC0ED007A704700BF8A
:105B2000704700BF0A44914214D030B40139551E69
:105B300041F2210211F8014F082380EA04200404F5
:105B40004CBF82EA40004000013B80B2F7D18D4259
:105B5000F0D130BC704700230122436083600360B2
:105B600003714370C2718372837043710272C37296
:105B70007047F8B50468C4F30D0405460E4604B337
:105B80002F681CF043FA092840F08880454C2369AF
:105B900023F440732361236943F400732361236971
:105BA00043F0010323613E601CF030FA23690928A9
:105BB00023F00103236171D12B6804332B60002093
:105BC000F8BD394B394A93422BD902F580429342B2
:105BD00026D902F5804293422AD902F580429342A7
:105BE00028D902F58032934226D902F50032934239
:105BF00024D902F50032934222D902F500329342B1
:105C000020D902F5003293421ED902F58022934238
:105C10001CD9B3F1016F1BD30520F6F777FBFBE727
:105C200008241CF0F3F9092814D04FF0FF30F8BD18
:105C30001024F6E71824F4E72024F2E72824F0E7FC
:105C40003024EEE73824ECE74024EAE74824E8E78C
:105C50005824E6E7134F3B6923F440733B613B69EB
:105C600043F400733B613B6923F0F8033B613B69FC
:105C700043F002031C433C613B6943F480333B61C6
:105C80001CF0C4F93B6923F002033B613B6909281E
:105C900023F0F8033B613FF473AFC6E76FF00100F8
:105CA000F8BD00BF003C024000400008FF3F000874
:105CB000F8B504460D468E180027B54201D120697B
:105CC000F8BDE368591CE160234415F8012B1A72F2
:105CD0000429F2D1206918B9A1682046FFF749FFCD
:105CE0002061E760E9E700BF03682DE9F041DF6963
:105CF0001FB13B46BDE8F0411847002A164611DDAA
:105D000004460D460E4400E023689B6820469847F1
:105D10000028F9D0236815F8011B1B682046984716
:105D2000AE42F1D1BDE8F08103689B69184700BF1E
:105D300003685B69184700BF03681B69184700BF09
:105D40000368DB68184700BF03689B68184700BFFB
:105D500003685B68184700BF03681B68184700BFEB
:105D6000014B1868F8E700BF841F002038B50C46C7
:105D7000097849B1054601342B6828461B689847C5
:105D800014F8011B0029F7D138BD00BF064B53F8AA
:105D900020302BB11A689B8851690B4201D11383C3
:105DA00070475383704700BF2CBA002003682DE969
:105DB000F04F03F13F4404F57E04604EA40A012530
:105DC000345D04F01F066409032C05FA06F500F0A3
:105DD000AF80042C00F0A780022C54D08588B5FA3F
:105DE00085F0C0F11F0080B2C40803EB840400F00A
:105DF0000700266A80000F27874026EA07062662EA
:105E0000276A01F0030602FA00F0721E3843012AE5
:105E1000C1F3810CC1F300182062C1F3411137D9DD
:105E20000024224601274FF0030E03E0102A04F15C
:105E3000020426D007FA02F0A84302F10102F5D1CC
:105E4000D3F800C00EFA04F0C04300EA0C0CC3F80B
:105E500000C0D3F8008006FA04FC4CEA080CC3F832
:105E600000C0D3F80CC000EA0C00D860D3F80CC016
:105E700001FA04F040EA0C00102AD86004F1020490
:105E8000D8D1BDE8F08F2E4C666C35436564A5E72C
:105E9000002002464FF0010E4FF0030904E00132EA
:105EA000102A00F102003CD00EFA02F737EA05048E
:105EB000F5D1D3F800A009FA00F4E4430AEA040A91
:105EC000C3F800A0D3F800B006FA00FA4AEA0B0AB9
:105ED000C3F800A0D3F808A004EA0A0AC3F808A08F
:105EE000D3F808B00CFA00FA4AEA0B0AC3F808A083
:105EF000D3F804A02AEA07075F60D3F804A008FAE1
:105F000002F747EA0A075F60DF683C40DC60DF6851
:105F100001FA00F401323C43102ADC6000F1020077
:105F2000C2D1BDE8F08F064C266B3543256355E79B
:105F3000034C266C3543256450E700BF0075040808
:105F400000380240026802F13F4303F57E032DE969
:105F5000F04F9B0A544DEB5C03F01F055B090124D5
:105F6000032B04FA05F400F09980042B00F09180D3
:105F7000022B3ED001F00306731E012BC1F3810CEE
:105F8000C1F300188588C1F3411137D90024234695
:105F900001274FF0030E03E0102B04F1020426D07A
:105FA00007FA03F0A84303F10103F5D1D2F800C0CA
:105FB0000EFA04F0C04300EA0C0CC2F800C0D2F89C
:105FC000008006FA04FC4CEA080CC2F800C0D2F8C3
:105FD0000CC000EA0C00D060D2F80CC001FA04F04A
:105FE00040EA0C00102BD06004F10204D8D1BDE8C7
:105FF000F08F2E4B5D6C2C435C64BBE700200346A6
:106000004FF0010E4FF0030904E00133102B00F1B3
:1060100002003CD00EFA03F737EA0504F5D1D2F8B6
:1060200000A009FA00F4E4430AEA040AC2F800A056
:10603000D2F800B006FA00FA4AEA0B0AC2F800A049
:10604000D2F808A004EA0A0AC2F808A0D2F808B0F8
:106050000CFA00FA4AEA0B0AC2F808A0D2F804A027
:106060002AEA07075760D2F804A008FA03F747EABC
:106070000A075760D7683C40D460D76801FA00F43B
:1060800001333C43102BD46000F10200C2D1BDE8C3
:10609000F08F064B1D6B2C431C636BE7034B1D6C91
:1060A0002C431C6466E700BF0075040800380240FA
:1060B00010B50409013C032C17D80D4B33F81420FC
:1060C00000F00F0042FA00F313F001030DD001239A
:1060D00003FA00F0013810402DF0D8F9054A064BBC
:1060E000125D104403EBC00010BD002010BD00BFC6
:1060F0008C76040888760408A0B800202DE9F04FBB
:106100004A484B494B4B4C4C4FF0010A4FF00209A7
:106110004FF004084FF0080C4FF0100E20274026D7
:10612000802530F8022B12F0010F03D01960A3F87C
:1061300004A0083312F0020F03D01960A3F80490F2
:10614000083312F0040F03D01960A3F80480083359
:1061500012F0080F03D01960A3F804C0083312F03E
:10616000100F03D01960A3F804E0083312F0200FD9
:1061700002D019609F80083312F0400F02D01960DE
:106180009E80083312F0800F02D019609D80083382
:1061900012F4807F05D04FF4807B1960A3F804B01F
:1061A000083312F4007F05D04FF4007B1960A3F888
:1061B00004B0083312F4806F05D04FF4806B19607F
:1061C000A3F804B0083312F4006F05D04FF4006B4D
:1061D0001960A3F804B0083312F4805F05D04FF4BF
:1061E000805B1960A3F804B0083312F4005F05D097
:1061F0004FF4005B1960A3F804B0083312F4804F29
:1062000005D04FF4804B1960A3F804B00833D20BCB
:1062100004D04FF4004219609A80083301F5806180
:10622000A1427FF47EAFBDE8F08F00BF8C760408FA
:1062300000000240A0B800200010024000286AD0F0
:1062400003682DE9F04F03F13F4404F57E045F4EEF
:10625000A40A0125345D04F01F066409032C05FA25
:1062600006F559D0042C00F0AC80022C59D085885A
:10627000B5FA85F0C0F11F0080B2C40803EB8404B6
:1062800000F00700266A80000F27874026EA0706ED
:106290002662276A01F003068240701E3A430128F5
:1062A000C1F3810CC1F300182262C1F341113DD941
:1062B0000024224601274FF0030E03E0102A04F1C8
:1062C000020426D007FA02F0A84302F10102F5D138
:1062D000D3F800C00EFA04F0C04300EA0C0CC3F877
:1062E00000C0D3F8008006FA04FC4CEA080CC3F89E
:1062F00000C0D3F80CC000EA0C00D860D3F80CC082
:1063000001FA04F040EA0C00102AD86004F10204FB
:10631000D8D1BDE8F08F70472D4C266C35432564ED
:10632000A5E72B4C666C35436564A0E70020024668
:106330004FF0010E4FF0030904E00132102A00F182
:1063400002003CD00EFA02F737EA0504F5D1D3F883
:1063500000A009FA00F4E4430AEA040AC3F800A022
:10636000D3F800B006FA00FA4AEA0B0AC3F800A014
:10637000D3F808A004EA0A0AC3F808A0D3F808B0C2
:106380000CFA00FA4AEA0B0AC3F808A0D3F804A0F2
:106390002AEA07075F60D3F804A008FA02F747EA81
:1063A0000A075F60DF683C40DC60DF6801FA00F4E8
:1063B00001323C43102ADC6000F10200C2D1BDE88A
:1063C000F08F034C266B3543256350E700750408B6
:1063D00000380240002855D0026802F13F4303F51F
:1063E0007E032DE9F04F9B0A544DEB5C03F01F0533
:1063F0005B090124032B04FA05F444D0042B00F0BC
:106400009780022B44D001F00306731E012BC1F3C9
:10641000810CC1F300188588C1F341113DD90024D6
:10642000234601274FF0030E03E0102B04F1020472
:1064300026D007FA03F0A84303F10103F5D1D2F8FF
:1064400000C00EFA04F0C04300EA0C0CC2F800C011
:10645000D2F8008006FA04FC4CEA080CC2F800C02E
:10646000D2F80CC000EA0C00D060D2F80CC001FADF
:1064700004F040EA0C00102BD06004F10204D8D1E3
:10648000BDE8F08F70472E4B1D6C2C431C64BAE79F
:106490002B4B5D6C2C435C64B5E7002003464FF04A
:1064A000010E4FF0030904E00133102B00F102004C
:1064B0003CD00EFA03F737EA0504F5D1D2F800A074
:1064C00009FA00F4E4430AEA040AC2F800A0D2F888
:1064D00000B006FA00FA4AEA0B0AC2F800A0D2F8A5
:1064E00008A004EA0A0AC2F808A0D2F808B00CFA18
:1064F00000FA4AEA0B0AC2F808A0D2F804A02AEA75
:1065000007075760D2F804A008FA03F747EA0A071A
:106510005760D7683C40D460D76801FA00F4013373
:106520003C43102BD46000F10200C2D1BDE8F08FD3
:10653000034B1D6B2C431C6365E700BF007504080B
:106540000038024010B1036882885A83704700BF48
:1065500010B1036882881A83704700BF18B10368BE
:10656000828809B95A8370471A83704710B40A4B5E
:106570000A4A1C7801238340234052F8200029B99D
:10658000B3FA83F149095DF8044BE7E7191C18BF1A
:1065900001215DF8044BE1E728BA00202CBA002065
:1065A00030B1036882881B691A4214BF01200020A1
:1065B000704700BF2DE9F0410B4E346873691C40F1
:1065C0000FD0DFF828800127B4FA84F3C3F11F034A
:1065D00007FA03F558F8230003689847AC43756140
:1065E000F2D1BDE8F08100BF003C014068BA002054
:1065F0002DE9F0410B4E346873691C400FD0DFF871
:1066000028800127B4FA84F3C3F11F0307FA03F5C6
:1066100058F8230003689847AC437561F2D1BDE890
:10662000F08100BF003C014068BA00202DE9F04134
:106630000B4E346873691C400FD0DFF828800127A7
:10664000B4FA84F3C3F11F0307FA03F558F82300E3
:1066500003689847AC437561F2D1BDE8F08100BF93
:10666000003C014068BA00202DE9F0410B4E34682F
:1066700073691C400FD0DFF828800127B4FA84F337
:10668000C3F11F0307FA03F558F82300036898477E
:10669000AC437561F2D1BDE8F08100BF003C014020
:1066A00068BA00202DE9F0410B4E346873691C4034
:1066B0000FD0DFF828800127B4FA84F3C3F11F0359
:1066C00007FA03F558F8230003689847AC4375614F
:1066D000F2D1BDE8F08100BF003C014068BA002063
:1066E0002DE9F0410B4E346873691C400FD0DFF880
:1066F00028800127B4FA84F3C3F11F0307FA03F5D6
:1067000058F8230003689847AC437561F2D1BDE89F
:10671000F08100BF003C014068BA00202DE9F04143
:106720000B4E346873691C400FD0DFF828800127B6
:10673000B4FA84F3C3F11F0307FA03F558F82300F2
:1067400003689847AC437561F2D1BDE8F08100BFA2
:10675000003C014068BA0020084A094808B5536C5B
:1067600043F480435364002140222EF0FEF9054B90
:106770004FF0FF321A60C3F8032008BD0038024012
:1067800068BA0020A8BA00202DE9F0410446184656
:106790000D46164698462CF07FF92768E672284485
:1067A000A07229467D69434632462046AC46BDE884
:1067B000F0416047036810B504461B68984723689A
:1067C00020469B689847A37B0133A37310BD08B58F
:1067D000FFF76EFC38B12D2282710022C271202198
:1067E000BDE80840F6E508BD0B4B984206D0A3F57E
:1067F000744398420DD04FF0FF3070470022074B92
:1068000003EB02135A89013292B25A81588980B23D
:1068100070470222F3E700BF003001406C5C0020AB
:106820002DE9F0410678012E82B005464CD0022EAB
:1068300052D1806841F0800110B104688088608383
:10684000686840F2E93402E0002C00F09980068983
:10685000013C16F0020FA4B2F6D089B2818140F259
:10686000E93102E0002900F08B800489013914F03D
:10687000010F89B2F6D0818981894FF0000C4FF465
:106880007A714FF6FF764FF0FF0E634502D129E093
:10689000B14225D004890139A70789B2F8D5A0F8FB
:1068A0000CE04FF47A7102E0B9B2B14218D0048919
:1068B000E40701F1FF37F7D58489A4B20AB1147057
:1068C00001320CF1010CE0E790F904E0BEF1FF3F6A
:1068D00002D0BEF1030F0FDD002002B0BDE8F08151
:1068E000FFF782FFAB68002B5CD01A689B8813838C
:1068F000012002B0BDE8F0814FEACE08DFF8ACC05D
:1069000008EB0E070CEB870778680028E5D06C7958
:106910003A6264000025E4B2BC75F9757D76BE76F6
:106920003B767E753D758388FA61990514D403889A
:10693000DA050CD44FF4805401E0013C28D00388E0
:106940009B05FAD403889BB243F480730380838849
:106950009BB243F440738380F0440CEB88024FF405
:10696000805401E0013C13D0537D002BFAD10CEB95
:10697000880898F8144084F0010002B0BDE8F08166
:106980008DE80C00FFF730FF68689DE80C0073E7A6
:10699000054A1388013370469BB21380F3F75CFD00
:1069A00020469AE7012098E7703B0020503A0020EB
:1069B0000378012B46D0022B42D12DE9F0418368A8
:1069C00001F07F0113B11C689B886383054617465D
:1069D000406840F2E93401E0002C3AD00689013CDD
:1069E00016F0020FA4B2F7D089B2818140F2E931EA
:1069F00000E071B30389013913F0010F89B2F8D0B7
:106A0000838940F2E93100E039B30489013914F097
:106A1000020F89B2F8D0BFB2878140F2E93300E0BB
:106A2000DBB10289013B12F0010F9BB2F8D08389E0
:106A3000AB68ABB11A689B8813830120BDE8F08175
:106A40000020704713460A46417990F90400F3F795
:106A5000DDBEFFF7C9FE6868D3E7FFF7C5FEE7E7CD
:106A60000120BDE8F08100BF427A02B9704710B53D
:106A700004460368406804F10A01984700236372E2
:106A800010BD00BF437A5A1C0344D2B242729972BD
:106A9000037A934200D802B9704710B504460368E0
:106AA000406804F10A0198470023637210BD00BFDB
:106AB00050B30123302803FA01F122D0312820D02D
:106AC00032281ED033281CD034281ED035281CD0A4
:106AD00020281AD0212818D0102812D0112810D020
:106AE00012280ED013280CD014280ED015280CD044
:106AF000162801D0172806D111F0030018BF012075
:106B000070474A0703D1002070478B07FBD0012054
:106B1000704700BF302829D0312829D0322829D009
:106B2000332829D0342829D0352829D0202829D025
:106B3000212829D0102829D0112829D0122829D07D
:106B4000132829D0142829D0152829D0162805D093
:106B5000172808BF0F2302D0002070470E23114AC8
:106B600003EB4303134493F8620070470023F6E7F6
:106B70000123F4E70223F2E70323F0E70423EEE71F
:106B80000523ECE70623EAE70723E8E70823E6E71F
:106B90000923E4E70A23E2E70B23E0E70C23DEE71F
:106BA0000D23DCE7604D040870B5448806460D46A9
:106BB000C4F30B042246002128462DF0D6FF33698A
:106BC000094A934209D3094A934206D222462846EB
:106BD0001946BDE870402CF0CBBE23B121462846B3
:106BE000BDE87040184770BD400600084207000825
:106BF000064B07498B4202D30023184670471A8878
:106C0000C2F30B029042F8D01433F3E7900100086E
:106C100040060008024A136823EA0000106070472B
:106C200018B10020F8B5174D2B78A52B28D16B781B
:106C3000BE2B25D1022229464FF6FF70FEF772FFC8
:106C4000114FAC1C22884AB1A618BE4218D2052AA0
:106C500016D92146FEF766FF3446F3E721460222A5
:106C6000FEF760FF0222A118FEF75CFF0634074B17
:106C7000641B1C8041F60F53C31A58425841F8BD9B
:106C80000020F8BD0040000800800008723B002092
:106C90002DE9F04FDFF84C914D4F8BB00326A7EB59
:106CA00009071822002104A82DF05FFF494BCDF8F9
:106CB000109005971A69002A04DA474A5A6002F1CF
:106CC00088325A6001228DF82420F322DA60434B87
:106CD000434C1B88ADF800300222694604A8FEF739
:106CE000E7FF022269464FF6FF70FEF71BFFDFF851
:106CF000F8A080464FF0000B544539D30AAC00256C
:106D000024F8245D0222214604A8FEF7D1FF0222C6
:106D100021464046FEF706FF40BAC043ADF80800E2
:106D2000022202A904A8FEF7C3FF079878B106ABB8
:106D3000C0F10402294618442DF017FF089818B92D
:106D4000069904A8FEF715FF0023089007939DF805
:106D50002430089A23B11F490B6943F000430B61AB
:106D6000013E2DD0002A9CD1FFF75CFF50B32CE0F0
:106D700065888DF80DB0C5F30B05AB1DADF8083077
:106D80002388C3F30B02ADF80A201B0B062202A9CD
:106D900004A88DF80C30FEF78BFF062202A94046AE
:106DA000FEF7C0FE616880462A4604A8FEF780FF11
:106DB000616840462A46FEF7B5FE143480469BE7DC
:106DC000002AD1D00520F5F7A1FA0BB0BDE8F08F6D
:106DD00000800008003C024023016745F04D040894
:106DE0009001000800400008400600080378202BAE
:106DF000024600F10100F9D0092BF7D02D2B2CD041
:106E00002B2B03BF5378B7EE000A0246B7EE000AF9
:106E1000A3F13001C8B209289FED467A10D8F2EEEE
:106E2000046A07EE901AF8EEE77A12F8013FE7EEEF
:106E3000267AA3F13001C8B20928B0EE677AF0D9FA
:106E40002E2B4CD003F0DF03452B0BD0F7EE007A4E
:106E500067EE276A20EE260A70475378BFEE000AD5
:106E60000246D5E710B451782D2959D02B290ABFF5
:106E70009178501C901C0024A1F13003092B53D8A9
:106E8000002303EB830301EB430310F8011FA1F17F
:106E90003002092AA3F13003F3D9B3F59A7F28BF52
:106EA0004FF49A73072B42D9DFED236A1A46F7EEA7
:106EB000007A083A072A67EEA67AFAD803F00703A1
:106EC0002BB1F2EE046A013B67EEA67AFBD124B344
:106ED000C7EE276A5DF8044B20EE260A7047537808
:106EE000A3F13001C8B2092802F10102AAD8F2EEDA
:106EF000046AF0EE665A07EE901AF8EEE77A12F896
:106F0000013F87EEA66AA3F13001C8B2092866EEF8
:106F1000A56A37EE067AEED994E767EE276AD9E7D5
:106F2000901C91780124A7E7F7EE007ACFE7F7EEFF
:106F3000007AC5E70000000020BCBE4CB5EEC00AD8
:106F4000DFED317AF1EE10FACCBF30EE270A30EEE9
:106F5000670ADFED2E7A20EE270A30B5FDEEC07A03
:106F600087B017EE904A054684EAE470002303A92F
:106F7000A0EBE47001930093029318F00FF8002C3B
:106F8000ACBF20232D2303A88DF800302BF084FD07
:106F9000012803A924D002282DD0032805BF3023BF
:106FA000684668468DF801302DF0E7FD68462BF005
:106FB00073FD0338C4B22246694628462DF014FEFC
:106FC00000232B5528462BF067FD2E22431C2A5404
:106FD0000DEB0401E8182DF0EDFD284607B030BD9B
:106FE000302368468DF801308DF802308DF803307B
:106FF0002DF0C3FDDAE7302368468DF801308DF8B7
:1070000002302DF0BAFDD1E76F12033A00007A4446
:107010002DE9F041064615460846B6FBF2F43CB9A8
:1070200005FB1464124B1B5D00F8013BBDE8F081C9
:10703000B4FBF2F767B90E4B05FB174705FB146469
:10704000DA5D00F8012B1B5D00F8013BBDE8F08123
:10705000B7FBF2F8B8F1000F02D04046FFF7D8FFB7
:1070600005FB1878024B13F8082000F8012BE3E722
:10707000B4800408104B2DE93048D3E9004554EAA8
:1070800005020BD103460122002018715871987136
:107090009A70DA7018801881BDE83088074B1A683A
:1070A00014EB020B45F1000C5A466346FEF7B4FBA5
:1070B0000120BDE8308800BFD024002060BA002045
:1070C000F0B402888578154FC37804794179A2F22B
:1070D000B27202F0030606EB4606013D05EB86059B
:1070E000013B37F815608579008940F2B557920861
:1070F00007FB0232931903EB430304EBC303C3EB17
:10710000031301EB8303C3EB031305EB830300219C
:107110004FF47A72C2FB0301F0BC7047604D040863
:10712000FAB170B48E18044603E0101A14D1B142BB
:1071300014D014F8012BA2F14103192B11F8013BD3
:10714000A3F1410598BF2032192D03F12000ECD99D
:10715000D01A01D1002BEAD170BC7047002070BC5E
:1071600070471046704700BF4FF0FF32FFF7D8BF9F
:10717000A0F16103192B98BF20387047A0F141039B
:10718000192B98BF20307047202805D009380428D3
:107190008CBF0020012070470120704761381928FA
:1071A0008CBF002001207047413819288CBF002077
:1071B00001207047303809288CBF0020012070471B
:1071C000A0F13003092B07D920F0200041381928FD
:1071D0008CBF0020012070470120704730B4026846
:1071E0001146531C036011F8024B0160D31C517807
:1071F00003609378151D05601B0443EA0123D078D2
:10720000234343EA006030BC704700BF0368591C49
:107210001A46016012F8021B0260587841EA002009
:10722000704700BF03685A1C02601878704700BF9F
:1072300038B50446006815462CF09AFB22682A44AB
:10724000226038BD036810B40A0E5C1C04601A701A
:1072500003680A0C5C1C04601A7003680A0A5C1C50
:1072600004601A7003685A1C026019705DF8044BC0
:10727000704700BF036810B40A0A5C1C04601A70EF
:1072800003685A1C026019705DF8044B704700BF18
:1072900003685A1C026010B4197003680A0A5C1C67
:1072A00004601A7003680A0C5C1C04601A7003689E
:1072B000090E5A1C026019705DF8044B704700BF3C
:1072C00003685A1C026019700368090A5A1C02609C
:1072D000197070472DE9F047002488B080460F46AA
:1072E0001E46A14605AD531C0393117839B32529D9
:1072F00033D1931CCDF810900393507830284ED0A2
:107300004FF0000AA0F13003DBB2092B42D96C2800
:1073100019D0642800F0938024D825281CD063D984
:10732000582876D063281BD131784046B847039A55
:10733000531C03931178043601340029D7D1204619
:1073400008B0BDE8F087039B5A1C03921B78642B9E
:107350007CD02AD8252B54D1252140460134B8476A
:10736000039AC0E7732833D044D975284FD106F16A
:10737000040E30682B4600220A217646FEF714FAE6
:10738000049A0095534639464046FEF7FFFA039AA1
:107390000444A8E704AA03A917F0DCFDB7E7D31C4F
:1073A000039390784FF0010AACE7732B10D05BD9B0
:1073B000752B3AD0782B96D1A3F15802B2FA82F20B
:1073C000306852092B4610210436FEF7EDF9D7E755
:1073D0003368049A0093394600234046FEF7D6FAF4
:1073E00004360444039A7EE70028B9D1204608B049
:1073F000BDE8F0876E28B3D1039A336804361C6069
:1074000071E72AD9582BD7D0632B8DD06BE778281A
:10741000A6D1A0F15802B2FA82F2306852092B4686
:107420001021FEF7C1F90436AAE706F1040E306810
:107430002B4600220A217646FEF7B6F9A0E7331D57
:10744000306829461E46FEF781F999E7331D3068FA
:1074500029461E46FEF77AF992E7002B7FF443AFE8
:10746000204608B0BDE8F0876E2BC6D03BE700BFD2
:107470000EB400B584B005AB019053F8042B064957
:10748000039301A8FFF726FF019B00221A7004B0A6
:107490005DF804EB03B07047815901082DE9F0470E
:1074A000484BB3F900708CB00646002F56D13D46CC
:1074B0003C460A8840F2B1739A4203D98B78581E31
:1074C0000B282FD9002301201946ADF824308DF860
:1074D00028308DF829308DF82A30ADF82C309C46B4
:1074E0009A4699461A46984686468DF826008DF8A3
:1074F00027000346002CACBF2B242D2404910795B4
:107500000697CDF80CC0CDF808A0CDF80490CDF8C2
:1075100000E0304605942C49FFF7AAFF40460CB026
:10752000BDE8F08791F803E00EF1FF301E28C9D8BE
:1075300091F80490B9F1170FC4D891F805A0BAF1E9
:107540003B0FBFD891F806C0BCF13B0FBAD80989F0
:10755000B1F57A7FB6D24FF00108CBE71B4C84FB24
:107560000734E319FC17C4EB6314C4EB0415A7EB51
